Component: ARM Compiler 5.06 update 1 (build 61) Tool: armlink [4d35a8]

==============================================================================

Section Cross References

    client_handling.o(i.client_find) refers to client_handling.o(.bss) for .bss
    client_handling.o(i.client_handling_ble_evt_handler) refers to client_handling.o(i.client_find) for client_find
    client_handling.o(i.client_handling_ble_evt_handler) refers to client_handling.o(i.__ARM_common_switch8) for __ARM_common_switch8
    client_handling.o(i.client_handling_ble_evt_handler) refers to device_manager_central.o(i.dm_security_setup_req) for dm_security_setup_req
    client_handling.o(i.client_handling_ble_evt_handler) refers to app_error.o(i.app_error_handler) for app_error_handler
    client_handling.o(i.client_handling_ble_evt_handler) refers to ble_db_discovery.o(i.ble_db_discovery_on_ble_evt) for ble_db_discovery_on_ble_evt
    client_handling.o(i.client_handling_ble_evt_handler) refers to client_handling.o(.bss) for .bss
    client_handling.o(i.client_handling_count) refers to client_handling.o(.data) for .data
    client_handling.o(i.client_handling_create) refers to memcpya.o(.text) for __aeabi_memcpy
    client_handling.o(i.client_handling_create) refers to ble_db_discovery.o(i.ble_db_discovery_start) for ble_db_discovery_start
    client_handling.o(i.client_handling_create) refers to app_error.o(i.app_error_handler) for app_error_handler
    client_handling.o(i.client_handling_create) refers to client_handling.o(.bss) for .bss
    client_handling.o(i.client_handling_create) refers to client_handling.o(.data) for .data
    client_handling.o(i.client_handling_destroy) refers to client_handling.o(.bss) for .bss
    client_handling.o(i.client_handling_destroy) refers to client_handling.o(.constdata) for .constdata
    client_handling.o(i.client_handling_destroy) refers to client_handling.o(.data) for .data
    client_handling.o(i.client_handling_dm_event_handler) refers to client_handling.o(i.notif_enable) for notif_enable
    client_handling.o(i.client_handling_dm_event_handler) refers to client_handling.o(.bss) for .bss
    client_handling.o(i.client_handling_init) refers to app_error.o(i.app_error_handler) for app_error_handler
    client_handling.o(i.client_handling_init) refers to ble_db_discovery.o(i.ble_db_discovery_init) for ble_db_discovery_init
    client_handling.o(i.client_handling_init) refers to ble_db_discovery.o(i.ble_db_discovery_evt_register) for ble_db_discovery_evt_register
    client_handling.o(i.client_handling_init) refers to client_handling.o(.constdata) for .constdata
    client_handling.o(i.client_handling_init) refers to client_handling.o(.data) for .data
    client_handling.o(i.client_handling_init) refers to client_handling.o(.bss) for .bss
    client_handling.o(i.client_handling_init) refers to client_handling.o(i.db_discovery_evt_handler) for db_discovery_evt_handler
    client_handling.o(i.client_handling_init) refers to client_handling.o(i.db_discovery_acc_evt_handler) for db_discovery_acc_evt_handler
    client_handling.o(i.db_discovery_acc_evt_handler) refers to client_handling.o(i.client_find) for client_find
    client_handling.o(i.db_discovery_acc_evt_handler) refers to app_error.o(i.app_error_handler) for app_error_handler
    client_handling.o(i.db_discovery_acc_evt_handler) refers to client_handling.o(.bss) for .bss
    client_handling.o(i.db_discovery_acc_evt_handler) refers to client_handling.o(.data) for .data
    client_handling.o(i.db_discovery_evt_handler) refers to client_handling.o(i.client_find) for client_find
    client_handling.o(i.db_discovery_evt_handler) refers to client_handling.o(i.notif_enable) for notif_enable
    client_handling.o(i.db_discovery_evt_handler) refers to client_handling.o(.bss) for .bss
    client_handling.o(i.db_discovery_evt_handler) refers to client_handling.o(.data) for .data
    client_handling.o(i.notif_enable) refers to app_error.o(i.app_error_handler) for app_error_handler
    client_handling.o(i.print_client_data) refers to printfa.o(i.__0sprintf) for __2sprintf
    client_handling.o(i.print_client_data) refers to debug_util.o(i.debug_printf) for debug_printf
    client_handling.o(i.print_client_data) refers to client_handling.o(.bss) for .bss
    client_handling.o(i.print_client_data) refers to client_handling.o(.data) for .data
    client_handling.o(i.print_client_data) refers to client_handling.o(.conststring) for .conststring
    client_handling.o(i.read_acc_other_device) refers to client_handling.o(.bss) for .bss
    main.o(i.assert_nrf_callback) refers to app_error.o(i.app_error_handler) for app_error_handler
    main.o(i.ble_evt_dispatch) refers to device_manager_central.o(i.dm_ble_evt_handler) for dm_ble_evt_handler
    main.o(i.ble_evt_dispatch) refers to client_handling.o(i.client_handling_ble_evt_handler) for client_handling_ble_evt_handler
    main.o(i.ble_evt_dispatch) refers to main.o(i.on_ble_evt) for on_ble_evt
    main.o(i.ble_stack_init) refers to softdevice_handler.o(i.softdevice_handler_init) for softdevice_handler_init
    main.o(i.ble_stack_init) refers to app_error.o(i.app_error_handler) for app_error_handler
    main.o(i.ble_stack_init) refers to softdevice_handler.o(i.softdevice_ble_evt_handler_set) for softdevice_ble_evt_handler_set
    main.o(i.ble_stack_init) refers to softdevice_handler.o(i.softdevice_sys_evt_handler_set) for softdevice_sys_evt_handler_set
    main.o(i.ble_stack_init) refers to main.o(.bss) for .bss
    main.o(i.ble_stack_init) refers to main.o(i.ble_evt_dispatch) for ble_evt_dispatch
    main.o(i.ble_stack_init) refers to main.o(i.sys_evt_dispatch) for sys_evt_dispatch
    main.o(i.device_manager_event_handler) refers to client_handling.o(i.client_handling_create) for client_handling_create
    main.o(i.device_manager_event_handler) refers to app_error.o(i.app_error_handler) for app_error_handler
    main.o(i.device_manager_event_handler) refers to main.o(i.scan_start) for scan_start
    main.o(i.device_manager_event_handler) refers to client_handling.o(i.client_handling_destroy) for client_handling_destroy
    main.o(i.device_manager_event_handler) refers to memcpya.o(.text) for __aeabi_memcpy
    main.o(i.device_manager_event_handler) refers to device_manager_central.o(i.dm_security_setup_req) for dm_security_setup_req
    main.o(i.device_manager_event_handler) refers to client_handling.o(i.client_handling_dm_event_handler) for client_handling_dm_event_handler
    main.o(i.device_manager_event_handler) refers to main.o(.data) for .data
    main.o(i.device_manager_init) refers to pstorage.o(i.pstorage_init) for pstorage_init
    main.o(i.device_manager_init) refers to app_error.o(i.app_error_handler) for app_error_handler
    main.o(i.device_manager_init) refers to device_manager_central.o(i.dm_init) for dm_init
    main.o(i.device_manager_init) refers to memseta.o(.text) for __aeabi_memclr
    main.o(i.device_manager_init) refers to device_manager_central.o(i.dm_register) for dm_register
    main.o(i.device_manager_init) refers to main.o(i.device_manager_event_handler) for device_manager_event_handler
    main.o(i.device_manager_init) refers to main.o(.data) for .data
    main.o(i.main) refers to simple_uart.o(i.simple_uart_config) for simple_uart_config
    main.o(i.main) refers to debug_util.o(i.debug_printf) for debug_printf
    main.o(i.main) refers to main.o(i.ble_stack_init) for ble_stack_init
    main.o(i.main) refers to client_handling.o(i.client_handling_init) for client_handling_init
    main.o(i.main) refers to main.o(i.device_manager_init) for device_manager_init
    main.o(i.main) refers to memcpya.o(.text) for __aeabi_memcpy4
    main.o(i.main) refers to app_pwm.o(i.app_pwm_init) for app_pwm_init
    main.o(i.main) refers to app_error.o(i.app_error_handler) for app_error_handler
    main.o(i.main) refers to app_pwm.o(i.app_pwm_enable) for app_pwm_enable
    main.o(i.main) refers to main.o(i.scan_start) for scan_start
    main.o(i.main) refers to nrf_delay.o(i.nrf_delay_ms) for nrf_delay_ms
    main.o(i.main) refers to client_handling.o(i.read_acc_other_device) for read_acc_other_device
    main.o(i.main) refers to printfa.o(i.__0sprintf) for __2sprintf
    main.o(i.main) refers to main.o(i.make_alarm) for make_alarm
    main.o(i.main) refers to main.o(.constdata) for .constdata
    main.o(i.main) refers to main.o(i.pwm_ready_callback) for pwm_ready_callback
    main.o(i.main) refers to main.o(.data) for .data
    main.o(i.make_alarm) refers to main.o(i.pwm_set_value) for pwm_set_value
    main.o(i.make_alarm) refers to nrf_delay.o(i.nrf_delay_ms) for nrf_delay_ms
    main.o(i.make_alarm) refers to main.o(.data) for .data
    main.o(i.on_ble_evt) refers to main.o(i.adv_report_parse) for adv_report_parse
    main.o(i.on_ble_evt) refers to memcmp.o(.text) for memcmp
    main.o(i.on_ble_evt) refers to main.o(.data) for .data
    main.o(i.on_ble_evt) refers to main.o(.constdata) for .constdata
    main.o(i.pwm_ready_callback) refers to main.o(.data) for .data
    main.o(i.pwm_set_value) refers to app_pwm.o(i.app_pwm_channel_duty_set) for app_pwm_channel_duty_set
    main.o(i.pwm_set_value) refers to app_error.o(i.app_error_handler) for app_error_handler
    main.o(i.pwm_set_value) refers to nrf_delay.o(i.nrf_delay_ms) for nrf_delay_ms
    main.o(i.pwm_set_value) refers to main.o(.data) for .data
    main.o(i.pwm_set_value) refers to main.o(.constdata) for .constdata
    main.o(i.scan_start) refers to pstorage.o(i.pstorage_access_status_get) for pstorage_access_status_get
    main.o(i.scan_start) refers to app_error.o(i.app_error_handler) for app_error_handler
    main.o(i.scan_start) refers to main.o(.data) for .data
    main.o(i.scan_start) refers to main.o(.constdata) for .constdata
    main.o(i.sys_evt_dispatch) refers to pstorage.o(i.pstorage_sys_event_handler) for pstorage_sys_event_handler
    main.o(i.sys_evt_dispatch) refers to main.o(i.scan_start) for scan_start
    main.o(i.sys_evt_dispatch) refers to main.o(.data) for .data
    main.o(.constdata) refers to main.o(.bss) for m_pwm_PWM1_cb
    main.o(.constdata) refers to main.o(.constdata) for m_pwm_PWM1_timer
    acc_lis2.o(i.acc_get_fifo_src) refers to acc_lis2.o(i.spia_rd8) for spia_rd8
    acc_lis2.o(i.acc_get_fifo_wtm) refers to acc_lis2.o(i.spia_rd8) for spia_rd8
    acc_lis2.o(i.acc_get_int1_cfg) refers to acc_lis2.o(i.spia_rd8) for spia_rd8
    acc_lis2.o(i.acc_get_int1_src) refers to acc_lis2.o(i.spia_rd8) for spia_rd8
    acc_lis2.o(i.acc_get_status) refers to acc_lis2.o(i.spia_rd8) for spia_rd8
    acc_lis2.o(i.acc_get_who_am_i) refers to acc_lis2.o(i.spia_rd8) for spia_rd8
    acc_lis2.o(i.acc_get_x) refers to acc_lis2.o(i.spia_rd16) for spia_rd16
    acc_lis2.o(i.acc_get_x8) refers to acc_lis2.o(i.spia_rd8) for spia_rd8
    acc_lis2.o(i.acc_get_xy) refers to acc_lis2.o(i.spia_rd8) for spia_rd8
    acc_lis2.o(i.acc_get_xyz) refers to idiv.o(.text) for __aeabi_idivmod
    acc_lis2.o(i.acc_get_xyz) refers to acc_lis2.o(.data) for .data
    acc_lis2.o(i.acc_get_xyz) refers to acc_lis2.o(.bss) for .bss
    acc_lis2.o(i.acc_get_xyz8) refers to acc_lis2.o(i.spia_rd16) for spia_rd16
    acc_lis2.o(i.acc_get_xyzreg) refers to acc_lis2.o(i.spia_rd8) for spia_rd8
    acc_lis2.o(i.acc_get_y8) refers to acc_lis2.o(i.spia_rd8) for spia_rd8
    acc_lis2.o(i.acc_get_z8) refers to acc_lis2.o(i.spia_rd8) for spia_rd8
    acc_lis2.o(i.acc_init) refers to acc_lis2.o(i.spia_init) for spia_init
    acc_lis2.o(i.acc_init) refers to nrf_delay.o(i.nrf_delay_ms) for nrf_delay_ms
    acc_lis2.o(i.acc_init) refers to acc_lis2.o(i.acc_set_400Hz_lp_mode) for acc_set_400Hz_lp_mode
    acc_lis2.o(i.acc_init) refers to acc_lis2.o(i.acc_get_status) for acc_get_status
    acc_lis2.o(i.acc_init) refers to acc_lis2.o(i.spia_wr8) for spia_wr8
    acc_lis2.o(i.acc_init) refers to acc_lis2.o(.data) for .data
    acc_lis2.o(i.acc_init_w_int) refers to acc_lis2.o(i.acc_init) for acc_init
    acc_lis2.o(i.acc_init_w_int) refers to acc_lis2.o(i.spia_wr8) for spia_wr8
    acc_lis2.o(i.acc_reset_fifo) refers to acc_lis2.o(i.spia_wr8) for spia_wr8
    acc_lis2.o(i.acc_set_100Hz_lp_mode) refers to acc_lis2.o(i.acc_set_100Hz_lp_mode_xy) for acc_set_100Hz_lp_mode_xy
    acc_lis2.o(i.acc_set_100Hz_lp_mode_xy) refers to acc_lis2.o(i.spia_wr8) for spia_wr8
    acc_lis2.o(i.acc_set_100Hz_lp_mode_xz) refers to acc_lis2.o(i.spia_wr8) for spia_wr8
    acc_lis2.o(i.acc_set_100Hz_lp_mode_yz) refers to acc_lis2.o(i.spia_wr8) for spia_wr8
    acc_lis2.o(i.acc_set_400Hz_lp_mode) refers to acc_lis2.o(i.spia_wr8) for spia_wr8
    acc_lis2.o(i.acc_set_400Hz_lp_mode_xy) refers to acc_lis2.o(i.spia_wr8) for spia_wr8
    acc_lis2.o(i.acc_set_400Hz_lp_mode_xz) refers to acc_lis2.o(i.spia_wr8) for spia_wr8
    acc_lis2.o(i.acc_set_400Hz_lp_mode_yz) refers to acc_lis2.o(i.spia_wr8) for spia_wr8
    acc_lis2.o(i.acc_start_xyz) refers to acc_lis2.o(i.acc_get_fifo_src) for acc_get_fifo_src
    acc_lis2.o(i.acc_start_xyz) refers to acc_lis2.o(i.send_recv_spi0_data) for send_recv_spi0_data
    acc_lis2.o(i.acc_start_xyz) refers to acc_lis2.o(.data) for .data
    acc_lis2.o(i.send_recv_spi0_data) refers to spi_master.o(i.spi_master_send_recv) for spi_master_send_recv
    acc_lis2.o(i.send_recv_spi0_data) refers to acc_lis2.o(.data) for .data
    acc_lis2.o(i.send_recv_spi0_data) refers to acc_lis2.o(.bss) for .bss
    acc_lis2.o(i.spi_master_event_handler) refers to acc_lis2.o(.data) for .data
    acc_lis2.o(i.spia_init) refers to memcpya.o(.text) for __aeabi_memcpy4
    acc_lis2.o(i.spia_init) refers to spi_master.o(i.spi_master_open) for spi_master_open
    acc_lis2.o(i.spia_init) refers to spi_master.o(i.spi_master_evt_handler_reg) for spi_master_evt_handler_reg
    acc_lis2.o(i.spia_init) refers to acc_lis2.o(.constdata) for .constdata
    acc_lis2.o(i.spia_init) refers to acc_lis2.o(i.spi_master_event_handler) for spi_master_event_handler
    acc_lis2.o(i.spia_rd16) refers to acc_lis2.o(i.send_recv_spi0_data) for send_recv_spi0_data
    acc_lis2.o(i.spia_rd16) refers to acc_lis2.o(.bss) for .bss
    acc_lis2.o(i.spia_rd16) refers to acc_lis2.o(.data) for .data
    acc_lis2.o(i.spia_rd8) refers to acc_lis2.o(i.send_recv_spi0_data) for send_recv_spi0_data
    acc_lis2.o(i.spia_rd8) refers to acc_lis2.o(.bss) for .bss
    acc_lis2.o(i.spia_rd8) refers to acc_lis2.o(.data) for .data
    acc_lis2.o(i.spia_wr8) refers to acc_lis2.o(i.send_recv_spi0_data) for send_recv_spi0_data
    acc_lis2.o(i.spia_wr8) refers to acc_lis2.o(.data) for .data
    simple_uart.o(i.simple_uart_get_with_timeout) refers to simple_uart.o(.emb_text) for __asm___13_simple_uart_c_5dda6715__nrf_delay_us
    simple_uart.o(i.simple_uart_putstring) refers to simple_uart.o(i.simple_uart_put) for simple_uart_put
    debug_util.o(i.debug_printf) refers to printfa.o(i.__0vsprintf) for vsprintf
    debug_util.o(i.debug_printf) refers to simple_uart.o(i.simple_uart_putstring) for simple_uart_putstring
    spi_master.o(i.SPI0_TWI0_IRQHandler) refers to spi_master.o(i.spi_master_get_instance) for spi_master_get_instance
    spi_master.o(i.SPI0_TWI0_IRQHandler) refers to spi_master.o(i.spi_master_send_recv_irq) for spi_master_send_recv_irq
    spi_master.o(i.spi_master_buffer_init) refers to app_error.o(i.app_error_handler) for app_error_handler
    spi_master.o(i.spi_master_buffer_release) refers to app_error.o(i.app_error_handler) for app_error_handler
    spi_master.o(i.spi_master_close) refers to spi_master.o(i.spi_master_get_instance) for spi_master_get_instance
    spi_master.o(i.spi_master_close) refers to app_error.o(i.app_error_handler) for app_error_handler
    spi_master.o(i.spi_master_close) refers to spi_master.o(i.nrf_gpio_pin_set) for nrf_gpio_pin_set
    spi_master.o(i.spi_master_close) refers to spi_master.o(i.spi_master_init_hw_instance) for spi_master_init_hw_instance
    spi_master.o(i.spi_master_get_instance) refers to spi_master.o(.bss) for .bss
    spi_master.o(i.spi_master_init_hw_instance) refers to app_error.o(i.app_error_handler) for app_error_handler
    spi_master.o(i.spi_master_open) refers to spi_master.o(i.spi_master_get_instance) for spi_master_get_instance
    spi_master.o(i.spi_master_open) refers to app_error.o(i.app_error_handler) for app_error_handler
    spi_master.o(i.spi_master_open) refers to spi_master.o(i.spi_master_init_hw_instance) for spi_master_init_hw_instance
    spi_master.o(i.spi_master_open) refers to spi_master.o(i.nrf_gpio_pin_set) for nrf_gpio_pin_set
    spi_master.o(i.spi_master_send_recv) refers to spi_master.o(i.spi_master_get_instance) for spi_master_get_instance
    spi_master.o(i.spi_master_send_recv) refers to app_error.o(i.app_error_handler) for app_error_handler
    spi_master.o(i.spi_master_send_recv) refers to spi_master.o(i.spi_master_buffer_init) for spi_master_buffer_init
    spi_master.o(i.spi_master_send_recv_irq) refers to app_error.o(i.app_error_handler) for app_error_handler
    spi_master.o(i.spi_master_send_recv_irq) refers to spi_master.o(i.spi_master_signal_evt) for spi_master_signal_evt
    spi_master.o(i.spi_master_send_recv_irq) refers to spi_master.o(i.nrf_gpio_pin_set) for nrf_gpio_pin_set
    spi_master.o(i.spi_master_send_recv_irq) refers to spi_master.o(i.spi_master_buffer_release) for spi_master_buffer_release
    spi_master.o(i.spi_master_signal_evt) refers to app_error.o(i.app_error_handler) for app_error_handler
    spi_master.o(i.spi_master_signal_evt) refers to spi_master.o(.constdata) for .constdata
    firfilter.o(i.fir_bp_filter) refers to firfilter.o(i.fir_split) for fir_split
    firfilter.o(i.fir_bp_filter) refers to firfilter.o(.data) for .data
    firfilter.o(i.fir_bp_filter) refers to firfilter.o(.bss) for .bss
    firfilter.o(i.fir_bp_filter) refers to firfilter.o(.constdata) for .constdata
    firfilter.o(i.fir_delay) refers to firfilter.o(.data) for .data
    firfilter.o(i.fir_delay) refers to firfilter.o(.bss) for .bss
    firfilter.o(i.fir_delay_1) refers to firfilter.o(.data) for .data
    firfilter.o(i.fir_delay_1) refers to firfilter.o(.bss) for .bss
    firfilter.o(i.fir_delay_2) refers to firfilter.o(.data) for .data
    firfilter.o(i.fir_delay_2) refers to firfilter.o(.bss) for .bss
    firfilter.o(i.fir_filter_tq) refers to firfilter.o(i.fir_split32) for fir_split32
    firfilter.o(i.fir_filter_tq) refers to firfilter.o(.data) for .data
    firfilter.o(i.fir_filter_tq) refers to firfilter.o(.bss) for .bss
    firfilter.o(i.fir_filter_tq) refers to firfilter.o(.constdata) for .constdata
    firfilter.o(i.fir_lp_filter) refers to firfilter.o(i.fir_split) for fir_split
    firfilter.o(i.fir_lp_filter) refers to firfilter.o(.data) for .data
    firfilter.o(i.fir_lp_filter) refers to firfilter.o(.bss) for .bss
    firfilter.o(i.fir_lp_filter) refers to firfilter.o(.constdata) for .constdata
    arm_startup_nrf51.o(RESET) refers to arm_startup_nrf51.o(STACK) for __initial_sp
    arm_startup_nrf51.o(RESET) refers to arm_startup_nrf51.o(.text) for Reset_Handler
    arm_startup_nrf51.o(RESET) refers to app_uart_fifo.o(i.UART0_IRQHandler) for UART0_IRQHandler
    arm_startup_nrf51.o(RESET) refers to spi_master.o(i.SPI0_TWI0_IRQHandler) for SPI0_TWI0_IRQHandler
    arm_startup_nrf51.o(RESET) refers to nrf_drv_gpiote.o(i.GPIOTE_IRQHandler) for GPIOTE_IRQHandler
    arm_startup_nrf51.o(RESET) refers to nrf_drv_timer.o(i.TIMER1_IRQHandler) for TIMER1_IRQHandler
    arm_startup_nrf51.o(RESET) refers to softdevice_handler.o(i.SWI2_IRQHandler) for SWI2_IRQHandler
    arm_startup_nrf51.o(.text) refers to system_nrf51.o(i.SystemInit) for SystemInit
    arm_startup_nrf51.o(.text) refers to entry.o(.ARM.Collect$$$$00000000) for __main
    system_nrf51.o(i.SystemCoreClockUpdate) refers to system_nrf51.o(.data) for .data
    system_nrf51.o(i.SystemInit) refers to system_nrf51.o(i.is_manual_peripheral_setup_needed) for is_manual_peripheral_setup_needed
    ble_advdata.o(i.adv_data_encode) refers to ble_advdata.o(i.name_encode) for name_encode
    ble_advdata.o(i.adv_data_encode) refers to ble_advdata.o(i.uint16_encode) for uint16_encode
    ble_advdata.o(i.adv_data_encode) refers to ble_advdata.o(i.uuid_list_encode) for uuid_list_encode
    ble_advdata.o(i.adv_data_encode) refers to ble_advdata.o(i.conn_int_encode) for conn_int_encode
    ble_advdata.o(i.adv_data_encode) refers to ble_advdata.o(i.manuf_specific_data_encode) for manuf_specific_data_encode
    ble_advdata.o(i.adv_data_encode) refers to ble_advdata.o(i.service_data_encode) for service_data_encode
    ble_advdata.o(i.ble_advdata_set) refers to ble_advdata.o(i.adv_data_encode) for adv_data_encode
    ble_advdata.o(i.conn_int_encode) refers to ble_advdata.o(i.uint16_encode) for uint16_encode
    ble_advdata.o(i.manuf_specific_data_encode) refers to ble_advdata.o(i.uint16_encode) for uint16_encode
    ble_advdata.o(i.manuf_specific_data_encode) refers to memcpya.o(.text) for __aeabi_memcpy
    ble_advdata.o(i.service_data_encode) refers to ble_advdata.o(i.uint16_encode) for uint16_encode
    ble_advdata.o(i.service_data_encode) refers to memcpya.o(.text) for __aeabi_memcpy
    ble_advdata.o(i.uuid_list_encode) refers to ble_advdata.o(i.uuid_list_sized_encode) for uuid_list_sized_encode
    ble_db_discovery.o(i.ble_db_discovery_close) refers to ble_db_discovery.o(.data) for .data
    ble_db_discovery.o(i.ble_db_discovery_evt_register) refers to ble_db_discovery.o(.data) for .data
    ble_db_discovery.o(i.ble_db_discovery_evt_register) refers to ble_db_discovery.o(.bss) for .bss
    ble_db_discovery.o(i.ble_db_discovery_init) refers to ble_db_discovery.o(.data) for .data
    ble_db_discovery.o(i.ble_db_discovery_on_ble_evt) refers to memseta.o(.text) for __aeabi_memclr
    ble_db_discovery.o(i.ble_db_discovery_on_ble_evt) refers to ble_db_discovery.o(i.on_descriptor_discovery_rsp) for on_descriptor_discovery_rsp
    ble_db_discovery.o(i.ble_db_discovery_on_ble_evt) refers to ble_db_discovery.o(i.discovery_complete_evt_trigger) for discovery_complete_evt_trigger
    ble_db_discovery.o(i.ble_db_discovery_on_ble_evt) refers to ble_db_discovery.o(i.on_srv_disc_completion) for on_srv_disc_completion
    ble_db_discovery.o(i.ble_db_discovery_on_ble_evt) refers to ble_db_discovery.o(i.characteristics_discover) for characteristics_discover
    ble_db_discovery.o(i.ble_db_discovery_on_ble_evt) refers to ble_db_discovery.o(i.discovery_error_evt_trigger) for discovery_error_evt_trigger
    ble_db_discovery.o(i.ble_db_discovery_on_ble_evt) refers to ble_db_discovery.o(i.on_characteristic_discovery_rsp) for on_characteristic_discovery_rsp
    ble_db_discovery.o(i.ble_db_discovery_on_ble_evt) refers to ble_db_discovery.o(.data) for .data
    ble_db_discovery.o(i.ble_db_discovery_start) refers to ble_db_discovery.o(.data) for .data
    ble_db_discovery.o(i.ble_db_discovery_start) refers to ble_db_discovery.o(.bss) for .bss
    ble_db_discovery.o(i.descriptors_discover) refers to ble_db_discovery.o(i.is_desc_discovery_reqd) for is_desc_discovery_reqd
    ble_db_discovery.o(i.discovery_complete_evt_trigger) refers to ble_db_discovery.o(i.registered_handler_get) for registered_handler_get
    ble_db_discovery.o(i.discovery_complete_evt_trigger) refers to memcpya.o(.text) for __aeabi_memcpy
    ble_db_discovery.o(i.discovery_complete_evt_trigger) refers to ble_db_discovery.o(i.pending_user_evts_send) for pending_user_evts_send
    ble_db_discovery.o(i.discovery_complete_evt_trigger) refers to ble_db_discovery.o(.data) for .data
    ble_db_discovery.o(i.discovery_complete_evt_trigger) refers to ble_db_discovery.o(.bss) for .bss
    ble_db_discovery.o(i.discovery_error_evt_trigger) refers to ble_db_discovery.o(i.registered_handler_get) for registered_handler_get
    ble_db_discovery.o(i.discovery_error_evt_trigger) refers to ble_db_discovery.o(i.pending_user_evts_send) for pending_user_evts_send
    ble_db_discovery.o(i.discovery_error_evt_trigger) refers to ble_db_discovery.o(.data) for .data
    ble_db_discovery.o(i.discovery_error_evt_trigger) refers to ble_db_discovery.o(.bss) for .bss
    ble_db_discovery.o(i.on_characteristic_discovery_rsp) refers to memcpya.o(.text) for __aeabi_memcpy
    ble_db_discovery.o(i.on_characteristic_discovery_rsp) refers to ble_db_discovery.o(i.characteristics_discover) for characteristics_discover
    ble_db_discovery.o(i.on_characteristic_discovery_rsp) refers to ble_db_discovery.o(i.descriptors_discover) for descriptors_discover
    ble_db_discovery.o(i.on_characteristic_discovery_rsp) refers to ble_db_discovery.o(i.discovery_error_evt_trigger) for discovery_error_evt_trigger
    ble_db_discovery.o(i.on_characteristic_discovery_rsp) refers to ble_db_discovery.o(i.discovery_complete_evt_trigger) for discovery_complete_evt_trigger
    ble_db_discovery.o(i.on_characteristic_discovery_rsp) refers to ble_db_discovery.o(i.on_srv_disc_completion) for on_srv_disc_completion
    ble_db_discovery.o(i.on_descriptor_discovery_rsp) refers to ble_db_discovery.o(i.descriptors_discover) for descriptors_discover
    ble_db_discovery.o(i.on_descriptor_discovery_rsp) refers to ble_db_discovery.o(i.discovery_error_evt_trigger) for discovery_error_evt_trigger
    ble_db_discovery.o(i.on_descriptor_discovery_rsp) refers to ble_db_discovery.o(i.discovery_complete_evt_trigger) for discovery_complete_evt_trigger
    ble_db_discovery.o(i.on_descriptor_discovery_rsp) refers to ble_db_discovery.o(i.on_srv_disc_completion) for on_srv_disc_completion
    ble_db_discovery.o(i.on_srv_disc_completion) refers to ble_db_discovery.o(i.discovery_error_evt_trigger) for discovery_error_evt_trigger
    ble_db_discovery.o(i.on_srv_disc_completion) refers to ble_db_discovery.o(.data) for .data
    ble_db_discovery.o(i.on_srv_disc_completion) refers to ble_db_discovery.o(.bss) for .bss
    ble_db_discovery.o(i.pending_user_evts_send) refers to ble_db_discovery.o(.data) for .data
    ble_db_discovery.o(i.pending_user_evts_send) refers to ble_db_discovery.o(.bss) for .bss
    ble_db_discovery.o(i.registered_handler_get) refers to ble_db_discovery.o(.bss) for .bss
    ble_db_discovery.o(i.registered_handler_get) refers to ble_db_discovery.o(.data) for .data
    ble_srv_common.o(i.ble_srv_ascii_to_utf8) refers to strlen.o(.text) for strlen
    ble_srv_common.o(i.characteristic_add) refers to ble_srv_common.o(i.set_security_req) for set_security_req
    ble_srv_common.o(i.characteristic_add) refers to memseta.o(.text) for __aeabi_memclr4
    ble_srv_common.o(i.set_security_req) refers to client_handling.o(i.__ARM_common_switch8) for __ARM_common_switch8
    device_manager_central.o(i.app_evt_notify) refers to device_manager_central.o(.bss) for .bss
    device_manager_central.o(i.connection_instance_find) refers to device_manager_central.o(.bss) for .bss
    device_manager_central.o(i.connection_instance_init) refers to memseta.o(.text) for __aeabi_memclr
    device_manager_central.o(i.connection_instance_init) refers to device_manager_central.o(.bss) for .bss
    device_manager_central.o(i.device_context_store) refers to pstorage.o(i.pstorage_block_identifier_get) for pstorage_block_identifier_get
    device_manager_central.o(i.device_context_store) refers to device_manager_central.o(.data) for .data
    device_manager_central.o(i.device_context_store) refers to device_manager_central.o(.bss) for .bss
    device_manager_central.o(i.device_context_store) refers to device_manager_central.o(i.storage_operation_dummy_handler) for storage_operation_dummy_handler
    device_manager_central.o(i.device_context_store) refers to device_manager_central.o(.constdata) for .constdata
    device_manager_central.o(i.device_context_store) refers to pstorage.o(i.pstorage_update) for pstorage_update
    device_manager_central.o(i.device_context_store) refers to pstorage.o(i.pstorage_store) for pstorage_store
    device_manager_central.o(i.device_instance_allocate) refers to memcpya.o(.text) for __aeabi_memcpy
    device_manager_central.o(i.device_instance_allocate) refers to device_manager_central.o(.bss) for .bss
    device_manager_central.o(i.device_instance_free) refers to pstorage.o(i.pstorage_block_identifier_get) for pstorage_block_identifier_get
    device_manager_central.o(i.device_instance_free) refers to pstorage.o(i.pstorage_clear) for pstorage_clear
    device_manager_central.o(i.device_instance_free) refers to device_manager_central.o(i.peer_instance_init) for peer_instance_init
    device_manager_central.o(i.device_instance_free) refers to device_manager_central.o(.data) for .data
    device_manager_central.o(i.dm_application_instance_set) refers to device_manager_central.o(.data) for .data
    device_manager_central.o(i.dm_application_instance_set) refers to device_manager_central.o(.bss) for .bss
    device_manager_central.o(i.dm_ble_evt_handler) refers to device_manager_central.o(i.dm_handle_initialize) for dm_handle_initialize
    device_manager_central.o(i.dm_ble_evt_handler) refers to app_error.o(i.app_error_handler) for app_error_handler
    device_manager_central.o(i.dm_ble_evt_handler) refers to device_manager_central.o(i.connection_instance_find) for connection_instance_find
    device_manager_central.o(i.dm_ble_evt_handler) refers to memcpya.o(.text) for __aeabi_memcpy
    device_manager_central.o(i.dm_ble_evt_handler) refers to memcmp.o(.text) for memcmp
    device_manager_central.o(i.dm_ble_evt_handler) refers to pstorage.o(i.pstorage_block_identifier_get) for pstorage_block_identifier_get
    device_manager_central.o(i.dm_ble_evt_handler) refers to pstorage.o(i.pstorage_load) for pstorage_load
    device_manager_central.o(i.dm_ble_evt_handler) refers to device_manager_central.o(i.device_context_store) for device_context_store
    device_manager_central.o(i.dm_ble_evt_handler) refers to device_manager_central.o(i.peer_instance_init) for peer_instance_init
    device_manager_central.o(i.dm_ble_evt_handler) refers to memseta.o(.text) for __aeabi_memclr4
    device_manager_central.o(i.dm_ble_evt_handler) refers to device_manager_central.o(i.app_evt_notify) for app_evt_notify
    device_manager_central.o(i.dm_ble_evt_handler) refers to device_manager_central.o(i.connection_instance_init) for connection_instance_init
    device_manager_central.o(i.dm_ble_evt_handler) refers to device_manager_central.o(i.initiate_security_request) for initiate_security_request
    device_manager_central.o(i.dm_ble_evt_handler) refers to device_manager_central.o(.data) for .data
    device_manager_central.o(i.dm_ble_evt_handler) refers to device_manager_central.o(.bss) for .bss
    device_manager_central.o(i.dm_ble_evt_handler) refers to device_manager_central.o(.constdata) for .constdata
    device_manager_central.o(i.dm_device_delete) refers to device_manager_central.o(i.device_instance_free) for device_instance_free
    device_manager_central.o(i.dm_device_delete) refers to device_manager_central.o(.data) for .data
    device_manager_central.o(i.dm_device_delete) refers to device_manager_central.o(.bss) for .bss
    device_manager_central.o(i.dm_device_delete_all) refers to device_manager_central.o(i.device_instance_free) for device_instance_free
    device_manager_central.o(i.dm_device_delete_all) refers to device_manager_central.o(.data) for .data
    device_manager_central.o(i.dm_device_delete_all) refers to device_manager_central.o(.bss) for .bss
    device_manager_central.o(i.dm_distributed_keys_get) refers to pstorage.o(i.pstorage_block_identifier_get) for pstorage_block_identifier_get
    device_manager_central.o(i.dm_distributed_keys_get) refers to pstorage.o(i.pstorage_load) for pstorage_load
    device_manager_central.o(i.dm_distributed_keys_get) refers to device_manager_central.o(.data) for .data
    device_manager_central.o(i.dm_distributed_keys_get) refers to device_manager_central.o(.bss) for .bss
    device_manager_central.o(i.dm_init) refers to device_manager_central.o(i.connection_instance_init) for connection_instance_init
    device_manager_central.o(i.dm_init) refers to memseta.o(.text) for __aeabi_memclr4
    device_manager_central.o(i.dm_init) refers to device_manager_central.o(i.peer_instance_init) for peer_instance_init
    device_manager_central.o(i.dm_init) refers to pstorage.o(i.pstorage_register) for pstorage_register
    device_manager_central.o(i.dm_init) refers to pstorage.o(i.pstorage_clear) for pstorage_clear
    device_manager_central.o(i.dm_init) refers to pstorage.o(i.pstorage_block_identifier_get) for pstorage_block_identifier_get
    device_manager_central.o(i.dm_init) refers to pstorage.o(i.pstorage_load) for pstorage_load
    device_manager_central.o(i.dm_init) refers to device_manager_central.o(.bss) for .bss
    device_manager_central.o(i.dm_init) refers to device_manager_central.o(i.dm_pstorage_cb_handler) for dm_pstorage_cb_handler
    device_manager_central.o(i.dm_init) refers to device_manager_central.o(.data) for .data
    device_manager_central.o(i.dm_peer_addr_get) refers to memcpya.o(.text) for __aeabi_memcpy
    device_manager_central.o(i.dm_peer_addr_get) refers to device_manager_central.o(.data) for .data
    device_manager_central.o(i.dm_peer_addr_get) refers to device_manager_central.o(.bss) for .bss
    device_manager_central.o(i.dm_peer_addr_set) refers to memcpya.o(.text) for __aeabi_memcpy
    device_manager_central.o(i.dm_peer_addr_set) refers to device_manager_central.o(i.device_context_store) for device_context_store
    device_manager_central.o(i.dm_peer_addr_set) refers to device_manager_central.o(.data) for .data
    device_manager_central.o(i.dm_peer_addr_set) refers to device_manager_central.o(.bss) for .bss
    device_manager_central.o(i.dm_pstorage_cb_handler) refers to device_manager_central.o(i.dm_handle_initialize) for dm_handle_initialize
    device_manager_central.o(i.dm_pstorage_cb_handler) refers to app_error.o(i.app_error_handler) for app_error_handler
    device_manager_central.o(i.dm_pstorage_cb_handler) refers to pstorage.o(i.pstorage_block_identifier_get) for pstorage_block_identifier_get
    device_manager_central.o(i.dm_pstorage_cb_handler) refers to memcmp.o(.text) for memcmp
    device_manager_central.o(i.dm_pstorage_cb_handler) refers to uidiv.o(.text) for __aeabi_uidivmod
    device_manager_central.o(i.dm_pstorage_cb_handler) refers to device_manager_central.o(i.app_evt_notify) for app_evt_notify
    device_manager_central.o(i.dm_pstorage_cb_handler) refers to device_manager_central.o(i.update_status_bit_reset) for update_status_bit_reset
    device_manager_central.o(i.dm_pstorage_cb_handler) refers to device_manager_central.o(.bss) for .bss
    device_manager_central.o(i.dm_pstorage_cb_handler) refers to device_manager_central.o(.data) for .data
    device_manager_central.o(i.dm_register) refers to memcpya.o(.text) for __aeabi_memcpy
    device_manager_central.o(i.dm_register) refers to device_manager_central.o(.data) for .data
    device_manager_central.o(i.dm_register) refers to device_manager_central.o(.bss) for .bss
    device_manager_central.o(i.dm_security_setup_req) refers to device_manager_central.o(i.device_instance_allocate) for device_instance_allocate
    device_manager_central.o(i.dm_security_setup_req) refers to device_manager_central.o(i.initiate_security_request) for initiate_security_request
    device_manager_central.o(i.dm_security_setup_req) refers to device_manager_central.o(.data) for .data
    device_manager_central.o(i.dm_security_setup_req) refers to device_manager_central.o(.bss) for .bss
    device_manager_central.o(i.dm_security_status_req) refers to device_manager_central.o(.data) for .data
    device_manager_central.o(i.dm_security_status_req) refers to device_manager_central.o(.bss) for .bss
    device_manager_central.o(i.dm_service_context_delete) refers to device_manager_central.o(.data) for .data
    device_manager_central.o(i.dm_service_context_delete) refers to device_manager_central.o(.bss) for .bss
    device_manager_central.o(i.dm_service_context_get) refers to pstorage.o(i.pstorage_block_identifier_get) for pstorage_block_identifier_get
    device_manager_central.o(i.dm_service_context_get) refers to device_manager_central.o(.data) for .data
    device_manager_central.o(i.dm_service_context_get) refers to device_manager_central.o(.bss) for .bss
    device_manager_central.o(i.dm_service_context_get) refers to device_manager_central.o(.constdata) for .constdata
    device_manager_central.o(i.dm_service_context_set) refers to memcpya.o(.text) for __aeabi_memcpy
    device_manager_central.o(i.dm_service_context_set) refers to pstorage.o(i.pstorage_block_identifier_get) for pstorage_block_identifier_get
    device_manager_central.o(i.dm_service_context_set) refers to device_manager_central.o(.data) for .data
    device_manager_central.o(i.dm_service_context_set) refers to device_manager_central.o(.bss) for .bss
    device_manager_central.o(i.dm_service_context_set) refers to device_manager_central.o(.constdata) for .constdata
    device_manager_central.o(i.dm_whitelist_create) refers to device_manager_central.o(.data) for .data
    device_manager_central.o(i.dm_whitelist_create) refers to device_manager_central.o(.bss) for .bss
    device_manager_central.o(i.gatts_context_apply) refers to device_manager_central.o(.bss) for .bss
    device_manager_central.o(i.gatts_context_load) refers to pstorage.o(i.pstorage_load) for pstorage_load
    device_manager_central.o(i.gatts_context_load) refers to device_manager_central.o(.bss) for .bss
    device_manager_central.o(i.gatts_context_store) refers to memcmp.o(.text) for memcmp
    device_manager_central.o(i.gatts_context_store) refers to memcpya.o(.text) for __aeabi_memcpy4
    device_manager_central.o(i.gatts_context_store) refers to device_manager_central.o(.bss) for .bss
    device_manager_central.o(i.gatts_context_store) refers to pstorage.o(i.pstorage_update) for pstorage_update
    device_manager_central.o(i.gatts_context_store) refers to pstorage.o(i.pstorage_store) for pstorage_store
    device_manager_central.o(i.gattsc_context_apply) refers to device_manager_central.o(i.gatts_context_apply) for gatts_context_apply
    device_manager_central.o(i.gattsc_context_load) refers to device_manager_central.o(i.gatts_context_load) for gatts_context_load
    device_manager_central.o(i.gattsc_context_store) refers to device_manager_central.o(i.gatts_context_store) for gatts_context_store
    device_manager_central.o(i.initiate_security_request) refers to device_manager_central.o(.bss) for .bss
    device_manager_central.o(i.peer_instance_init) refers to memseta.o(.text) for __aeabi_memclr
    device_manager_central.o(i.peer_instance_init) refers to device_manager_central.o(i.update_status_bit_reset) for update_status_bit_reset
    device_manager_central.o(i.peer_instance_init) refers to device_manager_central.o(.bss) for .bss
    device_manager_central.o(i.update_status_bit_reset) refers to device_manager_central.o(.data) for .data
    device_manager_central.o(.constdata) refers to device_manager_central.o(i.no_service_context_store) for no_service_context_store
    device_manager_central.o(.constdata) refers to device_manager_central.o(i.gatts_context_store) for gatts_context_store
    device_manager_central.o(.constdata) refers to device_manager_central.o(i.gattc_context_store) for gattc_context_store
    device_manager_central.o(.constdata) refers to device_manager_central.o(i.gattsc_context_store) for gattsc_context_store
    device_manager_central.o(.constdata) refers to device_manager_central.o(i.no_service_context_load) for no_service_context_load
    device_manager_central.o(.constdata) refers to device_manager_central.o(i.gatts_context_load) for gatts_context_load
    device_manager_central.o(.constdata) refers to device_manager_central.o(i.gattc_context_load) for gattc_context_load
    device_manager_central.o(.constdata) refers to device_manager_central.o(i.gattsc_context_load) for gattsc_context_load
    device_manager_central.o(.constdata) refers to device_manager_central.o(i.no_service_context_apply) for no_service_context_apply
    device_manager_central.o(.constdata) refers to device_manager_central.o(i.gatts_context_apply) for gatts_context_apply
    device_manager_central.o(.constdata) refers to device_manager_central.o(i.gattc_context_apply) for gattc_context_apply
    device_manager_central.o(.constdata) refers to device_manager_central.o(i.gattsc_context_apply) for gattsc_context_apply
    app_uart_fifo.o(i.UART0_IRQHandler) refers to app_fifo.o(i.app_fifo_put) for app_fifo_put
    app_uart_fifo.o(i.UART0_IRQHandler) refers to app_uart_fifo.o(i.on_uart_event) for on_uart_event
    app_uart_fifo.o(i.UART0_IRQHandler) refers to app_uart_fifo.o(.data) for .data
    app_uart_fifo.o(i.UART0_IRQHandler) refers to app_uart_fifo.o(.bss) for .bss
    app_uart_fifo.o(i.action_tx_send) refers to app_fifo.o(i.app_fifo_get) for app_fifo_get
    app_uart_fifo.o(i.action_tx_send) refers to app_uart_fifo.o(i.action_tx_stop) for action_tx_stop
    app_uart_fifo.o(i.action_tx_send) refers to app_uart_fifo.o(.data) for .data
    app_uart_fifo.o(i.action_tx_send) refers to app_uart_fifo.o(.bss) for .bss
    app_uart_fifo.o(i.action_tx_stop) refers to app_uart_fifo.o(.data) for .data
    app_uart_fifo.o(i.action_uart_deactivate) refers to app_uart_fifo.o(.data) for .data
    app_uart_fifo.o(i.app_uart_close) refers to app_uart_fifo.o(i.on_uart_event) for on_uart_event
    app_uart_fifo.o(i.app_uart_close) refers to nrf_drv_gpiote.o(i.nrf_drv_gpiote_in_uninit) for nrf_drv_gpiote_in_uninit
    app_uart_fifo.o(i.app_uart_flush) refers to app_fifo.o(i.app_fifo_flush) for app_fifo_flush
    app_uart_fifo.o(i.app_uart_flush) refers to app_uart_fifo.o(.bss) for .bss
    app_uart_fifo.o(i.app_uart_get) refers to app_fifo.o(i.app_fifo_get) for app_fifo_get
    app_uart_fifo.o(i.app_uart_get) refers to app_uart_fifo.o(.bss) for .bss
    app_uart_fifo.o(i.app_uart_get_connection_state) refers to app_uart_fifo.o(.data) for .data
    app_uart_fifo.o(i.app_uart_init) refers to app_fifo.o(i.app_fifo_init) for app_fifo_init
    app_uart_fifo.o(i.app_uart_init) refers to nrf_drv_gpiote.o(i.nrf_drv_gpiote_is_init) for nrf_drv_gpiote_is_init
    app_uart_fifo.o(i.app_uart_init) refers to nrf_drv_gpiote.o(i.nrf_drv_gpiote_init) for nrf_drv_gpiote_init
    app_uart_fifo.o(i.app_uart_init) refers to nrf_drv_gpiote.o(i.nrf_drv_gpiote_out_init) for nrf_drv_gpiote_out_init
    app_uart_fifo.o(i.app_uart_init) refers to nrf_drv_gpiote.o(i.nrf_drv_gpiote_in_init) for nrf_drv_gpiote_in_init
    app_uart_fifo.o(i.app_uart_init) refers to nrf_drv_gpiote.o(i.nrf_drv_gpiote_in_event_enable) for nrf_drv_gpiote_in_event_enable
    app_uart_fifo.o(i.app_uart_init) refers to nrf_drv_gpiote.o(i.nrf_drv_gpiote_in_is_set) for nrf_drv_gpiote_in_is_set
    app_uart_fifo.o(i.app_uart_init) refers to app_uart_fifo.o(i.on_uart_event) for on_uart_event
    app_uart_fifo.o(i.app_uart_init) refers to app_uart_fifo.o(.data) for .data
    app_uart_fifo.o(i.app_uart_init) refers to app_uart_fifo.o(.bss) for .bss
    app_uart_fifo.o(i.app_uart_init) refers to app_uart_fifo.o(.constdata) for .constdata
    app_uart_fifo.o(i.app_uart_init) refers to app_uart_fifo.o(i.gpiote_uart_event_handler) for gpiote_uart_event_handler
    app_uart_fifo.o(i.app_uart_put) refers to app_fifo.o(i.app_fifo_put) for app_fifo_put
    app_uart_fifo.o(i.app_uart_put) refers to app_uart_fifo.o(i.on_uart_event) for on_uart_event
    app_uart_fifo.o(i.app_uart_put) refers to app_uart_fifo.o(.bss) for .bss
    app_uart_fifo.o(i.gpiote_uart_event_handler) refers to nrf_drv_gpiote.o(i.nrf_drv_gpiote_in_is_set) for nrf_drv_gpiote_in_is_set
    app_uart_fifo.o(i.gpiote_uart_event_handler) refers to app_uart_fifo.o(i.on_uart_event) for on_uart_event
    app_uart_fifo.o(i.on_uart_event) refers to client_handling.o(i.__ARM_common_switch8) for __ARM_common_switch8
    app_uart_fifo.o(i.on_uart_event) refers to app_uart_fifo.o(i.action_tx_send) for action_tx_send
    app_uart_fifo.o(i.on_uart_event) refers to app_uart_fifo.o(i.action_uart_deactivate) for action_uart_deactivate
    app_uart_fifo.o(i.on_uart_event) refers to app_uart_fifo.o(i.action_tx_stop) for action_tx_stop
    app_uart_fifo.o(i.on_uart_event) refers to app_uart_fifo.o(.bss) for .bss
    app_uart_fifo.o(i.on_uart_event) refers to app_uart_fifo.o(.data) for .data
    pstorage.o(i.app_notify) refers to pstorage.o(.bss) for .bss
    pstorage.o(i.app_notify) refers to pstorage.o(.data) for .data
    pstorage.o(i.app_notify_error_state_transit) refers to pstorage.o(i.app_notify) for app_notify
    pstorage.o(i.app_notify_error_state_transit) refers to pstorage.o(i.sm_state_change) for sm_state_change
    pstorage.o(i.app_notify_error_state_transit) refers to pstorage.o(.bss) for .bss
    pstorage.o(i.clear_operation_execute) refers to pstorage.o(i.pstorage_flash_page_size) for pstorage_flash_page_size
    pstorage.o(i.clear_operation_execute) refers to uidiv.o(.text) for __aeabi_uidivmod
    pstorage.o(i.clear_operation_execute) refers to pstorage.o(i.sm_state_change) for sm_state_change
    pstorage.o(i.clear_operation_execute) refers to pstorage.o(.bss) for .bss
    pstorage.o(i.clear_operation_execute) refers to pstorage.o(.data) for .data
    pstorage.o(i.clear_post_processing_run) refers to pstorage.o(i.command_end_procedure_run) for command_end_procedure_run
    pstorage.o(i.clear_post_processing_run) refers to pstorage.o(i.sm_state_change) for sm_state_change
    pstorage.o(i.clear_post_processing_run) refers to pstorage.o(.bss) for .bss
    pstorage.o(i.cmd_process) refers to pstorage.o(i.clear_operation_execute) for clear_operation_execute
    pstorage.o(i.cmd_process) refers to pstorage.o(i.sm_state_change) for sm_state_change
    pstorage.o(i.cmd_process) refers to pstorage.o(.bss) for .bss
    pstorage.o(i.cmd_process) refers to pstorage.o(.data) for .data
    pstorage.o(i.cmd_queue_element_init) refers to pstorage.o(.bss) for .bss
    pstorage.o(i.cmd_queue_enqueue) refers to pstorage.o(i.cmd_process) for cmd_process
    pstorage.o(i.cmd_queue_enqueue) refers to pstorage.o(.bss) for .bss
    pstorage.o(i.cmd_queue_enqueue) refers to pstorage.o(.data) for .data
    pstorage.o(i.command_end_procedure_run) refers to pstorage.o(i.app_notify) for app_notify
    pstorage.o(i.command_end_procedure_run) refers to pstorage.o(i.cmd_queue_element_init) for cmd_queue_element_init
    pstorage.o(i.command_end_procedure_run) refers to pstorage.o(i.sm_state_change) for sm_state_change
    pstorage.o(i.command_end_procedure_run) refers to pstorage.o(.bss) for .bss
    pstorage.o(i.data_page_erase_state_run) refers to pstorage.o(i.is_page_erase_required) for is_page_erase_required
    pstorage.o(i.data_page_erase_state_run) refers to pstorage.o(i.swap_sub_state_state_change) for swap_sub_state_state_change
    pstorage.o(i.data_page_erase_state_run) refers to pstorage.o(i.clear_post_processing_run) for clear_post_processing_run
    pstorage.o(i.data_page_erase_state_run) refers to pstorage.o(i.swap_sub_state_err_busy_process) for swap_sub_state_err_busy_process
    pstorage.o(i.data_page_erase_state_run) refers to pstorage.o(.data) for .data
    pstorage.o(i.data_to_swap_write_state_run) refers to pstorage.o(i.swap_sub_state_state_change) for swap_sub_state_state_change
    pstorage.o(i.data_to_swap_write_state_run) refers to pstorage.o(i.swap_sub_state_err_busy_process) for swap_sub_state_err_busy_process
    pstorage.o(i.data_to_swap_write_state_run) refers to pstorage.o(.data) for .data
    pstorage.o(i.flash_api_err_code_process) refers to pstorage.o(i.app_notify_error_state_transit) for app_notify_error_state_transit
    pstorage.o(i.flash_api_err_code_process) refers to pstorage.o(.data) for .data
    pstorage.o(i.flash_operation_success_run) refers to pstorage.o(i.store_cmd_flash_write_execute) for store_cmd_flash_write_execute
    pstorage.o(i.flash_operation_success_run) refers to pstorage.o(i.command_end_procedure_run) for command_end_procedure_run
    pstorage.o(i.flash_operation_success_run) refers to pstorage.o(i.main_state_err_busy_process) for main_state_err_busy_process
    pstorage.o(i.flash_operation_success_run) refers to pstorage.o(i.is_page_erase_required) for is_page_erase_required
    pstorage.o(i.flash_operation_success_run) refers to pstorage.o(i.sm_state_change) for sm_state_change
    pstorage.o(i.flash_operation_success_run) refers to pstorage.o(i.clear_post_processing_run) for clear_post_processing_run
    pstorage.o(i.flash_operation_success_run) refers to pstorage.o(.data) for .data
    pstorage.o(i.flash_operation_success_run) refers to pstorage.o(.bss) for .bss
    pstorage.o(i.flash_operation_success_run) refers to pstorage.o(.constdata) for .constdata
    pstorage.o(i.flash_page_erase) refers to pstorage.o(i.flash_api_err_code_process) for flash_api_err_code_process
    pstorage.o(i.flash_write) refers to pstorage.o(i.flash_api_err_code_process) for flash_api_err_code_process
    pstorage.o(i.head_restore_state_run) refers to pstorage.o(i.pstorage_flash_page_size) for pstorage_flash_page_size
    pstorage.o(i.head_restore_state_run) refers to uidiv.o(.text) for __aeabi_uidivmod
    pstorage.o(i.head_restore_state_run) refers to pstorage.o(i.is_page_erase_required) for is_page_erase_required
    pstorage.o(i.head_restore_state_run) refers to pstorage.o(i.swap_sub_state_state_change) for swap_sub_state_state_change
    pstorage.o(i.head_restore_state_run) refers to pstorage.o(i.clear_post_processing_run) for clear_post_processing_run
    pstorage.o(i.head_restore_state_run) refers to pstorage.o(i.swap_sub_state_err_busy_process) for swap_sub_state_err_busy_process
    pstorage.o(i.head_restore_state_run) refers to pstorage.o(.data) for .data
    pstorage.o(i.head_restore_state_run) refers to pstorage.o(.bss) for .bss
    pstorage.o(i.is_page_erase_required) refers to pstorage.o(i.pstorage_flash_page_size) for pstorage_flash_page_size
    pstorage.o(i.is_page_erase_required) refers to uidiv.o(.text) for __aeabi_uidivmod
    pstorage.o(i.is_page_erase_required) refers to pstorage.o(.bss) for .bss
    pstorage.o(i.is_page_erase_required) refers to pstorage.o(.data) for .data
    pstorage.o(i.main_state_err_busy_process) refers to pstorage.o(i.sm_state_change) for sm_state_change
    pstorage.o(i.main_state_err_busy_process) refers to pstorage.o(.data) for .data
    pstorage.o(i.pstorage_access_status_get) refers to pstorage.o(.data) for .data
    pstorage.o(i.pstorage_access_status_get) refers to pstorage.o(.bss) for .bss
    pstorage.o(i.pstorage_block_identifier_get) refers to pstorage.o(.data) for .data
    pstorage.o(i.pstorage_block_identifier_get) refers to pstorage.o(.bss) for .bss
    pstorage.o(i.pstorage_clear) refers to pstorage.o(i.is_word_aligned) for is_word_aligned
    pstorage.o(i.pstorage_clear) refers to uidiv.o(.text) for __aeabi_uidivmod
    pstorage.o(i.pstorage_clear) refers to pstorage.o(i.cmd_queue_enqueue) for cmd_queue_enqueue
    pstorage.o(i.pstorage_clear) refers to pstorage.o(.data) for .data
    pstorage.o(i.pstorage_clear) refers to pstorage.o(.bss) for .bss
    pstorage.o(i.pstorage_flash_page_end) refers to pstorage.o(i.pstorage_flash_page_size) for pstorage_flash_page_size
    pstorage.o(i.pstorage_flash_page_end) refers to uidiv.o(.text) for __aeabi_uidivmod
    pstorage.o(i.pstorage_init) refers to pstorage.o(i.cmd_queue_element_init) for cmd_queue_element_init
    pstorage.o(i.pstorage_init) refers to pstorage.o(i.pstorage_flash_page_end) for pstorage_flash_page_end
    pstorage.o(i.pstorage_init) refers to pstorage.o(i.pstorage_flash_page_size) for pstorage_flash_page_size
    pstorage.o(i.pstorage_init) refers to pstorage.o(.bss) for .bss
    pstorage.o(i.pstorage_init) refers to pstorage.o(.data) for .data
    pstorage.o(i.pstorage_load) refers to pstorage.o(i.is_word_aligned) for is_word_aligned
    pstorage.o(i.pstorage_load) refers to memcpya.o(.text) for __aeabi_memcpy
    pstorage.o(i.pstorage_load) refers to pstorage.o(.data) for .data
    pstorage.o(i.pstorage_load) refers to pstorage.o(.bss) for .bss
    pstorage.o(i.pstorage_register) refers to pstorage.o(i.pstorage_flash_page_size) for pstorage_flash_page_size
    pstorage.o(i.pstorage_register) refers to pstorage.o(i.pstorage_flash_page_end) for pstorage_flash_page_end
    pstorage.o(i.pstorage_register) refers to idiv.o(.text) for __aeabi_idivmod
    pstorage.o(i.pstorage_register) refers to pstorage.o(.data) for .data
    pstorage.o(i.pstorage_register) refers to pstorage.o(.bss) for .bss
    pstorage.o(i.pstorage_store) refers to pstorage.o(i.is_word_aligned) for is_word_aligned
    pstorage.o(i.pstorage_store) refers to pstorage.o(i.cmd_queue_enqueue) for cmd_queue_enqueue
    pstorage.o(i.pstorage_store) refers to pstorage.o(.data) for .data
    pstorage.o(i.pstorage_store) refers to pstorage.o(.bss) for .bss
    pstorage.o(i.pstorage_sys_event_handler) refers to pstorage.o(i.sm_state_change) for sm_state_change
    pstorage.o(i.pstorage_sys_event_handler) refers to pstorage.o(i.swap_sub_state_state_change) for swap_sub_state_state_change
    pstorage.o(i.pstorage_sys_event_handler) refers to pstorage.o(i.app_notify_error_state_transit) for app_notify_error_state_transit
    pstorage.o(i.pstorage_sys_event_handler) refers to pstorage.o(i.flash_operation_success_run) for flash_operation_success_run
    pstorage.o(i.pstorage_sys_event_handler) refers to pstorage.o(.data) for .data
    pstorage.o(i.pstorage_update) refers to pstorage.o(i.is_word_aligned) for is_word_aligned
    pstorage.o(i.pstorage_update) refers to pstorage.o(i.cmd_queue_enqueue) for cmd_queue_enqueue
    pstorage.o(i.pstorage_update) refers to pstorage.o(.data) for .data
    pstorage.o(i.pstorage_update) refers to pstorage.o(.bss) for .bss
    pstorage.o(i.sm_state_change) refers to pstorage.o(i.flash_page_erase) for flash_page_erase
    pstorage.o(i.sm_state_change) refers to pstorage.o(i.cmd_process) for cmd_process
    pstorage.o(i.sm_state_change) refers to pstorage.o(i.store_cmd_flash_write_execute) for store_cmd_flash_write_execute
    pstorage.o(i.sm_state_change) refers to pstorage.o(i.state_data_erase_swap_entry_run) for state_data_erase_swap_entry_run
    pstorage.o(i.sm_state_change) refers to pstorage.o(.data) for .data
    pstorage.o(i.sm_state_change) refers to pstorage.o(.bss) for .bss
    pstorage.o(i.state_data_erase_swap_entry_run) refers to pstorage.o(i.pstorage_flash_page_size) for pstorage_flash_page_size
    pstorage.o(i.state_data_erase_swap_entry_run) refers to uidiv.o(.text) for __aeabi_uidivmod
    pstorage.o(i.state_data_erase_swap_entry_run) refers to pstorage.o(i.swap_sub_state_state_change) for swap_sub_state_state_change
    pstorage.o(i.state_data_erase_swap_entry_run) refers to pstorage.o(.data) for .data
    pstorage.o(i.state_data_erase_swap_entry_run) refers to pstorage.o(.bss) for .bss
    pstorage.o(i.state_erase_data_page_entry_run) refers to pstorage.o(i.flash_page_erase) for flash_page_erase
    pstorage.o(i.state_erase_data_page_entry_run) refers to pstorage.o(.data) for .data
    pstorage.o(i.state_restore_head_entry_run) refers to pstorage.o(i.pstorage_flash_page_end) for pstorage_flash_page_end
    pstorage.o(i.state_restore_head_entry_run) refers to pstorage.o(i.pstorage_flash_page_size) for pstorage_flash_page_size
    pstorage.o(i.state_restore_head_entry_run) refers to pstorage.o(i.flash_write) for flash_write
    pstorage.o(i.state_restore_head_entry_run) refers to pstorage.o(.data) for .data
    pstorage.o(i.state_restore_tail_entry_run) refers to pstorage.o(i.pstorage_flash_page_size) for pstorage_flash_page_size
    pstorage.o(i.state_restore_tail_entry_run) refers to uidiv.o(.text) for __aeabi_uidivmod
    pstorage.o(i.state_restore_tail_entry_run) refers to pstorage.o(i.pstorage_flash_page_end) for pstorage_flash_page_end
    pstorage.o(i.state_restore_tail_entry_run) refers to pstorage.o(i.flash_write) for flash_write
    pstorage.o(i.state_restore_tail_entry_run) refers to pstorage.o(.bss) for .bss
    pstorage.o(i.state_restore_tail_entry_run) refers to pstorage.o(.data) for .data
    pstorage.o(i.state_swap_erase_entry_run) refers to pstorage.o(i.pstorage_flash_page_size) for pstorage_flash_page_size
    pstorage.o(i.state_swap_erase_entry_run) refers to pstorage.o(i.pstorage_flash_page_end) for pstorage_flash_page_end
    pstorage.o(i.state_swap_erase_entry_run) refers to uidiv.o(.text) for __aeabi_uidivmod
    pstorage.o(i.state_swap_erase_entry_run) refers to pstorage.o(i.flash_page_erase) for flash_page_erase
    pstorage.o(i.state_write_data_swap_entry_run) refers to pstorage.o(i.pstorage_flash_page_size) for pstorage_flash_page_size
    pstorage.o(i.state_write_data_swap_entry_run) refers to pstorage.o(i.pstorage_flash_page_end) for pstorage_flash_page_end
    pstorage.o(i.state_write_data_swap_entry_run) refers to pstorage.o(i.flash_write) for flash_write
    pstorage.o(i.state_write_data_swap_entry_run) refers to pstorage.o(.data) for .data
    pstorage.o(i.store_cmd_flash_write_execute) refers to pstorage.o(i.pstorage_flash_page_size) for pstorage_flash_page_size
    pstorage.o(i.store_cmd_flash_write_execute) refers to pstorage.o(i.flash_write) for flash_write
    pstorage.o(i.store_cmd_flash_write_execute) refers to pstorage.o(.bss) for .bss
    pstorage.o(i.store_cmd_flash_write_execute) refers to pstorage.o(.data) for .data
    pstorage.o(i.swap_erase_state_run) refers to pstorage.o(i.swap_sub_state_state_change) for swap_sub_state_state_change
    pstorage.o(i.swap_erase_state_run) refers to pstorage.o(i.swap_sub_state_err_busy_process) for swap_sub_state_err_busy_process
    pstorage.o(i.swap_erase_state_run) refers to pstorage.o(.data) for .data
    pstorage.o(i.swap_sub_state_err_busy_process) refers to pstorage.o(i.swap_sub_state_state_change) for swap_sub_state_state_change
    pstorage.o(i.swap_sub_state_err_busy_process) refers to pstorage.o(.data) for .data
    pstorage.o(i.swap_sub_state_state_change) refers to pstorage.o(.data) for .data
    pstorage.o(i.swap_sub_state_state_change) refers to pstorage.o(.constdata) for .constdata
    pstorage.o(i.tail_restore_state_run) refers to pstorage.o(i.clear_post_processing_run) for clear_post_processing_run
    pstorage.o(i.tail_restore_state_run) refers to pstorage.o(i.swap_sub_state_err_busy_process) for swap_sub_state_err_busy_process
    pstorage.o(i.tail_restore_state_run) refers to pstorage.o(.data) for .data
    pstorage.o(.constdata) refers to pstorage.o(i.state_swap_erase_entry_run) for state_swap_erase_entry_run
    pstorage.o(.constdata) refers to pstorage.o(i.state_write_data_swap_entry_run) for state_write_data_swap_entry_run
    pstorage.o(.constdata) refers to pstorage.o(i.state_erase_data_page_entry_run) for state_erase_data_page_entry_run
    pstorage.o(.constdata) refers to pstorage.o(i.state_restore_tail_entry_run) for state_restore_tail_entry_run
    pstorage.o(.constdata) refers to pstorage.o(i.state_restore_head_entry_run) for state_restore_head_entry_run
    pstorage.o(.constdata) refers to pstorage.o(i.swap_erase_state_run) for swap_erase_state_run
    pstorage.o(.constdata) refers to pstorage.o(i.data_to_swap_write_state_run) for data_to_swap_write_state_run
    pstorage.o(.constdata) refers to pstorage.o(i.data_page_erase_state_run) for data_page_erase_state_run
    pstorage.o(.constdata) refers to pstorage.o(i.tail_restore_state_run) for tail_restore_state_run
    pstorage.o(.constdata) refers to pstorage.o(i.head_restore_state_run) for head_restore_state_run
    nrf_drv_gpiote.o(i.GPIOTE_IRQHandler) refers to nrf_drv_gpiote.o(i.nrf_gpiote_event_is_set) for nrf_gpiote_event_is_set
    nrf_drv_gpiote.o(i.GPIOTE_IRQHandler) refers to nrf_drv_gpiote.o(i.channel_port_get) for channel_port_get
    nrf_drv_gpiote.o(i.GPIOTE_IRQHandler) refers to nrf_drv_gpiote.o(i.nrf_gpio_cfg_sense_set) for nrf_gpio_cfg_sense_set
    nrf_drv_gpiote.o(i.GPIOTE_IRQHandler) refers to nrf_drv_gpiote.o(.bss) for .bss
    nrf_drv_gpiote.o(i.channel_free) refers to nrf_drv_gpiote.o(.bss) for .bss
    nrf_drv_gpiote.o(i.channel_port_alloc) refers to nrf_drv_gpiote.o(.bss) for .bss
    nrf_drv_gpiote.o(i.channel_port_get) refers to nrf_drv_gpiote.o(.bss) for .bss
    nrf_drv_gpiote.o(i.nrf_drv_gpiote_in_event_addr_get) refers to nrf_drv_gpiote.o(i.channel_port_get) for channel_port_get
    nrf_drv_gpiote.o(i.nrf_drv_gpiote_in_event_disable) refers to nrf_drv_gpiote.o(i.pin_in_use_by_port) for pin_in_use_by_port
    nrf_drv_gpiote.o(i.nrf_drv_gpiote_in_event_disable) refers to nrf_drv_gpiote.o(i.pin_in_use_by_te) for pin_in_use_by_te
    nrf_drv_gpiote.o(i.nrf_drv_gpiote_in_event_disable) refers to nrf_drv_gpiote.o(i.channel_port_get) for channel_port_get
    nrf_drv_gpiote.o(i.nrf_drv_gpiote_in_event_enable) refers to nrf_drv_gpiote.o(i.pin_in_use_by_port) for pin_in_use_by_port
    nrf_drv_gpiote.o(i.nrf_drv_gpiote_in_event_enable) refers to nrf_drv_gpiote.o(i.channel_port_get) for channel_port_get
    nrf_drv_gpiote.o(i.nrf_drv_gpiote_in_event_enable) refers to nrf_drv_gpiote.o(i.nrf_gpio_cfg_sense_set) for nrf_gpio_cfg_sense_set
    nrf_drv_gpiote.o(i.nrf_drv_gpiote_in_event_enable) refers to nrf_drv_gpiote.o(i.pin_in_use_by_te) for pin_in_use_by_te
    nrf_drv_gpiote.o(i.nrf_drv_gpiote_in_event_enable) refers to nrf_drv_gpiote.o(.bss) for .bss
    nrf_drv_gpiote.o(i.nrf_drv_gpiote_in_init) refers to nrf_drv_gpiote.o(i.channel_port_alloc) for channel_port_alloc
    nrf_drv_gpiote.o(i.nrf_drv_gpiote_in_init) refers to nrf_drv_gpiote.o(.bss) for .bss
    nrf_drv_gpiote.o(i.nrf_drv_gpiote_in_uninit) refers to nrf_drv_gpiote.o(i.nrf_drv_gpiote_in_event_disable) for nrf_drv_gpiote_in_event_disable
    nrf_drv_gpiote.o(i.nrf_drv_gpiote_in_uninit) refers to nrf_drv_gpiote.o(i.pin_in_use_by_te) for pin_in_use_by_te
    nrf_drv_gpiote.o(i.nrf_drv_gpiote_in_uninit) refers to nrf_drv_gpiote.o(i.channel_port_get) for channel_port_get
    nrf_drv_gpiote.o(i.nrf_drv_gpiote_in_uninit) refers to nrf_drv_gpiote.o(i.channel_free) for channel_free
    nrf_drv_gpiote.o(i.nrf_drv_gpiote_in_uninit) refers to nrf_drv_gpiote.o(.bss) for .bss
    nrf_drv_gpiote.o(i.nrf_drv_gpiote_init) refers to nrf_drv_gpiote.o(i.channel_free) for channel_free
    nrf_drv_gpiote.o(i.nrf_drv_gpiote_init) refers to nrf_drv_common.o(i.nrf_drv_common_irq_enable) for nrf_drv_common_irq_enable
    nrf_drv_gpiote.o(i.nrf_drv_gpiote_init) refers to nrf_drv_gpiote.o(.bss) for .bss
    nrf_drv_gpiote.o(i.nrf_drv_gpiote_is_init) refers to nrf_drv_gpiote.o(.bss) for .bss
    nrf_drv_gpiote.o(i.nrf_drv_gpiote_out_init) refers to nrf_drv_gpiote.o(i.channel_port_alloc) for channel_port_alloc
    nrf_drv_gpiote.o(i.nrf_drv_gpiote_out_init) refers to nrf_drv_gpiote.o(.bss) for .bss
    nrf_drv_gpiote.o(i.nrf_drv_gpiote_out_task_addr_get) refers to nrf_drv_gpiote.o(i.channel_port_get) for channel_port_get
    nrf_drv_gpiote.o(i.nrf_drv_gpiote_out_task_disable) refers to nrf_drv_gpiote.o(.bss) for .bss
    nrf_drv_gpiote.o(i.nrf_drv_gpiote_out_task_enable) refers to nrf_drv_gpiote.o(.bss) for .bss
    nrf_drv_gpiote.o(i.nrf_drv_gpiote_out_task_force) refers to nrf_drv_gpiote.o(.bss) for .bss
    nrf_drv_gpiote.o(i.nrf_drv_gpiote_out_task_trigger) refers to nrf_drv_gpiote.o(i.channel_port_get) for channel_port_get
    nrf_drv_gpiote.o(i.nrf_drv_gpiote_out_uninit) refers to nrf_drv_gpiote.o(i.pin_in_use_by_te) for pin_in_use_by_te
    nrf_drv_gpiote.o(i.nrf_drv_gpiote_out_uninit) refers to nrf_drv_gpiote.o(i.channel_free) for channel_free
    nrf_drv_gpiote.o(i.nrf_drv_gpiote_out_uninit) refers to nrf_drv_gpiote.o(.bss) for .bss
    nrf_drv_gpiote.o(i.nrf_drv_gpiote_uninit) refers to nrf_drv_gpiote.o(i.nrf_drv_gpiote_in_uninit) for nrf_drv_gpiote_in_uninit
    nrf_drv_gpiote.o(i.nrf_drv_gpiote_uninit) refers to nrf_drv_gpiote.o(i.nrf_drv_gpiote_out_uninit) for nrf_drv_gpiote_out_uninit
    nrf_drv_gpiote.o(i.nrf_drv_gpiote_uninit) refers to nrf_drv_gpiote.o(.bss) for .bss
    nrf_drv_gpiote.o(i.pin_in_use_by_port) refers to nrf_drv_gpiote.o(.bss) for .bss
    nrf_drv_gpiote.o(i.pin_in_use_by_te) refers to nrf_drv_gpiote.o(.bss) for .bss
    nrf_delay.o(i.nrf_delay_ms) refers to nrf_delay.o(.emb_text) for __asm___11_nrf_delay_c_532987f3__nrf_delay_us
    nrf_drv_ppi.o(i.is_allocated_channel) refers to nrf_drv_ppi.o(.data) for .data
    nrf_drv_ppi.o(i.is_allocated_group) refers to nrf_drv_ppi.o(.data) for .data
    nrf_drv_ppi.o(i.is_app_channel) refers to nrf_drv_ppi.o(i.are_app_channels) for are_app_channels
    nrf_drv_ppi.o(i.nrf_drv_ppi_channel_alloc) refers to nrf_drv_ppi.o(i.current_int_priority_get) for current_int_priority_get
    nrf_drv_ppi.o(i.nrf_drv_ppi_channel_alloc) refers to app_error.o(i.app_error_handler) for app_error_handler
    nrf_drv_ppi.o(i.nrf_drv_ppi_channel_alloc) refers to nrf_drv_ppi.o(i.is_allocated_channel) for is_allocated_channel
    nrf_drv_ppi.o(i.nrf_drv_ppi_channel_alloc) refers to nrf_drv_ppi.o(.data) for .data
    nrf_drv_ppi.o(i.nrf_drv_ppi_channel_assign) refers to nrf_drv_ppi.o(i.is_programmable_app_channel) for is_programmable_app_channel
    nrf_drv_ppi.o(i.nrf_drv_ppi_channel_assign) refers to nrf_drv_ppi.o(i.is_allocated_channel) for is_allocated_channel
    nrf_drv_ppi.o(i.nrf_drv_ppi_channel_disable) refers to nrf_drv_ppi.o(i.is_app_channel) for is_app_channel
    nrf_drv_ppi.o(i.nrf_drv_ppi_channel_disable) refers to nrf_drv_ppi.o(i.is_programmable_app_channel) for is_programmable_app_channel
    nrf_drv_ppi.o(i.nrf_drv_ppi_channel_disable) refers to nrf_drv_ppi.o(i.is_allocated_channel) for is_allocated_channel
    nrf_drv_ppi.o(i.nrf_drv_ppi_channel_enable) refers to nrf_drv_ppi.o(i.is_app_channel) for is_app_channel
    nrf_drv_ppi.o(i.nrf_drv_ppi_channel_enable) refers to nrf_drv_ppi.o(i.is_programmable_app_channel) for is_programmable_app_channel
    nrf_drv_ppi.o(i.nrf_drv_ppi_channel_enable) refers to nrf_drv_ppi.o(i.is_allocated_channel) for is_allocated_channel
    nrf_drv_ppi.o(i.nrf_drv_ppi_channel_free) refers to nrf_drv_ppi.o(i.is_programmable_app_channel) for is_programmable_app_channel
    nrf_drv_ppi.o(i.nrf_drv_ppi_channel_free) refers to nrf_drv_ppi.o(i.current_int_priority_get) for current_int_priority_get
    nrf_drv_ppi.o(i.nrf_drv_ppi_channel_free) refers to app_error.o(i.app_error_handler) for app_error_handler
    nrf_drv_ppi.o(i.nrf_drv_ppi_channel_free) refers to nrf_drv_ppi.o(.data) for .data
    nrf_drv_ppi.o(i.nrf_drv_ppi_channels_include_in_group) refers to nrf_drv_ppi.o(i.is_app_group) for is_app_group
    nrf_drv_ppi.o(i.nrf_drv_ppi_channels_include_in_group) refers to nrf_drv_ppi.o(i.is_allocated_group) for is_allocated_group
    nrf_drv_ppi.o(i.nrf_drv_ppi_channels_include_in_group) refers to nrf_drv_ppi.o(i.are_app_channels) for are_app_channels
    nrf_drv_ppi.o(i.nrf_drv_ppi_channels_include_in_group) refers to nrf_drv_ppi.o(i.current_int_priority_get) for current_int_priority_get
    nrf_drv_ppi.o(i.nrf_drv_ppi_channels_include_in_group) refers to app_error.o(i.app_error_handler) for app_error_handler
    nrf_drv_ppi.o(i.nrf_drv_ppi_channels_remove_from_group) refers to nrf_drv_ppi.o(i.is_app_group) for is_app_group
    nrf_drv_ppi.o(i.nrf_drv_ppi_channels_remove_from_group) refers to nrf_drv_ppi.o(i.is_allocated_group) for is_allocated_group
    nrf_drv_ppi.o(i.nrf_drv_ppi_channels_remove_from_group) refers to nrf_drv_ppi.o(i.are_app_channels) for are_app_channels
    nrf_drv_ppi.o(i.nrf_drv_ppi_channels_remove_from_group) refers to nrf_drv_ppi.o(i.current_int_priority_get) for current_int_priority_get
    nrf_drv_ppi.o(i.nrf_drv_ppi_channels_remove_from_group) refers to app_error.o(i.app_error_handler) for app_error_handler
    nrf_drv_ppi.o(i.nrf_drv_ppi_group_alloc) refers to nrf_drv_ppi.o(i.current_int_priority_get) for current_int_priority_get
    nrf_drv_ppi.o(i.nrf_drv_ppi_group_alloc) refers to app_error.o(i.app_error_handler) for app_error_handler
    nrf_drv_ppi.o(i.nrf_drv_ppi_group_alloc) refers to nrf_drv_ppi.o(i.is_allocated_group) for is_allocated_group
    nrf_drv_ppi.o(i.nrf_drv_ppi_group_alloc) refers to nrf_drv_ppi.o(.data) for .data
    nrf_drv_ppi.o(i.nrf_drv_ppi_group_disable) refers to nrf_drv_ppi.o(i.is_app_group) for is_app_group
    nrf_drv_ppi.o(i.nrf_drv_ppi_group_enable) refers to nrf_drv_ppi.o(i.is_app_group) for is_app_group
    nrf_drv_ppi.o(i.nrf_drv_ppi_group_enable) refers to nrf_drv_ppi.o(i.is_allocated_group) for is_allocated_group
    nrf_drv_ppi.o(i.nrf_drv_ppi_group_free) refers to nrf_drv_ppi.o(i.is_app_group) for is_app_group
    nrf_drv_ppi.o(i.nrf_drv_ppi_group_free) refers to nrf_drv_ppi.o(i.is_allocated_group) for is_allocated_group
    nrf_drv_ppi.o(i.nrf_drv_ppi_group_free) refers to nrf_drv_ppi.o(i.current_int_priority_get) for current_int_priority_get
    nrf_drv_ppi.o(i.nrf_drv_ppi_group_free) refers to app_error.o(i.app_error_handler) for app_error_handler
    nrf_drv_ppi.o(i.nrf_drv_ppi_group_free) refers to nrf_drv_ppi.o(.data) for .data
    nrf_drv_ppi.o(i.nrf_drv_ppi_init) refers to nrf_drv_ppi.o(.data) for .data
    nrf_drv_ppi.o(i.nrf_drv_ppi_uninit) refers to nrf_drv_ppi.o(.data) for .data
    nrf_drv_timer.o(i.TIMER1_IRQHandler) refers to nrf_drv_timer.o(.data) for .data
    nrf_drv_timer.o(i.nrf_drv_timer_disable) refers to nrf_drv_timer.o(.data) for .data
    nrf_drv_timer.o(i.nrf_drv_timer_enable) refers to nrf_drv_timer.o(.data) for .data
    nrf_drv_timer.o(i.nrf_drv_timer_extended_compare) refers to nrf_drv_timer.o(i.nrf_drv_timer_compare) for nrf_drv_timer_compare
    nrf_drv_timer.o(i.nrf_drv_timer_init) refers to nrf_drv_common.o(i.nrf_drv_common_irq_enable) for nrf_drv_common_irq_enable
    nrf_drv_timer.o(i.nrf_drv_timer_init) refers to nrf_drv_timer.o(.data) for .data
    nrf_drv_timer.o(i.nrf_drv_timer_init) refers to nrf_drv_timer.o(.constdata) for .constdata
    nrf_drv_timer.o(i.nrf_drv_timer_uninit) refers to nrf_drv_timer.o(i.nrf_drv_timer_disable) for nrf_drv_timer_disable
    nrf_drv_timer.o(i.nrf_drv_timer_uninit) refers to nrf_drv_timer.o(.data) for .data
    app_pwm.o(i.app_pwm_channel_duty_get) refers to app_pwm.o(i.app_pwm_channel_duty_ticks_get) for app_pwm_channel_duty_ticks_get
    app_pwm.o(i.app_pwm_channel_duty_get) refers to uidiv.o(.text) for __aeabi_uidivmod
    app_pwm.o(i.app_pwm_channel_duty_set) refers to uidiv.o(.text) for __aeabi_uidivmod
    app_pwm.o(i.app_pwm_channel_duty_set) refers to app_pwm.o(i.app_pwm_channel_duty_ticks_set) for app_pwm_channel_duty_ticks_set
    app_pwm.o(i.app_pwm_channel_duty_ticks_set) refers to app_pwm.o(i.pwm_transition_0or100_to_0or100) for pwm_transition_0or100_to_0or100
    app_pwm.o(i.app_pwm_channel_duty_ticks_set) refers to app_pwm.o(i.pwm_transition_0or100_to_n) for pwm_transition_0or100_to_n
    app_pwm.o(i.app_pwm_channel_duty_ticks_set) refers to app_pwm.o(i.pwm_transition_n_to_0or100) for pwm_transition_n_to_0or100
    app_pwm.o(i.app_pwm_channel_duty_ticks_set) refers to app_pwm.o(i.pwm_transition_n_to_m) for pwm_transition_n_to_m
    app_pwm.o(i.app_pwm_channel_duty_ticks_set) refers to nrf_drv_timer.o(i.nrf_drv_timer_compare_int_enable) for nrf_drv_timer_compare_int_enable
    app_pwm.o(i.app_pwm_channel_duty_ticks_set) refers to app_pwm.o(.data) for .data
    app_pwm.o(i.app_pwm_channel_init) refers to nrf_drv_gpiote.o(i.nrf_drv_gpiote_out_init) for nrf_drv_gpiote_out_init
    app_pwm.o(i.app_pwm_channel_init) refers to nrf_drv_gpiote.o(i.nrf_drv_gpiote_out_task_enable) for nrf_drv_gpiote_out_task_enable
    app_pwm.o(i.app_pwm_channel_init) refers to nrf_drv_ppi.o(i.nrf_drv_ppi_channel_alloc) for nrf_drv_ppi_channel_alloc
    app_pwm.o(i.app_pwm_channel_init) refers to nrf_drv_ppi.o(i.nrf_drv_ppi_channel_disable) for nrf_drv_ppi_channel_disable
    app_pwm.o(i.app_pwm_channel_init) refers to nrf_drv_gpiote.o(i.nrf_drv_gpiote_out_task_addr_get) for nrf_drv_gpiote_out_task_addr_get
    app_pwm.o(i.app_pwm_channel_init) refers to nrf_drv_timer.o(i.nrf_drv_timer_compare_event_address_get) for nrf_drv_timer_compare_event_address_get
    app_pwm.o(i.app_pwm_channel_init) refers to nrf_drv_ppi.o(i.nrf_drv_ppi_channel_assign) for nrf_drv_ppi_channel_assign
    app_pwm.o(i.app_pwm_channel_init) refers to nrf_drv_gpiote.o(i.nrf_drv_gpiote_out_task_trigger) for nrf_drv_gpiote_out_task_trigger
    app_pwm.o(i.app_pwm_channel_init) refers to app_pwm.o(.constdata) for .constdata
    app_pwm.o(i.app_pwm_disable) refers to nrf_drv_timer.o(i.nrf_drv_timer_disable) for nrf_drv_timer_disable
    app_pwm.o(i.app_pwm_disable) refers to nrf_drv_timer.o(i.nrf_drv_timer_compare_int_disable) for nrf_drv_timer_compare_int_disable
    app_pwm.o(i.app_pwm_enable) refers to nrf_drv_timer.o(i.nrf_drv_timer_enable) for nrf_drv_timer_enable
    app_pwm.o(i.app_pwm_init) refers to nrf_drv_ppi.o(i.nrf_drv_ppi_init) for nrf_drv_ppi_init
    app_pwm.o(i.app_pwm_init) refers to nrf_drv_gpiote.o(i.nrf_drv_gpiote_is_init) for nrf_drv_gpiote_is_init
    app_pwm.o(i.app_pwm_init) refers to nrf_drv_gpiote.o(i.nrf_drv_gpiote_init) for nrf_drv_gpiote_init
    app_pwm.o(i.app_pwm_init) refers to nrf_drv_ppi.o(i.nrf_drv_ppi_channel_alloc) for nrf_drv_ppi_channel_alloc
    app_pwm.o(i.app_pwm_init) refers to nrf_drv_ppi.o(i.nrf_drv_ppi_group_alloc) for nrf_drv_ppi_group_alloc
    app_pwm.o(i.app_pwm_init) refers to app_pwm.o(i.pwm_dealloc) for pwm_dealloc
    app_pwm.o(i.app_pwm_init) refers to app_pwm.o(i.app_pwm_channel_init) for app_pwm_channel_init
    app_pwm.o(i.app_pwm_init) refers to app_pwm.o(i.app_pwm_channel_duty_ticks_set) for app_pwm_channel_duty_ticks_set
    app_pwm.o(i.app_pwm_init) refers to nrf_drv_timer.o(i.nrf_drv_timer_init) for nrf_drv_timer_init
    app_pwm.o(i.app_pwm_init) refers to nrf_drv_timer.o(i.nrf_drv_timer_us_to_ticks) for nrf_drv_timer_us_to_ticks
    app_pwm.o(i.app_pwm_init) refers to nrf_drv_timer.o(i.nrf_drv_timer_clear) for nrf_drv_timer_clear
    app_pwm.o(i.app_pwm_init) refers to nrf_drv_timer.o(i.nrf_drv_timer_extended_compare) for nrf_drv_timer_extended_compare
    app_pwm.o(i.app_pwm_init) refers to nrf_drv_timer.o(i.nrf_drv_timer_compare_int_disable) for nrf_drv_timer_compare_int_disable
    app_pwm.o(i.app_pwm_init) refers to app_pwm.o(i.pan73_workaround) for pan73_workaround
    app_pwm.o(i.app_pwm_init) refers to app_pwm.o(.constdata) for .constdata
    app_pwm.o(i.app_pwm_init) refers to app_pwm.o(i.pwm_ready_tick) for pwm_ready_tick
    app_pwm.o(i.app_pwm_init) refers to app_pwm.o(.data) for .data
    app_pwm.o(i.app_pwm_uninit) refers to app_pwm.o(i.app_pwm_disable) for app_pwm_disable
    app_pwm.o(i.app_pwm_uninit) refers to app_pwm.o(i.pan73_workaround) for pan73_workaround
    app_pwm.o(i.app_pwm_uninit) refers to app_pwm.o(i.pwm_dealloc) for pwm_dealloc
    app_pwm.o(i.pwm_channel_ppi_disable) refers to nrf_drv_ppi.o(i.nrf_drv_ppi_channel_disable) for nrf_drv_ppi_channel_disable
    app_pwm.o(i.pwm_dealloc) refers to nrf_drv_ppi.o(i.nrf_drv_ppi_channel_free) for nrf_drv_ppi_channel_free
    app_pwm.o(i.pwm_dealloc) refers to nrf_drv_ppi.o(i.nrf_drv_ppi_group_free) for nrf_drv_ppi_group_free
    app_pwm.o(i.pwm_dealloc) refers to nrf_drv_gpiote.o(i.nrf_drv_gpiote_out_uninit) for nrf_drv_gpiote_out_uninit
    app_pwm.o(i.pwm_dealloc) refers to nrf_drv_timer.o(i.nrf_drv_timer_uninit) for nrf_drv_timer_uninit
    app_pwm.o(i.pwm_ppi_disable) refers to nrf_drv_ppi.o(i.nrf_drv_ppi_channel_disable) for nrf_drv_ppi_channel_disable
    app_pwm.o(i.pwm_ready_tick) refers to nrf_drv_timer.o(i.nrf_drv_timer_compare_int_disable) for nrf_drv_timer_compare_int_disable
    app_pwm.o(i.pwm_ready_tick) refers to app_pwm.o(.data) for .data
    app_pwm.o(i.pwm_transition_0or100_to_0or100) refers to app_pwm.o(i.pwm_ppi_disable) for pwm_ppi_disable
    app_pwm.o(i.pwm_transition_0or100_to_0or100) refers to app_pwm.o(i.pwm_channel_ppi_disable) for pwm_channel_ppi_disable
    app_pwm.o(i.pwm_transition_0or100_to_0or100) refers to nrf_drv_gpiote.o(i.nrf_drv_gpiote_out_task_force) for nrf_drv_gpiote_out_task_force
    app_pwm.o(i.pwm_transition_0or100_to_0or100) refers to nrf_drv_timer.o(i.nrf_drv_timer_compare) for nrf_drv_timer_compare
    app_pwm.o(i.pwm_transition_0or100_to_n) refers to app_pwm.o(i.pwm_ppi_disable) for pwm_ppi_disable
    app_pwm.o(i.pwm_transition_0or100_to_n) refers to app_pwm.o(i.pwm_channel_ppi_disable) for pwm_channel_ppi_disable
    app_pwm.o(i.pwm_transition_0or100_to_n) refers to nrf_drv_timer.o(i.nrf_drv_timer_compare) for nrf_drv_timer_compare
    app_pwm.o(i.pwm_transition_0or100_to_n) refers to nrf_drv_ppi.o(i.nrf_drv_ppi_channels_remove_from_group) for nrf_drv_ppi_channels_remove_from_group
    app_pwm.o(i.pwm_transition_0or100_to_n) refers to nrf_drv_ppi.o(i.nrf_drv_ppi_channels_include_in_group) for nrf_drv_ppi_channels_include_in_group
    app_pwm.o(i.pwm_transition_0or100_to_n) refers to nrf_drv_timer.o(i.nrf_drv_timer_compare_event_address_get) for nrf_drv_timer_compare_event_address_get
    app_pwm.o(i.pwm_transition_0or100_to_n) refers to nrf_drv_ppi.o(i.nrf_drv_ppi_channel_assign) for nrf_drv_ppi_channel_assign
    app_pwm.o(i.pwm_transition_0or100_to_n) refers to nrf_drv_ppi.o(i.nrf_drv_ppi_channel_enable) for nrf_drv_ppi_channel_enable
    app_pwm.o(i.pwm_transition_n_to_0or100) refers to app_pwm.o(i.pwm_ppi_disable) for pwm_ppi_disable
    app_pwm.o(i.pwm_transition_n_to_0or100) refers to nrf_drv_ppi.o(i.nrf_drv_ppi_channels_remove_from_group) for nrf_drv_ppi_channels_remove_from_group
    app_pwm.o(i.pwm_transition_n_to_0or100) refers to nrf_drv_ppi.o(i.nrf_drv_ppi_channels_include_in_group) for nrf_drv_ppi_channels_include_in_group
    app_pwm.o(i.pwm_transition_n_to_0or100) refers to nrf_drv_timer.o(i.nrf_drv_timer_compare_event_address_get) for nrf_drv_timer_compare_event_address_get
    app_pwm.o(i.pwm_transition_n_to_0or100) refers to nrf_drv_ppi.o(i.nrf_drv_ppi_channel_assign) for nrf_drv_ppi_channel_assign
    app_pwm.o(i.pwm_transition_n_to_0or100) refers to nrf_drv_ppi.o(i.nrf_drv_ppi_channel_enable) for nrf_drv_ppi_channel_enable
    app_pwm.o(i.pwm_transition_n_to_m) refers to app_pwm.o(i.pwm_ppi_disable) for pwm_ppi_disable
    app_pwm.o(i.pwm_transition_n_to_m) refers to nrf_drv_ppi.o(i.nrf_drv_ppi_channels_remove_from_group) for nrf_drv_ppi_channels_remove_from_group
    app_pwm.o(i.pwm_transition_n_to_m) refers to nrf_drv_ppi.o(i.nrf_drv_ppi_channels_include_in_group) for nrf_drv_ppi_channels_include_in_group
    app_pwm.o(i.pwm_transition_n_to_m) refers to nrf_drv_timer.o(i.nrf_drv_timer_compare_event_address_get) for nrf_drv_timer_compare_event_address_get
    app_pwm.o(i.pwm_transition_n_to_m) refers to nrf_drv_ppi.o(i.nrf_drv_ppi_channel_assign) for nrf_drv_ppi_channel_assign
    app_pwm.o(i.pwm_transition_n_to_m) refers to nrf_drv_gpiote.o(i.nrf_drv_gpiote_out_task_addr_get) for nrf_drv_gpiote_out_task_addr_get
    app_pwm.o(i.pwm_transition_n_to_m) refers to nrf_drv_timer.o(i.nrf_drv_timer_compare) for nrf_drv_timer_compare
    app_pwm.o(i.pwm_transition_n_to_m) refers to nrf_drv_ppi.o(i.nrf_drv_ppi_group_enable) for nrf_drv_ppi_group_enable
    retarget.o(i.fgetc) refers to app_uart_fifo.o(i.app_uart_get) for app_uart_get
    retarget.o(i.fputc) refers to app_uart_fifo.o(i.app_uart_put) for app_uart_put
    softdevice_handler.o(i.SWI2_IRQHandler) refers to app_error.o(i.app_error_handler) for app_error_handler
    softdevice_handler.o(i.SWI2_IRQHandler) refers to softdevice_handler.o(i.intern_softdevice_events_execute) for intern_softdevice_events_execute
    softdevice_handler.o(i.SWI2_IRQHandler) refers to softdevice_handler.o(.data) for .data
    softdevice_handler.o(i.intern_softdevice_events_execute) refers to app_error.o(i.app_error_handler) for app_error_handler
    softdevice_handler.o(i.intern_softdevice_events_execute) refers to softdevice_handler.o(.data) for .data
    softdevice_handler.o(i.softdevice_assertion_handler) refers (Weak) to main.o(i.assert_nrf_callback) for assert_nrf_callback
    softdevice_handler.o(i.softdevice_ble_evt_handler_set) refers to softdevice_handler.o(.data) for .data
    softdevice_handler.o(i.softdevice_handler_init) refers to softdevice_handler.o(.data) for .data
    softdevice_handler.o(i.softdevice_handler_init) refers to softdevice_handler.o(i.softdevice_assertion_handler) for softdevice_assertion_handler
    softdevice_handler.o(i.softdevice_handler_sd_disable) refers to softdevice_handler.o(.data) for .data
    softdevice_handler.o(i.softdevice_sys_evt_handler_set) refers to softdevice_handler.o(.data) for .data
    entry.o(.ARM.Collect$$$$00000000) refers (Special) to entry10a.o(.ARM.Collect$$$$0000000D) for __rt_final_cpp
    entry.o(.ARM.Collect$$$$00000000) refers (Special) to entry11a.o(.ARM.Collect$$$$0000000F) for __rt_final_exit
    entry.o(.ARM.Collect$$$$00000000) refers (Special) to entry7b.o(.ARM.Collect$$$$00000008) for _main_clock
    entry.o(.ARM.Collect$$$$00000000) refers (Special) to entry8b.o(.ARM.Collect$$$$0000000A) for _main_cpp_init
    entry.o(.ARM.Collect$$$$00000000) refers (Special) to entry9a.o(.ARM.Collect$$$$0000000B) for _main_init
    entry.o(.ARM.Collect$$$$00000000) refers (Special) to entry5.o(.ARM.Collect$$$$00000004) for _main_scatterload
    entry.o(.ARM.Collect$$$$00000000) refers (Special) to entry2.o(.ARM.Collect$$$$00000001) for _main_stk
    idiv.o(.text) refers to uidiv.o(.text) for __aeabi_uidivmod
    printfb.o(i.__0fprintf$bare) refers to printfb.o(i._printf_core) for _printf_core
    printfb.o(i.__0fprintf$bare) refers to retarget.o(i.fputc) for fputc
    printfb.o(i.__0printf$bare) refers to printfb.o(i._printf_core) for _printf_core
    printfb.o(i.__0printf$bare) refers to retarget.o(i.fputc) for fputc
    printfb.o(i.__0printf$bare) refers to retarget.o(.data) for __stdout
    printfb.o(i.__0snprintf$bare) refers to printfb.o(i._printf_core) for _printf_core
    printfb.o(i.__0snprintf$bare) refers to printfb.o(i._snputc) for _snputc
    printfb.o(i.__0sprintf$bare) refers to printfb.o(i._printf_core) for _printf_core
    printfb.o(i.__0sprintf$bare) refers to printfb.o(i._sputc) for _sputc
    printfb.o(i.__0vfprintf$bare) refers to printfb.o(i._printf_core) for _printf_core
    printfb.o(i.__0vfprintf$bare) refers to retarget.o(i.fputc) for fputc
    printfb.o(i.__0vprintf$bare) refers to printfb.o(i._printf_core) for _printf_core
    printfb.o(i.__0vprintf$bare) refers to retarget.o(i.fputc) for fputc
    printfb.o(i.__0vprintf$bare) refers to retarget.o(.data) for __stdout
    printfb.o(i.__0vsnprintf$bare) refers to printfb.o(i._printf_core) for _printf_core
    printfb.o(i.__0vsnprintf$bare) refers to printfb.o(i._snputc) for _snputc
    printfb.o(i.__0vsprintf$bare) refers to printfb.o(i._printf_core) for _printf_core
    printfb.o(i.__0vsprintf$bare) refers to printfb.o(i._sputc) for _sputc
    printf0.o(i.__0fprintf$0) refers to printf0.o(i._printf_core) for _printf_core
    printf0.o(i.__0fprintf$0) refers to retarget.o(i.fputc) for fputc
    printf0.o(i.__0printf$0) refers to printf0.o(i._printf_core) for _printf_core
    printf0.o(i.__0printf$0) refers to retarget.o(i.fputc) for fputc
    printf0.o(i.__0printf$0) refers to retarget.o(.data) for __stdout
    printf0.o(i.__0snprintf$0) refers to printf0.o(i._printf_core) for _printf_core
    printf0.o(i.__0snprintf$0) refers to printf0.o(i._snputc) for _snputc
    printf0.o(i.__0sprintf$0) refers to printf0.o(i._printf_core) for _printf_core
    printf0.o(i.__0sprintf$0) refers to printf0.o(i._sputc) for _sputc
    printf0.o(i.__0vfprintf$0) refers to printf0.o(i._printf_core) for _printf_core
    printf0.o(i.__0vfprintf$0) refers to retarget.o(i.fputc) for fputc
    printf0.o(i.__0vprintf$0) refers to printf0.o(i._printf_core) for _printf_core
    printf0.o(i.__0vprintf$0) refers to retarget.o(i.fputc) for fputc
    printf0.o(i.__0vprintf$0) refers to retarget.o(.data) for __stdout
    printf0.o(i.__0vsnprintf$0) refers to printf0.o(i._printf_core) for _printf_core
    printf0.o(i.__0vsnprintf$0) refers to printf0.o(i._snputc) for _snputc
    printf0.o(i.__0vsprintf$0) refers to printf0.o(i._printf_core) for _printf_core
    printf0.o(i.__0vsprintf$0) refers to printf0.o(i._sputc) for _sputc
    printf1.o(i.__0fprintf$1) refers to printf1.o(i._printf_core) for _printf_core
    printf1.o(i.__0fprintf$1) refers to retarget.o(i.fputc) for fputc
    printf1.o(i.__0printf$1) refers to printf1.o(i._printf_core) for _printf_core
    printf1.o(i.__0printf$1) refers to retarget.o(i.fputc) for fputc
    printf1.o(i.__0printf$1) refers to retarget.o(.data) for __stdout
    printf1.o(i.__0snprintf$1) refers to printf1.o(i._printf_core) for _printf_core
    printf1.o(i.__0snprintf$1) refers to printf1.o(i._snputc) for _snputc
    printf1.o(i.__0sprintf$1) refers to printf1.o(i._printf_core) for _printf_core
    printf1.o(i.__0sprintf$1) refers to printf1.o(i._sputc) for _sputc
    printf1.o(i.__0vfprintf$1) refers to printf1.o(i._printf_core) for _printf_core
    printf1.o(i.__0vfprintf$1) refers to retarget.o(i.fputc) for fputc
    printf1.o(i.__0vprintf$1) refers to printf1.o(i._printf_core) for _printf_core
    printf1.o(i.__0vprintf$1) refers to retarget.o(i.fputc) for fputc
    printf1.o(i.__0vprintf$1) refers to retarget.o(.data) for __stdout
    printf1.o(i.__0vsnprintf$1) refers to printf1.o(i._printf_core) for _printf_core
    printf1.o(i.__0vsnprintf$1) refers to printf1.o(i._snputc) for _snputc
    printf1.o(i.__0vsprintf$1) refers to printf1.o(i._printf_core) for _printf_core
    printf1.o(i.__0vsprintf$1) refers to printf1.o(i._sputc) for _sputc
    printf1.o(i._printf_core) refers to uidiv.o(.text) for __aeabi_uidivmod
    printf2.o(i.__0fprintf$2) refers to printf2.o(i._printf_core) for _printf_core
    printf2.o(i.__0fprintf$2) refers to retarget.o(i.fputc) for fputc
    printf2.o(i.__0printf$2) refers to printf2.o(i._printf_core) for _printf_core
    printf2.o(i.__0printf$2) refers to retarget.o(i.fputc) for fputc
    printf2.o(i.__0printf$2) refers to retarget.o(.data) for __stdout
    printf2.o(i.__0snprintf$2) refers to printf2.o(i._printf_core) for _printf_core
    printf2.o(i.__0snprintf$2) refers to printf2.o(i._snputc) for _snputc
    printf2.o(i.__0sprintf$2) refers to printf2.o(i._printf_core) for _printf_core
    printf2.o(i.__0sprintf$2) refers to printf2.o(i._sputc) for _sputc
    printf2.o(i.__0vfprintf$2) refers to printf2.o(i._printf_core) for _printf_core
    printf2.o(i.__0vfprintf$2) refers to retarget.o(i.fputc) for fputc
    printf2.o(i.__0vprintf$2) refers to printf2.o(i._printf_core) for _printf_core
    printf2.o(i.__0vprintf$2) refers to retarget.o(i.fputc) for fputc
    printf2.o(i.__0vprintf$2) refers to retarget.o(.data) for __stdout
    printf2.o(i.__0vsnprintf$2) refers to printf2.o(i._printf_core) for _printf_core
    printf2.o(i.__0vsnprintf$2) refers to printf2.o(i._snputc) for _snputc
    printf2.o(i.__0vsprintf$2) refers to printf2.o(i._printf_core) for _printf_core
    printf2.o(i.__0vsprintf$2) refers to printf2.o(i._sputc) for _sputc
    printf3.o(i.__0fprintf$3) refers to printf3.o(i._printf_core) for _printf_core
    printf3.o(i.__0fprintf$3) refers to retarget.o(i.fputc) for fputc
    printf3.o(i.__0printf$3) refers to printf3.o(i._printf_core) for _printf_core
    printf3.o(i.__0printf$3) refers to retarget.o(i.fputc) for fputc
    printf3.o(i.__0printf$3) refers to retarget.o(.data) for __stdout
    printf3.o(i.__0snprintf$3) refers to printf3.o(i._printf_core) for _printf_core
    printf3.o(i.__0snprintf$3) refers to printf3.o(i._snputc) for _snputc
    printf3.o(i.__0sprintf$3) refers to printf3.o(i._printf_core) for _printf_core
    printf3.o(i.__0sprintf$3) refers to printf3.o(i._sputc) for _sputc
    printf3.o(i.__0vfprintf$3) refers to printf3.o(i._printf_core) for _printf_core
    printf3.o(i.__0vfprintf$3) refers to retarget.o(i.fputc) for fputc
    printf3.o(i.__0vprintf$3) refers to printf3.o(i._printf_core) for _printf_core
    printf3.o(i.__0vprintf$3) refers to retarget.o(i.fputc) for fputc
    printf3.o(i.__0vprintf$3) refers to retarget.o(.data) for __stdout
    printf3.o(i.__0vsnprintf$3) refers to printf3.o(i._printf_core) for _printf_core
    printf3.o(i.__0vsnprintf$3) refers to printf3.o(i._snputc) for _snputc
    printf3.o(i.__0vsprintf$3) refers to printf3.o(i._printf_core) for _printf_core
    printf3.o(i.__0vsprintf$3) refers to printf3.o(i._sputc) for _sputc
    printf3.o(i._printf_core) refers to uidiv.o(.text) for __aeabi_uidivmod
    printf4.o(i.__0fprintf$4) refers to printf4.o(i._printf_core) for _printf_core
    printf4.o(i.__0fprintf$4) refers to retarget.o(i.fputc) for fputc
    printf4.o(i.__0printf$4) refers to printf4.o(i._printf_core) for _printf_core
    printf4.o(i.__0printf$4) refers to retarget.o(i.fputc) for fputc
    printf4.o(i.__0printf$4) refers to retarget.o(.data) for __stdout
    printf4.o(i.__0snprintf$4) refers to printf4.o(i._printf_core) for _printf_core
    printf4.o(i.__0snprintf$4) refers to printf4.o(i._snputc) for _snputc
    printf4.o(i.__0sprintf$4) refers to printf4.o(i._printf_core) for _printf_core
    printf4.o(i.__0sprintf$4) refers to printf4.o(i._sputc) for _sputc
    printf4.o(i.__0vfprintf$4) refers to printf4.o(i._printf_core) for _printf_core
    printf4.o(i.__0vfprintf$4) refers to retarget.o(i.fputc) for fputc
    printf4.o(i.__0vprintf$4) refers to printf4.o(i._printf_core) for _printf_core
    printf4.o(i.__0vprintf$4) refers to retarget.o(i.fputc) for fputc
    printf4.o(i.__0vprintf$4) refers to retarget.o(.data) for __stdout
    printf4.o(i.__0vsnprintf$4) refers to printf4.o(i._printf_core) for _printf_core
    printf4.o(i.__0vsnprintf$4) refers to printf4.o(i._snputc) for _snputc
    printf4.o(i.__0vsprintf$4) refers to printf4.o(i._printf_core) for _printf_core
    printf4.o(i.__0vsprintf$4) refers to printf4.o(i._sputc) for _sputc
    printf4.o(i._printf_core) refers to uldiv.o(.text) for __aeabi_uldivmod
    printf5.o(i.__0fprintf$5) refers to printf5.o(i._printf_core) for _printf_core
    printf5.o(i.__0fprintf$5) refers to retarget.o(i.fputc) for fputc
    printf5.o(i.__0printf$5) refers to printf5.o(i._printf_core) for _printf_core
    printf5.o(i.__0printf$5) refers to retarget.o(i.fputc) for fputc
    printf5.o(i.__0printf$5) refers to retarget.o(.data) for __stdout
    printf5.o(i.__0snprintf$5) refers to printf5.o(i._printf_core) for _printf_core
    printf5.o(i.__0snprintf$5) refers to printf5.o(i._snputc) for _snputc
    printf5.o(i.__0sprintf$5) refers to printf5.o(i._printf_core) for _printf_core
    printf5.o(i.__0sprintf$5) refers to printf5.o(i._sputc) for _sputc
    printf5.o(i.__0vfprintf$5) refers to printf5.o(i._printf_core) for _printf_core
    printf5.o(i.__0vfprintf$5) refers to retarget.o(i.fputc) for fputc
    printf5.o(i.__0vprintf$5) refers to printf5.o(i._printf_core) for _printf_core
    printf5.o(i.__0vprintf$5) refers to retarget.o(i.fputc) for fputc
    printf5.o(i.__0vprintf$5) refers to retarget.o(.data) for __stdout
    printf5.o(i.__0vsnprintf$5) refers to printf5.o(i._printf_core) for _printf_core
    printf5.o(i.__0vsnprintf$5) refers to printf5.o(i._snputc) for _snputc
    printf5.o(i.__0vsprintf$5) refers to printf5.o(i._printf_core) for _printf_core
    printf5.o(i.__0vsprintf$5) refers to printf5.o(i._sputc) for _sputc
    printf5.o(i._printf_core) refers to uldiv.o(.text) for __aeabi_uldivmod
    printf6.o(i.__0fprintf$6) refers to printf6.o(i._printf_core) for _printf_core
    printf6.o(i.__0fprintf$6) refers to retarget.o(i.fputc) for fputc
    printf6.o(i.__0printf$6) refers to printf6.o(i._printf_core) for _printf_core
    printf6.o(i.__0printf$6) refers to retarget.o(i.fputc) for fputc
    printf6.o(i.__0printf$6) refers to retarget.o(.data) for __stdout
    printf6.o(i.__0snprintf$6) refers to printf6.o(i._printf_core) for _printf_core
    printf6.o(i.__0snprintf$6) refers to printf6.o(i._snputc) for _snputc
    printf6.o(i.__0sprintf$6) refers to printf6.o(i._printf_core) for _printf_core
    printf6.o(i.__0sprintf$6) refers to printf6.o(i._sputc) for _sputc
    printf6.o(i.__0vfprintf$6) refers to printf6.o(i._printf_core) for _printf_core
    printf6.o(i.__0vfprintf$6) refers to retarget.o(i.fputc) for fputc
    printf6.o(i.__0vprintf$6) refers to printf6.o(i._printf_core) for _printf_core
    printf6.o(i.__0vprintf$6) refers to retarget.o(i.fputc) for fputc
    printf6.o(i.__0vprintf$6) refers to retarget.o(.data) for __stdout
    printf6.o(i.__0vsnprintf$6) refers to printf6.o(i._printf_core) for _printf_core
    printf6.o(i.__0vsnprintf$6) refers to printf6.o(i._snputc) for _snputc
    printf6.o(i.__0vsprintf$6) refers to printf6.o(i._printf_core) for _printf_core
    printf6.o(i.__0vsprintf$6) refers to printf6.o(i._sputc) for _sputc
    printf6.o(i._printf_core) refers to printf6.o(i._printf_pre_padding) for _printf_pre_padding
    printf6.o(i._printf_core) refers to printf6.o(i._printf_post_padding) for _printf_post_padding
    printf6.o(i._printf_core) refers to uidiv.o(.text) for __aeabi_uidivmod
    printf7.o(i.__0fprintf$7) refers to printf7.o(i._printf_core) for _printf_core
    printf7.o(i.__0fprintf$7) refers to retarget.o(i.fputc) for fputc
    printf7.o(i.__0printf$7) refers to printf7.o(i._printf_core) for _printf_core
    printf7.o(i.__0printf$7) refers to retarget.o(i.fputc) for fputc
    printf7.o(i.__0printf$7) refers to retarget.o(.data) for __stdout
    printf7.o(i.__0snprintf$7) refers to printf7.o(i._printf_core) for _printf_core
    printf7.o(i.__0snprintf$7) refers to printf7.o(i._snputc) for _snputc
    printf7.o(i.__0sprintf$7) refers to printf7.o(i._printf_core) for _printf_core
    printf7.o(i.__0sprintf$7) refers to printf7.o(i._sputc) for _sputc
    printf7.o(i.__0vfprintf$7) refers to printf7.o(i._printf_core) for _printf_core
    printf7.o(i.__0vfprintf$7) refers to retarget.o(i.fputc) for fputc
    printf7.o(i.__0vprintf$7) refers to printf7.o(i._printf_core) for _printf_core
    printf7.o(i.__0vprintf$7) refers to retarget.o(i.fputc) for fputc
    printf7.o(i.__0vprintf$7) refers to retarget.o(.data) for __stdout
    printf7.o(i.__0vsnprintf$7) refers to printf7.o(i._printf_core) for _printf_core
    printf7.o(i.__0vsnprintf$7) refers to printf7.o(i._snputc) for _snputc
    printf7.o(i.__0vsprintf$7) refers to printf7.o(i._printf_core) for _printf_core
    printf7.o(i.__0vsprintf$7) refers to printf7.o(i._sputc) for _sputc
    printf7.o(i._printf_core) refers to printf7.o(i._printf_pre_padding) for _printf_pre_padding
    printf7.o(i._printf_core) refers to printf7.o(i._printf_post_padding) for _printf_post_padding
    printf7.o(i._printf_core) refers to uldiv.o(.text) for __aeabi_uldivmod
    printf8.o(i.__0fprintf$8) refers to printf8.o(i._printf_core) for _printf_core
    printf8.o(i.__0fprintf$8) refers to retarget.o(i.fputc) for fputc
    printf8.o(i.__0printf$8) refers to printf8.o(i._printf_core) for _printf_core
    printf8.o(i.__0printf$8) refers to retarget.o(i.fputc) for fputc
    printf8.o(i.__0printf$8) refers to retarget.o(.data) for __stdout
    printf8.o(i.__0snprintf$8) refers to printf8.o(i._printf_core) for _printf_core
    printf8.o(i.__0snprintf$8) refers to printf8.o(i._snputc) for _snputc
    printf8.o(i.__0sprintf$8) refers to printf8.o(i._printf_core) for _printf_core
    printf8.o(i.__0sprintf$8) refers to printf8.o(i._sputc) for _sputc
    printf8.o(i.__0vfprintf$8) refers to printf8.o(i._printf_core) for _printf_core
    printf8.o(i.__0vfprintf$8) refers to retarget.o(i.fputc) for fputc
    printf8.o(i.__0vprintf$8) refers to printf8.o(i._printf_core) for _printf_core
    printf8.o(i.__0vprintf$8) refers to retarget.o(i.fputc) for fputc
    printf8.o(i.__0vprintf$8) refers to retarget.o(.data) for __stdout
    printf8.o(i.__0vsnprintf$8) refers to printf8.o(i._printf_core) for _printf_core
    printf8.o(i.__0vsnprintf$8) refers to printf8.o(i._snputc) for _snputc
    printf8.o(i.__0vsprintf$8) refers to printf8.o(i._printf_core) for _printf_core
    printf8.o(i.__0vsprintf$8) refers to printf8.o(i._sputc) for _sputc
    printf8.o(i._printf_core) refers to printf8.o(i._printf_pre_padding) for _printf_pre_padding
    printf8.o(i._printf_core) refers to printf8.o(i._printf_post_padding) for _printf_post_padding
    printf8.o(i._printf_core) refers to uldiv.o(.text) for __aeabi_uldivmod
    printfa.o(i.__0fprintf) refers (Special) to iusefp.o(.text) for __I$use$fp
    printfa.o(i.__0fprintf) refers to printfa.o(i._printf_core) for _printf_core
    printfa.o(i.__0fprintf) refers to retarget.o(i.fputc) for fputc
    printfa.o(i.__0printf) refers (Special) to iusefp.o(.text) for __I$use$fp
    printfa.o(i.__0printf) refers to printfa.o(i._printf_core) for _printf_core
    printfa.o(i.__0printf) refers to retarget.o(i.fputc) for fputc
    printfa.o(i.__0printf) refers to retarget.o(.data) for __stdout
    printfa.o(i.__0snprintf) refers (Special) to iusefp.o(.text) for __I$use$fp
    printfa.o(i.__0snprintf) refers to printfa.o(i._printf_core) for _printf_core
    printfa.o(i.__0snprintf) refers to printfa.o(i._snputc) for _snputc
    printfa.o(i.__0sprintf) refers (Special) to iusefp.o(.text) for __I$use$fp
    printfa.o(i.__0sprintf) refers to printfa.o(i._printf_core) for _printf_core
    printfa.o(i.__0sprintf) refers to printfa.o(i._sputc) for _sputc
    printfa.o(i.__0vfprintf) refers (Special) to iusefp.o(.text) for __I$use$fp
    printfa.o(i.__0vfprintf) refers to printfa.o(i._printf_core) for _printf_core
    printfa.o(i.__0vfprintf) refers to retarget.o(i.fputc) for fputc
    printfa.o(i.__0vprintf) refers (Special) to iusefp.o(.text) for __I$use$fp
    printfa.o(i.__0vprintf) refers to printfa.o(i._printf_core) for _printf_core
    printfa.o(i.__0vprintf) refers to retarget.o(i.fputc) for fputc
    printfa.o(i.__0vprintf) refers to retarget.o(.data) for __stdout
    printfa.o(i.__0vsnprintf) refers (Special) to iusefp.o(.text) for __I$use$fp
    printfa.o(i.__0vsnprintf) refers to printfa.o(i._printf_core) for _printf_core
    printfa.o(i.__0vsnprintf) refers to printfa.o(i._snputc) for _snputc
    printfa.o(i.__0vsprintf) refers (Special) to iusefp.o(.text) for __I$use$fp
    printfa.o(i.__0vsprintf) refers to printfa.o(i._printf_core) for _printf_core
    printfa.o(i.__0vsprintf) refers to printfa.o(i._sputc) for _sputc
    printfa.o(i._fp_digits) refers (Special) to iusefp.o(.text) for __I$use$fp
    printfa.o(i._fp_digits) refers to dmul.o(.text) for __aeabi_dmul
    printfa.o(i._fp_digits) refers to ddiv.o(.text) for __aeabi_ddiv
    printfa.o(i._fp_digits) refers to cdrcmple.o(.text) for __aeabi_cdrcmple
    printfa.o(i._fp_digits) refers to dadd.o(.text) for __aeabi_dadd
    printfa.o(i._fp_digits) refers to dfixul.o(.text) for __aeabi_d2ulz
    printfa.o(i._fp_digits) refers to uldiv.o(.text) for __aeabi_uldivmod
    printfa.o(i._printf_core) refers (Special) to iusefp.o(.text) for __I$use$fp
    printfa.o(i._printf_core) refers to printfa.o(i._printf_pre_padding) for _printf_pre_padding
    printfa.o(i._printf_core) refers to uldiv.o(.text) for __aeabi_uldivmod
    printfa.o(i._printf_core) refers to printfa.o(i._printf_post_padding) for _printf_post_padding
    printfa.o(i._printf_core) refers to printfa.o(i._fp_digits) for _fp_digits
    printfa.o(i._printf_core) refers to uidiv.o(.text) for __aeabi_uidivmod
    printfa.o(i._printf_post_padding) refers (Special) to iusefp.o(.text) for __I$use$fp
    printfa.o(i._printf_pre_padding) refers (Special) to iusefp.o(.text) for __I$use$fp
    printfa.o(i._snputc) refers (Special) to iusefp.o(.text) for __I$use$fp
    printfa.o(i._sputc) refers (Special) to iusefp.o(.text) for __I$use$fp
    entry2.o(.ARM.Collect$$$$00000001) refers to entry2.o(.ARM.Collect$$$$00002712) for __lit__00000000
    entry2.o(.ARM.Collect$$$$00002712) refers to arm_startup_nrf51.o(STACK) for __initial_sp
    entry2.o(__vectab_stack_and_reset_area) refers to arm_startup_nrf51.o(STACK) for __initial_sp
    entry2.o(__vectab_stack_and_reset_area) refers to entry.o(.ARM.Collect$$$$00000000) for __main
    entry5.o(.ARM.Collect$$$$00000004) refers to init.o(.text) for __scatterload
    entry9a.o(.ARM.Collect$$$$0000000B) refers to main.o(i.main) for main
    entry9b.o(.ARM.Collect$$$$0000000C) refers to main.o(i.main) for main
    uldiv.o(.text) refers to llushr.o(.text) for __aeabi_llsr
    uldiv.o(.text) refers to llshl.o(.text) for __aeabi_llsl
    dadd.o(.text) refers to llshl.o(.text) for __aeabi_llsl
    dadd.o(.text) refers to llsshr.o(.text) for __aeabi_lasr
    dadd.o(.text) refers to depilogue.o(.text) for _double_epilogue
    dmul.o(.text) refers to depilogue.o(.text) for _double_epilogue
    ddiv.o(.text) refers to depilogue.o(.text) for _double_round
    dfixul.o(.text) refers to llushr.o(.text) for __aeabi_llsr
    dfixul.o(.text) refers to llshl.o(.text) for __aeabi_llsl
    init.o(.text) refers to entry5.o(.ARM.Collect$$$$00000004) for __main_after_scatterload
    depilogue.o(.text) refers to depilogue.o(i.__ARM_clz) for __ARM_clz
    depilogue.o(.text) refers to llshl.o(.text) for __aeabi_llsl
    depilogue.o(.text) refers to llushr.o(.text) for __aeabi_llsr
    spi_master.o(i.spi_master_get_state) refers to spi_master.o(i.spi_master_get_instance) for spi_master_get_instance
    spi_master.o(i.spi_master_get_state) refers to app_error.o(i.app_error_handler) for app_error_handler
    spi_master.o(i.spi_master_evt_handler_reg) refers to spi_master.o(i.spi_master_get_instance) for spi_master_get_instance
    spi_master.o(i.spi_master_evt_handler_reg) refers to app_error.o(i.app_error_handler) for app_error_handler


==============================================================================

Removing Unused input sections from the image.

    Removing client_handling.o(.rev16_text), (4 bytes).
    Removing client_handling.o(.revsh_text), (4 bytes).
    Removing client_handling.o(.emb_text), (30 bytes).
    Removing client_handling.o(i.client_handling_count), (12 bytes).
    Removing client_handling.o(i.print_client_data), (56 bytes).
    Removing client_handling.o(.conststring), (73 bytes).
    Removing main.o(.rev16_text), (4 bytes).
    Removing main.o(.revsh_text), (4 bytes).
    Removing main.o(.emb_text), (30 bytes).
    Removing main.o(i.assert_nrf_callback), (20 bytes).
    Removing acc_lis2.o(.rev16_text), (4 bytes).
    Removing acc_lis2.o(.revsh_text), (4 bytes).
    Removing acc_lis2.o(.emb_text), (30 bytes).
    Removing acc_lis2.o(i.acc_get_fifo_src), (12 bytes).
    Removing acc_lis2.o(i.acc_get_fifo_wtm), (12 bytes).
    Removing acc_lis2.o(i.acc_get_int1_cfg), (12 bytes).
    Removing acc_lis2.o(i.acc_get_int1_src), (12 bytes).
    Removing acc_lis2.o(i.acc_get_status), (12 bytes).
    Removing acc_lis2.o(i.acc_get_who_am_i), (12 bytes).
    Removing acc_lis2.o(i.acc_get_x), (12 bytes).
    Removing acc_lis2.o(i.acc_get_x8), (12 bytes).
    Removing acc_lis2.o(i.acc_get_xy), (52 bytes).
    Removing acc_lis2.o(i.acc_get_xyz), (188 bytes).
    Removing acc_lis2.o(i.acc_get_xyz8), (40 bytes).
    Removing acc_lis2.o(i.acc_get_xyzreg), (14 bytes).
    Removing acc_lis2.o(i.acc_get_y8), (12 bytes).
    Removing acc_lis2.o(i.acc_get_z8), (12 bytes).
    Removing acc_lis2.o(i.acc_init), (116 bytes).
    Removing acc_lis2.o(i.acc_init_w_int), (72 bytes).
    Removing acc_lis2.o(i.acc_reset_fifo), (20 bytes).
    Removing acc_lis2.o(i.acc_set_100Hz_lp_mode), (8 bytes).
    Removing acc_lis2.o(i.acc_set_100Hz_lp_mode_xy), (12 bytes).
    Removing acc_lis2.o(i.acc_set_100Hz_lp_mode_xz), (12 bytes).
    Removing acc_lis2.o(i.acc_set_100Hz_lp_mode_yz), (12 bytes).
    Removing acc_lis2.o(i.acc_set_400Hz_lp_mode), (12 bytes).
    Removing acc_lis2.o(i.acc_set_400Hz_lp_mode_xy), (12 bytes).
    Removing acc_lis2.o(i.acc_set_400Hz_lp_mode_xz), (12 bytes).
    Removing acc_lis2.o(i.acc_set_400Hz_lp_mode_yz), (12 bytes).
    Removing acc_lis2.o(i.acc_start_xyz), (60 bytes).
    Removing acc_lis2.o(i.send_recv_spi0_data), (36 bytes).
    Removing acc_lis2.o(i.spi_master_event_handler), (20 bytes).
    Removing acc_lis2.o(i.spia_init), (104 bytes).
    Removing acc_lis2.o(i.spia_rd16), (64 bytes).
    Removing acc_lis2.o(i.spia_rd8), (52 bytes).
    Removing acc_lis2.o(i.spia_wr8), (36 bytes).
    Removing acc_lis2.o(.bss), (26 bytes).
    Removing acc_lis2.o(.constdata), (28 bytes).
    Removing acc_lis2.o(.data), (9 bytes).
    Removing simple_uart.o(.rev16_text), (4 bytes).
    Removing simple_uart.o(.revsh_text), (4 bytes).
    Removing simple_uart.o(.emb_text), (30 bytes).
    Removing simple_uart.o(i.simple_uart_get), (28 bytes).
    Removing simple_uart.o(i.simple_uart_get_with_timeout), (64 bytes).
    Removing spi_master.o(.rev16_text), (4 bytes).
    Removing spi_master.o(.revsh_text), (4 bytes).
    Removing spi_master.o(i.spi_master_buffer_init), (72 bytes).
    Removing spi_master.o(i.spi_master_close), (132 bytes).
    Removing spi_master.o(i.spi_master_init_hw_instance), (58 bytes).
    Removing spi_master.o(i.spi_master_open), (268 bytes).
    Removing spi_master.o(i.spi_master_send_recv), (292 bytes).
    Removing firfilter.o(i.fir_bp_filter), (32 bytes).
    Removing firfilter.o(i.fir_clear), (20 bytes).
    Removing firfilter.o(i.fir_delay), (40 bytes).
    Removing firfilter.o(i.fir_delay_1), (40 bytes).
    Removing firfilter.o(i.fir_delay_2), (40 bytes).
    Removing firfilter.o(i.fir_filter_tq), (32 bytes).
    Removing firfilter.o(i.fir_lp_filter), (32 bytes).
    Removing firfilter.o(i.fir_split), (116 bytes).
    Removing firfilter.o(i.fir_split32), (74 bytes).
    Removing firfilter.o(.bss), (296 bytes).
    Removing firfilter.o(.constdata), (218 bytes).
    Removing firfilter.o(.data), (24 bytes).
    Removing arm_startup_nrf51.o(HEAP), (0 bytes).
    Removing system_nrf51.o(.rev16_text), (4 bytes).
    Removing system_nrf51.o(.revsh_text), (4 bytes).
    Removing system_nrf51.o(i.SystemCoreClockUpdate), (16 bytes).
    Removing ble_advdata.o(i.adv_data_encode), (330 bytes).
    Removing ble_advdata.o(i.ble_advdata_set), (90 bytes).
    Removing ble_advdata.o(i.conn_int_encode), (132 bytes).
    Removing ble_advdata.o(i.manuf_specific_data_encode), (100 bytes).
    Removing ble_advdata.o(i.name_encode), (106 bytes).
    Removing ble_advdata.o(i.service_data_encode), (124 bytes).
    Removing ble_advdata.o(i.uint16_encode), (10 bytes).
    Removing ble_advdata.o(i.uuid_list_encode), (38 bytes).
    Removing ble_advdata.o(i.uuid_list_sized_encode), (162 bytes).
    Removing ble_db_discovery.o(i.ble_db_discovery_close), (20 bytes).
    Removing ble_srv_common.o(i.ble_srv_ascii_to_utf8), (18 bytes).
    Removing ble_srv_common.o(i.ble_srv_report_ref_encode), (12 bytes).
    Removing ble_srv_common.o(i.characteristic_add), (264 bytes).
    Removing ble_srv_common.o(i.set_security_req), (52 bytes).
    Removing device_manager_central.o(.rev16_text), (4 bytes).
    Removing device_manager_central.o(.revsh_text), (4 bytes).
    Removing device_manager_central.o(i.device_instance_free), (44 bytes).
    Removing device_manager_central.o(i.dm_application_context_delete), (8 bytes).
    Removing device_manager_central.o(i.dm_application_context_get), (8 bytes).
    Removing device_manager_central.o(i.dm_application_context_set), (8 bytes).
    Removing device_manager_central.o(i.dm_application_instance_set), (64 bytes).
    Removing device_manager_central.o(i.dm_device_add), (8 bytes).
    Removing device_manager_central.o(i.dm_device_delete), (92 bytes).
    Removing device_manager_central.o(i.dm_device_delete_all), (92 bytes).
    Removing device_manager_central.o(i.dm_distributed_keys_get), (172 bytes).
    Removing device_manager_central.o(i.dm_peer_addr_get), (128 bytes).
    Removing device_manager_central.o(i.dm_peer_addr_set), (136 bytes).
    Removing device_manager_central.o(i.dm_security_status_req), (116 bytes).
    Removing device_manager_central.o(i.dm_service_context_delete), (88 bytes).
    Removing device_manager_central.o(i.dm_service_context_get), (180 bytes).
    Removing device_manager_central.o(i.dm_service_context_set), (180 bytes).
    Removing device_manager_central.o(i.dm_whitelist_create), (188 bytes).
    Removing device_manager_central.o(.constdata), (4 bytes).
    Removing app_uart_fifo.o(.rev16_text), (4 bytes).
    Removing app_uart_fifo.o(.revsh_text), (4 bytes).
    Removing app_uart_fifo.o(i.app_uart_close), (36 bytes).
    Removing app_uart_fifo.o(i.app_uart_flush), (28 bytes).
    Removing app_uart_fifo.o(i.app_uart_get), (16 bytes).
    Removing app_uart_fifo.o(i.app_uart_get_connection_state), (20 bytes).
    Removing app_uart_fifo.o(i.app_uart_init), (404 bytes).
    Removing app_uart_fifo.o(i.app_uart_put), (28 bytes).
    Removing app_uart_fifo.o(i.gpiote_uart_event_handler), (22 bytes).
    Removing app_uart_fifo.o(.constdata), (8 bytes).
    Removing pstorage.o(.rev16_text), (4 bytes).
    Removing pstorage.o(.revsh_text), (4 bytes).
    Removing nrf_drv_common.o(.rev16_text), (4 bytes).
    Removing nrf_drv_common.o(.revsh_text), (4 bytes).
    Removing nrf_drv_gpiote.o(.rev16_text), (4 bytes).
    Removing nrf_drv_gpiote.o(.revsh_text), (4 bytes).
    Removing nrf_drv_gpiote.o(i.nrf_drv_gpiote_in_event_addr_get), (24 bytes).
    Removing nrf_drv_gpiote.o(i.nrf_drv_gpiote_in_event_disable), (84 bytes).
    Removing nrf_drv_gpiote.o(i.nrf_drv_gpiote_in_event_enable), (160 bytes).
    Removing nrf_drv_gpiote.o(i.nrf_drv_gpiote_in_init), (148 bytes).
    Removing nrf_drv_gpiote.o(i.nrf_drv_gpiote_in_is_set), (20 bytes).
    Removing nrf_drv_gpiote.o(i.nrf_drv_gpiote_in_uninit), (80 bytes).
    Removing nrf_drv_gpiote.o(i.nrf_drv_gpiote_out_clear), (16 bytes).
    Removing nrf_drv_gpiote.o(i.nrf_drv_gpiote_out_set), (16 bytes).
    Removing nrf_drv_gpiote.o(i.nrf_drv_gpiote_out_task_disable), (32 bytes).
    Removing nrf_drv_gpiote.o(i.nrf_drv_gpiote_out_toggle), (28 bytes).
    Removing nrf_drv_gpiote.o(i.nrf_drv_gpiote_uninit), (56 bytes).
    Removing nrf_drv_gpiote.o(i.pin_in_use_by_port), (24 bytes).
    Removing nrf_delay.o(.rev16_text), (4 bytes).
    Removing nrf_delay.o(.revsh_text), (4 bytes).
    Removing nrf_drv_ppi.o(.rev16_text), (4 bytes).
    Removing nrf_drv_ppi.o(.revsh_text), (4 bytes).
    Removing nrf_drv_ppi.o(i.nrf_drv_ppi_group_disable), (36 bytes).
    Removing nrf_drv_ppi.o(i.nrf_drv_ppi_uninit), (88 bytes).
    Removing nrf_drv_timer.o(.rev16_text), (4 bytes).
    Removing nrf_drv_timer.o(.revsh_text), (4 bytes).
    Removing nrf_drv_timer.o(i.nrf_drv_timer_capture), (28 bytes).
    Removing nrf_drv_timer.o(i.nrf_drv_timer_capture_get), (14 bytes).
    Removing nrf_drv_timer.o(i.nrf_drv_timer_capture_task_address_get), (12 bytes).
    Removing nrf_drv_timer.o(i.nrf_drv_timer_event_address_get), (6 bytes).
    Removing nrf_drv_timer.o(i.nrf_drv_timer_increment), (8 bytes).
    Removing nrf_drv_timer.o(i.nrf_drv_timer_ms_to_ticks), (22 bytes).
    Removing nrf_drv_timer.o(i.nrf_drv_timer_pause), (8 bytes).
    Removing nrf_drv_timer.o(i.nrf_drv_timer_resume), (8 bytes).
    Removing nrf_drv_timer.o(i.nrf_drv_timer_task_address_get), (6 bytes).
    Removing app_error.o(.rev16_text), (4 bytes).
    Removing app_error.o(.revsh_text), (4 bytes).
    Removing app_fifo.o(i.app_fifo_flush), (8 bytes).
    Removing app_fifo.o(i.app_fifo_init), (36 bytes).
    Removing app_pwm.o(.rev16_text), (4 bytes).
    Removing app_pwm.o(.revsh_text), (4 bytes).
    Removing app_pwm.o(i.app_pwm_channel_duty_get), (30 bytes).
    Removing app_pwm.o(i.app_pwm_channel_duty_ticks_get), (14 bytes).
    Removing app_pwm.o(i.app_pwm_cycle_ticks_get), (8 bytes).
    Removing app_pwm.o(i.app_pwm_disable), (28 bytes).
    Removing app_pwm.o(i.app_pwm_uninit), (52 bytes).
    Removing retarget.o(.rev16_text), (4 bytes).
    Removing retarget.o(.revsh_text), (4 bytes).
    Removing retarget.o(i.fgetc), (18 bytes).
    Removing retarget.o(i.fputc), (14 bytes).
    Removing retarget.o(.data), (4 bytes).
    Removing retarget.o(.data), (4 bytes).
    Removing softdevice_handler.o(.rev16_text), (4 bytes).
    Removing softdevice_handler.o(.revsh_text), (4 bytes).
    Removing softdevice_handler.o(i.softdevice_handler_sd_disable), (24 bytes).
    Removing spi_master.o(i.spi_master_get_state), (26 bytes).
    Removing spi_master.o(i.spi_master_evt_handler_reg), (26 bytes).

176 unused section(s) (total 8220 bytes) removed from the image.

==============================================================================

Image Symbol Table

    Local Symbols

    Symbol Name                              Value     Ov Type        Size  Object(Section)

    ../clib/microlib/division.c              0x00000000   Number         0  uldiv.o ABSOLUTE
    ../clib/microlib/division.c              0x00000000   Number         0  idiv.o ABSOLUTE
    ../clib/microlib/division.c              0x00000000   Number         0  uidiv.o ABSOLUTE
    ../clib/microlib/init/entry.s            0x00000000   Number         0  entry11a.o ABSOLUTE
    ../clib/microlib/init/entry.s            0x00000000   Number         0  entry9b.o ABSOLUTE
    ../clib/microlib/init/entry.s            0x00000000   Number         0  entry11b.o ABSOLUTE
    ../clib/microlib/init/entry.s            0x00000000   Number         0  entry8a.o ABSOLUTE
    ../clib/microlib/init/entry.s            0x00000000   Number         0  entry7b.o ABSOLUTE
    ../clib/microlib/init/entry.s            0x00000000   Number         0  entry2.o ABSOLUTE
    ../clib/microlib/init/entry.s            0x00000000   Number         0  entry5.o ABSOLUTE
    ../clib/microlib/init/entry.s            0x00000000   Number         0  entry.o ABSOLUTE
    ../clib/microlib/init/entry.s            0x00000000   Number         0  entry7a.o ABSOLUTE
    ../clib/microlib/init/entry.s            0x00000000   Number         0  entry10b.o ABSOLUTE
    ../clib/microlib/init/entry.s            0x00000000   Number         0  entry8b.o ABSOLUTE
    ../clib/microlib/init/entry.s            0x00000000   Number         0  entry10a.o ABSOLUTE
    ../clib/microlib/init/entry.s            0x00000000   Number         0  entry9a.o ABSOLUTE
    ../clib/microlib/longlong.c              0x00000000   Number         0  llushr.o ABSOLUTE
    ../clib/microlib/longlong.c              0x00000000   Number         0  llshl.o ABSOLUTE
    ../clib/microlib/longlong.c              0x00000000   Number         0  llsshr.o ABSOLUTE
    ../clib/microlib/printf/printf.c         0x00000000   Number         0  printf0.o ABSOLUTE
    ../clib/microlib/printf/printf.c         0x00000000   Number         0  printf2.o ABSOLUTE
    ../clib/microlib/printf/printf.c         0x00000000   Number         0  printf6.o ABSOLUTE
    ../clib/microlib/printf/printf.c         0x00000000   Number         0  printf4.o ABSOLUTE
    ../clib/microlib/printf/printf.c         0x00000000   Number         0  printf1.o ABSOLUTE
    ../clib/microlib/printf/printf.c         0x00000000   Number         0  printf5.o ABSOLUTE
    ../clib/microlib/printf/printf.c         0x00000000   Number         0  printfa.o ABSOLUTE
    ../clib/microlib/printf/printf.c         0x00000000   Number         0  printf8.o ABSOLUTE
    ../clib/microlib/printf/printf.c         0x00000000   Number         0  printf7.o ABSOLUTE
    ../clib/microlib/printf/printf.c         0x00000000   Number         0  printf3.o ABSOLUTE
    ../clib/microlib/printf/printf.c         0x00000000   Number         0  printfb.o ABSOLUTE
    ../clib/microlib/printf/stubs.s          0x00000000   Number         0  stubs.o ABSOLUTE
    ../clib/microlib/string/memcmp.c         0x00000000   Number         0  memcmp.o ABSOLUTE
    ../clib/microlib/string/memcpy.c         0x00000000   Number         0  memcpyb.o ABSOLUTE
    ../clib/microlib/string/memcpy.c         0x00000000   Number         0  memcpya.o ABSOLUTE
    ../clib/microlib/string/memset.c         0x00000000   Number         0  memseta.o ABSOLUTE
    ../clib/microlib/string/strlen.c         0x00000000   Number         0  strlen.o ABSOLUTE
    ../clib/microlib/stubs.s                 0x00000000   Number         0  iusefp.o ABSOLUTE
    ../fplib/microlib/fpadd.c                0x00000000   Number         0  dadd.o ABSOLUTE
    ../fplib/microlib/fpdiv.c                0x00000000   Number         0  ddiv.o ABSOLUTE
    ../fplib/microlib/fpepilogue.c           0x00000000   Number         0  depilogue.o ABSOLUTE
    ../fplib/microlib/fpfix.c                0x00000000   Number         0  dfixul.o ABSOLUTE
    ../fplib/microlib/fpmul.c                0x00000000   Number         0  dmul.o ABSOLUTE
    ..\..\..\client_handling.c               0x00000000   Number         0  client_handling.o ABSOLUTE
    ..\..\..\main.c                          0x00000000   Number         0  main.o ABSOLUTE
    ..\\..\\..\\client_handling.c            0x00000000   Number         0  client_handling.o ABSOLUTE
    ..\\..\\..\\main.c                       0x00000000   Number         0  main.o ABSOLUTE
    C:\Keil_v5\ARM\PACK\NordicSemiconductor\nRF_BLE\3.0.1\common\ble_srv_common.c 0x00000000   Number         0  ble_srv_common.o ABSOLUTE
    C:\Keil_v5\ARM\PACK\NordicSemiconductor\nRF_BLE\3.0.1\device_manager\device_manager_central.c 0x00000000   Number         0  device_manager_central.o ABSOLUTE
    C:\Keil_v5\ARM\PACK\NordicSemiconductor\nRF_Drivers\3.0.1\common\nrf_drv_common.c 0x00000000   Number         0  nrf_drv_common.o ABSOLUTE
    C:\Keil_v5\ARM\PACK\NordicSemiconductor\nRF_Drivers\3.0.1\gpiote\nrf_drv_gpiote.c 0x00000000   Number         0  nrf_drv_gpiote.o ABSOLUTE
    C:\Keil_v5\ARM\PACK\NordicSemiconductor\nRF_Drivers\3.0.1\hal\nrf_delay.c 0x00000000   Number         0  nrf_delay.o ABSOLUTE
    C:\Keil_v5\ARM\PACK\NordicSemiconductor\nRF_Drivers\3.0.1\ppi\nrf_drv_ppi.c 0x00000000   Number         0  nrf_drv_ppi.o ABSOLUTE
    C:\Keil_v5\ARM\PACK\NordicSemiconductor\nRF_Drivers\3.0.1\timer\nrf_drv_timer.c 0x00000000   Number         0  nrf_drv_timer.o ABSOLUTE
    C:\\Keil_v5\\ARM\\PACK\\NordicSemiconductor\\nRF_BLE\\3.0.1\\device_manager\\device_manager_central.c 0x00000000   Number         0  device_manager_central.o ABSOLUTE
    C:\\Keil_v5\\ARM\\PACK\\NordicSemiconductor\\nRF_Drivers\\3.0.1\\common\\nrf_drv_common.c 0x00000000   Number         0  nrf_drv_common.o ABSOLUTE
    C:\\Keil_v5\\ARM\\PACK\\NordicSemiconductor\\nRF_Drivers\\3.0.1\\gpiote\\nrf_drv_gpiote.c 0x00000000   Number         0  nrf_drv_gpiote.o ABSOLUTE
    C:\\Keil_v5\\ARM\\PACK\\NordicSemiconductor\\nRF_Drivers\\3.0.1\\hal\\nrf_delay.c 0x00000000   Number         0  nrf_delay.o ABSOLUTE
    C:\\Keil_v5\\ARM\\PACK\\NordicSemiconductor\\nRF_Drivers\\3.0.1\\ppi\\nrf_drv_ppi.c 0x00000000   Number         0  nrf_drv_ppi.o ABSOLUTE
    C:\\Keil_v5\\ARM\\PACK\\NordicSemiconductor\\nRF_Drivers\\3.0.1\\timer\\nrf_drv_timer.c 0x00000000   Number         0  nrf_drv_timer.o ABSOLUTE
    RTE\Accelerometer\acc_lis2.c             0x00000000   Number         0  acc_lis2.o ABSOLUTE
    RTE\Device\nRF51422_xxAC\arm_startup_nrf51.s 0x00000000   Number         0  arm_startup_nrf51.o ABSOLUTE
    RTE\Device\nRF51422_xxAC\system_nrf51.c  0x00000000   Number         0  system_nrf51.o ABSOLUTE
    RTE\\Accelerometer\\acc_lis2.c           0x00000000   Number         0  acc_lis2.o ABSOLUTE
    RTE\\Device\\nRF51422_xxAC\\system_nrf51.c 0x00000000   Number         0  system_nrf51.o ABSOLUTE
    RTE\\nRF_Drivers\\nRF51422_xxAC\\app_uart_fifo.c 0x00000000   Number         0  app_uart_fifo.o ABSOLUTE
    RTE\\nRF_Drivers\\nRF51422_xxAC\\pstorage.c 0x00000000   Number         0  pstorage.o ABSOLUTE
    RTE\\nRF_Libraries\\nRF51422_xxAC\\app_error.c 0x00000000   Number         0  app_error.o ABSOLUTE
    RTE\\nRF_Libraries\\nRF51422_xxAC\\app_pwm.c 0x00000000   Number         0  app_pwm.o ABSOLUTE
    RTE\\nRF_Libraries\\nRF51422_xxAC\\retarget.c 0x00000000   Number         0  retarget.o ABSOLUTE
    RTE\\nRF_Libraries\\nRF51422_xxAC\\simple_uart.c 0x00000000   Number         0  simple_uart.o ABSOLUTE
    RTE\\nRF_Libraries\\nRF51422_xxAC\\spi_master.c 0x00000000   Number         0  spi_master.o ABSOLUTE
    RTE\\nRF_SoftDevice\\nRF51422_xxAC\\softdevice_handler.c 0x00000000   Number         0  softdevice_handler.o ABSOLUTE
    RTE\nRF_BLE\nRF51422_xxAC\ble_advdata.c  0x00000000   Number         0  ble_advdata.o ABSOLUTE
    RTE\nRF_BLE\nRF51422_xxAC\ble_db_discovery.c 0x00000000   Number         0  ble_db_discovery.o ABSOLUTE
    RTE\nRF_Drivers\nRF51422_xxAC\app_uart_fifo.c 0x00000000   Number         0  app_uart_fifo.o ABSOLUTE
    RTE\nRF_Drivers\nRF51422_xxAC\pstorage.c 0x00000000   Number         0  pstorage.o ABSOLUTE
    RTE\nRF_Libraries\nRF51422_xxAC\app_error.c 0x00000000   Number         0  app_error.o ABSOLUTE
    RTE\nRF_Libraries\nRF51422_xxAC\app_fifo.c 0x00000000   Number         0  app_fifo.o ABSOLUTE
    RTE\nRF_Libraries\nRF51422_xxAC\app_pwm.c 0x00000000   Number         0  app_pwm.o ABSOLUTE
    RTE\nRF_Libraries\nRF51422_xxAC\app_trace.c 0x00000000   Number         0  app_trace.o ABSOLUTE
    RTE\nRF_Libraries\nRF51422_xxAC\debug_util.c 0x00000000   Number         0  debug_util.o ABSOLUTE
    RTE\nRF_Libraries\nRF51422_xxAC\firfilter.c 0x00000000   Number         0  firfilter.o ABSOLUTE
    RTE\nRF_Libraries\nRF51422_xxAC\nrf_assert.c 0x00000000   Number         0  nrf_assert.o ABSOLUTE
    RTE\nRF_Libraries\nRF51422_xxAC\retarget.c 0x00000000   Number         0  retarget.o ABSOLUTE
    RTE\nRF_Libraries\nRF51422_xxAC\simple_uart.c 0x00000000   Number         0  simple_uart.o ABSOLUTE
    RTE\nRF_Libraries\nRF51422_xxAC\spi_master.c 0x00000000   Number         0  spi_master.o ABSOLUTE
    RTE\nRF_SoftDevice\nRF51422_xxAC\softdevice_handler.c 0x00000000   Number         0  softdevice_handler.o ABSOLUTE
    cdrcmple.s                               0x00000000   Number         0  cdrcmple.o ABSOLUTE
    dc.s                                     0x00000000   Number         0  dc.o ABSOLUTE
    handlers.s                               0x00000000   Number         0  handlers.o ABSOLUTE
    init.s                                   0x00000000   Number         0  init.o ABSOLUTE
    RESET                                    0x0001d000   Section      192  arm_startup_nrf51.o(RESET)
    .ARM.Collect$$$$00000000                 0x0001d0c0   Section        0  entry.o(.ARM.Collect$$$$00000000)
    .ARM.Collect$$$$00000001                 0x0001d0c0   Section        4  entry2.o(.ARM.Collect$$$$00000001)
    .ARM.Collect$$$$00000004                 0x0001d0c4   Section        4  entry5.o(.ARM.Collect$$$$00000004)
    .ARM.Collect$$$$00000008                 0x0001d0c8   Section        0  entry7b.o(.ARM.Collect$$$$00000008)
    .ARM.Collect$$$$0000000A                 0x0001d0c8   Section        0  entry8b.o(.ARM.Collect$$$$0000000A)
    .ARM.Collect$$$$0000000B                 0x0001d0c8   Section        8  entry9a.o(.ARM.Collect$$$$0000000B)
    .ARM.Collect$$$$0000000D                 0x0001d0d0   Section        0  entry10a.o(.ARM.Collect$$$$0000000D)
    .ARM.Collect$$$$0000000F                 0x0001d0d0   Section        0  entry11a.o(.ARM.Collect$$$$0000000F)
    .ARM.Collect$$$$00002712                 0x0001d0d0   Section        4  entry2.o(.ARM.Collect$$$$00002712)
    __lit__00000000                          0x0001d0d0   Data           4  entry2.o(.ARM.Collect$$$$00002712)
    .emb_text                                0x0001d0d4   Section       30  nrf_delay.o(.emb_text)
    .text                                    0x0001d0f4   Section       56  arm_startup_nrf51.o(.text)
    .text                                    0x0001d12c   Section        0  uidiv.o(.text)
    .text                                    0x0001d158   Section        0  idiv.o(.text)
    .text                                    0x0001d180   Section        0  memcpya.o(.text)
    .text                                    0x0001d1a4   Section        0  memseta.o(.text)
    .text                                    0x0001d1c8   Section        0  memcmp.o(.text)
    .text                                    0x0001d1e2   Section        0  uldiv.o(.text)
    .text                                    0x0001d242   Section        0  iusefp.o(.text)
    .text                                    0x0001d244   Section        0  dadd.o(.text)
    .text                                    0x0001d3a8   Section        0  dmul.o(.text)
    .text                                    0x0001d478   Section        0  ddiv.o(.text)
    .text                                    0x0001d568   Section        0  dfixul.o(.text)
    .text                                    0x0001d5a8   Section       40  cdrcmple.o(.text)
    .text                                    0x0001d5d0   Section       36  init.o(.text)
    .text                                    0x0001d5f4   Section        0  llshl.o(.text)
    .text                                    0x0001d614   Section        0  llushr.o(.text)
    .text                                    0x0001d636   Section        0  llsshr.o(.text)
    .text                                    0x0001d65c   Section        0  depilogue.o(.text)
    i.GPIOTE_IRQHandler                      0x0001d71c   Section        0  nrf_drv_gpiote.o(i.GPIOTE_IRQHandler)
    i.SPI0_TWI0_IRQHandler                   0x0001d818   Section        0  spi_master.o(i.SPI0_TWI0_IRQHandler)
    i.SWI2_IRQHandler                        0x0001d844   Section        0  softdevice_handler.o(i.SWI2_IRQHandler)
    i.SystemInit                             0x0001d868   Section        0  system_nrf51.o(i.SystemInit)
    i.TIMER1_IRQHandler                      0x0001d8bc   Section        0  nrf_drv_timer.o(i.TIMER1_IRQHandler)
    i.UART0_IRQHandler                       0x0001d908   Section        0  app_uart_fifo.o(i.UART0_IRQHandler)
    i.__0sprintf                             0x0001d988   Section        0  printfa.o(i.__0sprintf)
    i.__0vsprintf                            0x0001d9b0   Section        0  printfa.o(i.__0vsprintf)
    i.__ARM_clz                              0x0001d9d4   Section        0  depilogue.o(i.__ARM_clz)
    i.__ARM_common_switch8                   0x0001da02   Section        0  client_handling.o(i.__ARM_common_switch8)
    i.__scatterload_copy                     0x0001da1c   Section       14  handlers.o(i.__scatterload_copy)
    i.__scatterload_null                     0x0001da2a   Section        2  handlers.o(i.__scatterload_null)
    i.__scatterload_zeroinit                 0x0001da2c   Section       14  handlers.o(i.__scatterload_zeroinit)
    i._fp_digits                             0x0001da3c   Section        0  printfa.o(i._fp_digits)
    _fp_digits                               0x0001da3d   Thumb Code   316  printfa.o(i._fp_digits)
    i._printf_core                           0x0001db94   Section        0  printfa.o(i._printf_core)
    _printf_core                             0x0001db95   Thumb Code  1754  printfa.o(i._printf_core)
    i._printf_post_padding                   0x0001e280   Section        0  printfa.o(i._printf_post_padding)
    _printf_post_padding                     0x0001e281   Thumb Code    32  printfa.o(i._printf_post_padding)
    i._printf_pre_padding                    0x0001e2a0   Section        0  printfa.o(i._printf_pre_padding)
    _printf_pre_padding                      0x0001e2a1   Thumb Code    44  printfa.o(i._printf_pre_padding)
    i._sputc                                 0x0001e2cc   Section        0  printfa.o(i._sputc)
    _sputc                                   0x0001e2cd   Thumb Code    10  printfa.o(i._sputc)
    i.action_tx_send                         0x0001e2d8   Section        0  app_uart_fifo.o(i.action_tx_send)
    action_tx_send                           0x0001e2d9   Thumb Code    56  app_uart_fifo.o(i.action_tx_send)
    i.action_tx_stop                         0x0001e324   Section        0  app_uart_fifo.o(i.action_tx_stop)
    i.action_uart_deactivate                 0x0001e348   Section        0  app_uart_fifo.o(i.action_uart_deactivate)
    action_uart_deactivate                   0x0001e349   Thumb Code    20  app_uart_fifo.o(i.action_uart_deactivate)
    i.adv_report_parse                       0x0001e368   Section        0  main.o(i.adv_report_parse)
    adv_report_parse                         0x0001e369   Thumb Code    46  main.o(i.adv_report_parse)
    i.app_error_handler                      0x0001e398   Section        0  app_error.o(i.app_error_handler)
    i.app_evt_notify                         0x0001e3b4   Section        0  device_manager_central.o(i.app_evt_notify)
    app_evt_notify                           0x0001e3b5   Thumb Code     6  device_manager_central.o(i.app_evt_notify)
    i.app_fifo_get                           0x0001e3c0   Section        0  app_fifo.o(i.app_fifo_get)
    i.app_fifo_put                           0x0001e3e2   Section        0  app_fifo.o(i.app_fifo_put)
    i.app_notify                             0x0001e404   Section        0  pstorage.o(i.app_notify)
    app_notify                               0x0001e405   Thumb Code    34  pstorage.o(i.app_notify)
    i.app_notify_error_state_transit         0x0001e430   Section        0  pstorage.o(i.app_notify_error_state_transit)
    app_notify_error_state_transit           0x0001e431   Thumb Code    26  pstorage.o(i.app_notify_error_state_transit)
    i.app_pwm_channel_duty_set               0x0001e450   Section        0  app_pwm.o(i.app_pwm_channel_duty_set)
    i.app_pwm_channel_duty_ticks_set         0x0001e470   Section        0  app_pwm.o(i.app_pwm_channel_duty_ticks_set)
    i.app_pwm_channel_init                   0x0001e4fc   Section        0  app_pwm.o(i.app_pwm_channel_init)
    app_pwm_channel_init                     0x0001e4fd   Thumb Code   200  app_pwm.o(i.app_pwm_channel_init)
    i.app_pwm_enable                         0x0001e5c8   Section        0  app_pwm.o(i.app_pwm_enable)
    i.app_pwm_init                           0x0001e5dc   Section        0  app_pwm.o(i.app_pwm_init)
    i.are_app_channels                       0x0001e758   Section        0  nrf_drv_ppi.o(i.are_app_channels)
    are_app_channels                         0x0001e759   Thumb Code    12  nrf_drv_ppi.o(i.are_app_channels)
    i.ble_db_discovery_evt_register          0x0001e764   Section        0  ble_db_discovery.o(i.ble_db_discovery_evt_register)
    i.ble_db_discovery_init                  0x0001e7b0   Section        0  ble_db_discovery.o(i.ble_db_discovery_init)
    i.ble_db_discovery_on_ble_evt            0x0001e7c8   Section        0  ble_db_discovery.o(i.ble_db_discovery_on_ble_evt)
    i.ble_db_discovery_start                 0x0001e868   Section        0  ble_db_discovery.o(i.ble_db_discovery_start)
    i.ble_evt_dispatch                       0x0001e8c8   Section        0  main.o(i.ble_evt_dispatch)
    ble_evt_dispatch                         0x0001e8c9   Thumb Code    22  main.o(i.ble_evt_dispatch)
    i.ble_stack_init                         0x0001e8e0   Section        0  main.o(i.ble_stack_init)
    ble_stack_init                           0x0001e8e1   Thumb Code    92  main.o(i.ble_stack_init)
    i.channel_free                           0x0001e948   Section        0  nrf_drv_gpiote.o(i.channel_free)
    channel_free                             0x0001e949   Thumb Code    22  nrf_drv_gpiote.o(i.channel_free)
    i.channel_port_alloc                     0x0001e964   Section        0  nrf_drv_gpiote.o(i.channel_port_alloc)
    channel_port_alloc                       0x0001e965   Thumb Code    64  nrf_drv_gpiote.o(i.channel_port_alloc)
    i.channel_port_get                       0x0001e9a8   Section        0  nrf_drv_gpiote.o(i.channel_port_get)
    channel_port_get                         0x0001e9a9   Thumb Code    10  nrf_drv_gpiote.o(i.channel_port_get)
    i.characteristics_discover               0x0001e9b8   Section        0  ble_db_discovery.o(i.characteristics_discover)
    characteristics_discover                 0x0001e9b9   Thumb Code    56  ble_db_discovery.o(i.characteristics_discover)
    i.clear_operation_execute                0x0001e9f0   Section        0  pstorage.o(i.clear_operation_execute)
    clear_operation_execute                  0x0001e9f1   Thumb Code   252  pstorage.o(i.clear_operation_execute)
    i.clear_post_processing_run              0x0001eaf4   Section        0  pstorage.o(i.clear_post_processing_run)
    clear_post_processing_run                0x0001eaf5   Thumb Code    32  pstorage.o(i.clear_post_processing_run)
    i.client_find                            0x0001eb18   Section        0  client_handling.o(i.client_find)
    client_find                              0x0001eb19   Thumb Code    30  client_handling.o(i.client_find)
    i.client_handling_ble_evt_handler        0x0001eb3c   Section        0  client_handling.o(i.client_handling_ble_evt_handler)
    i.client_handling_create                 0x0001ec6c   Section        0  client_handling.o(i.client_handling_create)
    i.client_handling_destroy                0x0001ecd0   Section        0  client_handling.o(i.client_handling_destroy)
    i.client_handling_dm_event_handler       0x0001ed34   Section        0  client_handling.o(i.client_handling_dm_event_handler)
    i.client_handling_init                   0x0001ed58   Section        0  client_handling.o(i.client_handling_init)
    i.cmd_process                            0x0001edf8   Section        0  pstorage.o(i.cmd_process)
    cmd_process                              0x0001edf9   Thumb Code    46  pstorage.o(i.cmd_process)
    i.cmd_queue_element_init                 0x0001ee30   Section        0  pstorage.o(i.cmd_queue_element_init)
    cmd_queue_element_init                   0x0001ee31   Thumb Code    26  pstorage.o(i.cmd_queue_element_init)
    i.cmd_queue_enqueue                      0x0001ee50   Section        0  pstorage.o(i.cmd_queue_enqueue)
    cmd_queue_enqueue                        0x0001ee51   Thumb Code    68  pstorage.o(i.cmd_queue_enqueue)
    i.command_end_procedure_run              0x0001ee9c   Section        0  pstorage.o(i.command_end_procedure_run)
    command_end_procedure_run                0x0001ee9d   Thumb Code    56  pstorage.o(i.command_end_procedure_run)
    i.connection_instance_find               0x0001eed8   Section        0  device_manager_central.o(i.connection_instance_find)
    connection_instance_find                 0x0001eed9   Thumb Code    54  device_manager_central.o(i.connection_instance_find)
    i.connection_instance_init               0x0001ef18   Section        0  device_manager_central.o(i.connection_instance_init)
    connection_instance_init                 0x0001ef19   Thumb Code    30  device_manager_central.o(i.connection_instance_init)
    i.current_int_priority_get               0x0001ef3c   Section        0  nrf_drv_ppi.o(i.current_int_priority_get)
    current_int_priority_get                 0x0001ef3d   Thumb Code    60  nrf_drv_ppi.o(i.current_int_priority_get)
    i.data_page_erase_state_run              0x0001ef80   Section        0  pstorage.o(i.data_page_erase_state_run)
    data_page_erase_state_run                0x0001ef81   Thumb Code    80  pstorage.o(i.data_page_erase_state_run)
    i.data_to_swap_write_state_run           0x0001efd4   Section        0  pstorage.o(i.data_to_swap_write_state_run)
    data_to_swap_write_state_run             0x0001efd5   Thumb Code    34  pstorage.o(i.data_to_swap_write_state_run)
    i.db_discovery_acc_evt_handler           0x0001effc   Section        0  client_handling.o(i.db_discovery_acc_evt_handler)
    db_discovery_acc_evt_handler             0x0001effd   Thumb Code   162  client_handling.o(i.db_discovery_acc_evt_handler)
    i.db_discovery_evt_handler               0x0001f0ac   Section        0  client_handling.o(i.db_discovery_evt_handler)
    db_discovery_evt_handler                 0x0001f0ad   Thumb Code    86  client_handling.o(i.db_discovery_evt_handler)
    i.debug_printf                           0x0001f110   Section        0  debug_util.o(i.debug_printf)
    i.descriptors_discover                   0x0001f12e   Section        0  ble_db_discovery.o(i.descriptors_discover)
    descriptors_discover                     0x0001f12f   Thumb Code   132  ble_db_discovery.o(i.descriptors_discover)
    i.device_context_store                   0x0001f1b4   Section        0  device_manager_central.o(i.device_context_store)
    device_context_store                     0x0001f1b5   Thumb Code   150  device_manager_central.o(i.device_context_store)
    i.device_instance_allocate               0x0001f268   Section        0  device_manager_central.o(i.device_instance_allocate)
    device_instance_allocate                 0x0001f269   Thumb Code    74  device_manager_central.o(i.device_instance_allocate)
    i.device_manager_event_handler           0x0001f2bc   Section        0  main.o(i.device_manager_event_handler)
    device_manager_event_handler             0x0001f2bd   Thumb Code   180  main.o(i.device_manager_event_handler)
    i.device_manager_init                    0x0001f374   Section        0  main.o(i.device_manager_init)
    device_manager_init                      0x0001f375   Thumb Code   144  main.o(i.device_manager_init)
    i.discovery_complete_evt_trigger         0x0001f410   Section        0  ble_db_discovery.o(i.discovery_complete_evt_trigger)
    discovery_complete_evt_trigger           0x0001f411   Thumb Code   100  ble_db_discovery.o(i.discovery_complete_evt_trigger)
    i.discovery_error_evt_trigger            0x0001f47c   Section        0  ble_db_discovery.o(i.discovery_error_evt_trigger)
    discovery_error_evt_trigger              0x0001f47d   Thumb Code    72  ble_db_discovery.o(i.discovery_error_evt_trigger)
    i.dm_ble_evt_handler                     0x0001f4cc   Section        0  device_manager_central.o(i.dm_ble_evt_handler)
    i.dm_handle_initialize                   0x0001f83c   Section        0  device_manager_central.o(i.dm_handle_initialize)
    i.dm_init                                0x0001f858   Section        0  device_manager_central.o(i.dm_init)
    i.dm_pstorage_cb_handler                 0x0001f918   Section        0  device_manager_central.o(i.dm_pstorage_cb_handler)
    dm_pstorage_cb_handler                   0x0001f919   Thumb Code   364  device_manager_central.o(i.dm_pstorage_cb_handler)
    i.dm_register                            0x0001fa90   Section        0  device_manager_central.o(i.dm_register)
    i.dm_security_setup_req                  0x0001fae8   Section        0  device_manager_central.o(i.dm_security_setup_req)
    i.flash_api_err_code_process             0x0001fbbc   Section        0  pstorage.o(i.flash_api_err_code_process)
    flash_api_err_code_process               0x0001fbbd   Thumb Code    28  pstorage.o(i.flash_api_err_code_process)
    i.flash_operation_success_run            0x0001fbdc   Section        0  pstorage.o(i.flash_operation_success_run)
    flash_operation_success_run              0x0001fbdd   Thumb Code   114  pstorage.o(i.flash_operation_success_run)
    i.flash_page_erase                       0x0001fc5c   Section        0  pstorage.o(i.flash_page_erase)
    flash_page_erase                         0x0001fc5d   Thumb Code    10  pstorage.o(i.flash_page_erase)
    i.flash_write                            0x0001fc66   Section        0  pstorage.o(i.flash_write)
    flash_write                              0x0001fc67   Thumb Code    10  pstorage.o(i.flash_write)
    i.gattc_context_apply                    0x0001fc70   Section        0  device_manager_central.o(i.gattc_context_apply)
    gattc_context_apply                      0x0001fc71   Thumb Code     4  device_manager_central.o(i.gattc_context_apply)
    i.gattc_context_load                     0x0001fc74   Section        0  device_manager_central.o(i.gattc_context_load)
    gattc_context_load                       0x0001fc75   Thumb Code     4  device_manager_central.o(i.gattc_context_load)
    i.gattc_context_store                    0x0001fc78   Section        0  device_manager_central.o(i.gattc_context_store)
    gattc_context_store                      0x0001fc79   Thumb Code     4  device_manager_central.o(i.gattc_context_store)
    i.gatts_context_apply                    0x0001fc7c   Section        0  device_manager_central.o(i.gatts_context_apply)
    gatts_context_apply                      0x0001fc7d   Thumb Code    56  device_manager_central.o(i.gatts_context_apply)
    i.gatts_context_load                     0x0001fcbc   Section        0  device_manager_central.o(i.gatts_context_load)
    gatts_context_load                       0x0001fcbd   Thumb Code    42  device_manager_central.o(i.gatts_context_load)
    i.gatts_context_store                    0x0001fcec   Section        0  device_manager_central.o(i.gatts_context_store)
    gatts_context_store                      0x0001fced   Thumb Code   146  device_manager_central.o(i.gatts_context_store)
    i.gattsc_context_apply                   0x0001fd8c   Section        0  device_manager_central.o(i.gattsc_context_apply)
    gattsc_context_apply                     0x0001fd8d   Thumb Code     8  device_manager_central.o(i.gattsc_context_apply)
    i.gattsc_context_load                    0x0001fd94   Section        0  device_manager_central.o(i.gattsc_context_load)
    gattsc_context_load                      0x0001fd95   Thumb Code     8  device_manager_central.o(i.gattsc_context_load)
    i.gattsc_context_store                   0x0001fd9c   Section        0  device_manager_central.o(i.gattsc_context_store)
    gattsc_context_store                     0x0001fd9d   Thumb Code     8  device_manager_central.o(i.gattsc_context_store)
    i.head_restore_state_run                 0x0001fda4   Section        0  pstorage.o(i.head_restore_state_run)
    head_restore_state_run                   0x0001fda5   Thumb Code   110  pstorage.o(i.head_restore_state_run)
    i.initiate_security_request              0x0001fe1c   Section        0  device_manager_central.o(i.initiate_security_request)
    i.intern_softdevice_events_execute       0x0001fe78   Section        0  softdevice_handler.o(i.intern_softdevice_events_execute)
    i.is_allocated_channel                   0x0001fef8   Section        0  nrf_drv_ppi.o(i.is_allocated_channel)
    is_allocated_channel                     0x0001fef9   Thumb Code    20  nrf_drv_ppi.o(i.is_allocated_channel)
    i.is_allocated_group                     0x0001ff10   Section        0  nrf_drv_ppi.o(i.is_allocated_group)
    is_allocated_group                       0x0001ff11   Thumb Code    20  nrf_drv_ppi.o(i.is_allocated_group)
    i.is_app_channel                         0x0001ff28   Section        0  nrf_drv_ppi.o(i.is_app_channel)
    is_app_channel                           0x0001ff29   Thumb Code    14  nrf_drv_ppi.o(i.is_app_channel)
    i.is_app_group                           0x0001ff36   Section        0  nrf_drv_ppi.o(i.is_app_group)
    is_app_group                             0x0001ff37   Thumb Code    12  nrf_drv_ppi.o(i.is_app_group)
    i.is_desc_discovery_reqd                 0x0001ff42   Section        0  ble_db_discovery.o(i.is_desc_discovery_reqd)
    is_desc_discovery_reqd                   0x0001ff43   Thumb Code    66  ble_db_discovery.o(i.is_desc_discovery_reqd)
    i.is_manual_peripheral_setup_needed      0x0001ff84   Section        0  system_nrf51.o(i.is_manual_peripheral_setup_needed)
    is_manual_peripheral_setup_needed        0x0001ff85   Thumb Code    66  system_nrf51.o(i.is_manual_peripheral_setup_needed)
    i.is_page_erase_required                 0x0001ffcc   Section        0  pstorage.o(i.is_page_erase_required)
    is_page_erase_required                   0x0001ffcd   Thumb Code    60  pstorage.o(i.is_page_erase_required)
    i.is_programmable_app_channel            0x00020010   Section        0  nrf_drv_ppi.o(i.is_programmable_app_channel)
    is_programmable_app_channel              0x00020011   Thumb Code    12  nrf_drv_ppi.o(i.is_programmable_app_channel)
    i.is_word_aligned                        0x0002001c   Section        0  pstorage.o(i.is_word_aligned)
    is_word_aligned                          0x0002001d   Thumb Code    12  pstorage.o(i.is_word_aligned)
    i.main                                   0x00020028   Section        0  main.o(i.main)
    i.main_state_err_busy_process            0x0002015c   Section        0  pstorage.o(i.main_state_err_busy_process)
    main_state_err_busy_process              0x0002015d   Thumb Code    20  pstorage.o(i.main_state_err_busy_process)
    i.make_alarm                             0x00020174   Section        0  main.o(i.make_alarm)
    i.no_service_context_apply               0x000201e4   Section        0  device_manager_central.o(i.no_service_context_apply)
    no_service_context_apply                 0x000201e5   Thumb Code     4  device_manager_central.o(i.no_service_context_apply)
    i.no_service_context_load                0x000201e8   Section        0  device_manager_central.o(i.no_service_context_load)
    no_service_context_load                  0x000201e9   Thumb Code     4  device_manager_central.o(i.no_service_context_load)
    i.no_service_context_store               0x000201ec   Section        0  device_manager_central.o(i.no_service_context_store)
    no_service_context_store                 0x000201ed   Thumb Code     4  device_manager_central.o(i.no_service_context_store)
    i.notif_enable                           0x000201f0   Section        0  client_handling.o(i.notif_enable)
    notif_enable                             0x000201f1   Thumb Code    66  client_handling.o(i.notif_enable)
    i.nrf_delay_ms                           0x00020234   Section        0  nrf_delay.o(i.nrf_delay_ms)
    i.nrf_drv_common_irq_enable              0x00020250   Section        0  nrf_drv_common.o(i.nrf_drv_common_irq_enable)
    i.nrf_drv_gpiote_init                    0x000202b0   Section        0  nrf_drv_gpiote.o(i.nrf_drv_gpiote_init)
    i.nrf_drv_gpiote_is_init                 0x00020304   Section        0  nrf_drv_gpiote.o(i.nrf_drv_gpiote_is_init)
    i.nrf_drv_gpiote_out_init                0x00020314   Section        0  nrf_drv_gpiote.o(i.nrf_drv_gpiote_out_init)
    i.nrf_drv_gpiote_out_task_addr_get       0x000203a8   Section        0  nrf_drv_gpiote.o(i.nrf_drv_gpiote_out_task_addr_get)
    i.nrf_drv_gpiote_out_task_enable         0x000203bc   Section        0  nrf_drv_gpiote.o(i.nrf_drv_gpiote_out_task_enable)
    i.nrf_drv_gpiote_out_task_force          0x000203ec   Section        0  nrf_drv_gpiote.o(i.nrf_drv_gpiote_out_task_force)
    i.nrf_drv_gpiote_out_task_trigger        0x0002041c   Section        0  nrf_drv_gpiote.o(i.nrf_drv_gpiote_out_task_trigger)
    i.nrf_drv_gpiote_out_uninit              0x00020434   Section        0  nrf_drv_gpiote.o(i.nrf_drv_gpiote_out_uninit)
    i.nrf_drv_ppi_channel_alloc              0x00020464   Section        0  nrf_drv_ppi.o(i.nrf_drv_ppi_channel_alloc)
    i.nrf_drv_ppi_channel_assign             0x000204f4   Section        0  nrf_drv_ppi.o(i.nrf_drv_ppi_channel_assign)
    i.nrf_drv_ppi_channel_disable            0x00020534   Section        0  nrf_drv_ppi.o(i.nrf_drv_ppi_channel_disable)
    i.nrf_drv_ppi_channel_enable             0x0002056c   Section        0  nrf_drv_ppi.o(i.nrf_drv_ppi_channel_enable)
    i.nrf_drv_ppi_channel_free               0x000205a4   Section        0  nrf_drv_ppi.o(i.nrf_drv_ppi_channel_free)
    i.nrf_drv_ppi_channels_include_in_group  0x00020614   Section        0  nrf_drv_ppi.o(i.nrf_drv_ppi_channels_include_in_group)
    i.nrf_drv_ppi_channels_remove_from_group 0x00020698   Section        0  nrf_drv_ppi.o(i.nrf_drv_ppi_channels_remove_from_group)
    i.nrf_drv_ppi_group_alloc                0x0002071c   Section        0  nrf_drv_ppi.o(i.nrf_drv_ppi_group_alloc)
    i.nrf_drv_ppi_group_enable               0x000207a8   Section        0  nrf_drv_ppi.o(i.nrf_drv_ppi_group_enable)
    i.nrf_drv_ppi_group_free                 0x000207d8   Section        0  nrf_drv_ppi.o(i.nrf_drv_ppi_group_free)
    i.nrf_drv_ppi_init                       0x0002085c   Section        0  nrf_drv_ppi.o(i.nrf_drv_ppi_init)
    i.nrf_drv_timer_clear                    0x00020874   Section        0  nrf_drv_timer.o(i.nrf_drv_timer_clear)
    i.nrf_drv_timer_compare                  0x0002087c   Section        0  nrf_drv_timer.o(i.nrf_drv_timer_compare)
    i.nrf_drv_timer_compare_event_address_get 0x000208a6   Section        0  nrf_drv_timer.o(i.nrf_drv_timer_compare_event_address_get)
    i.nrf_drv_timer_compare_int_disable      0x000208b4   Section        0  nrf_drv_timer.o(i.nrf_drv_timer_compare_int_disable)
    i.nrf_drv_timer_compare_int_enable       0x000208c6   Section        0  nrf_drv_timer.o(i.nrf_drv_timer_compare_int_enable)
    i.nrf_drv_timer_disable                  0x000208e8   Section        0  nrf_drv_timer.o(i.nrf_drv_timer_disable)
    i.nrf_drv_timer_enable                   0x000208fc   Section        0  nrf_drv_timer.o(i.nrf_drv_timer_enable)
    i.nrf_drv_timer_extended_compare         0x00020910   Section        0  nrf_drv_timer.o(i.nrf_drv_timer_extended_compare)
    i.nrf_drv_timer_init                     0x00020940   Section        0  nrf_drv_timer.o(i.nrf_drv_timer_init)
    i.nrf_drv_timer_uninit                   0x000209e4   Section        0  nrf_drv_timer.o(i.nrf_drv_timer_uninit)
    i.nrf_drv_timer_us_to_ticks              0x00020a48   Section        0  nrf_drv_timer.o(i.nrf_drv_timer_us_to_ticks)
    i.nrf_gpio_cfg_sense_set                 0x00020a60   Section        0  nrf_drv_gpiote.o(i.nrf_gpio_cfg_sense_set)
    nrf_gpio_cfg_sense_set                   0x00020a61   Thumb Code    26  nrf_drv_gpiote.o(i.nrf_gpio_cfg_sense_set)
    i.nrf_gpio_pin_set                       0x00020a80   Section        0  spi_master.o(i.nrf_gpio_pin_set)
    nrf_gpio_pin_set                         0x00020a81   Thumb Code    10  spi_master.o(i.nrf_gpio_pin_set)
    i.nrf_gpiote_event_is_set                0x00020a90   Section        0  nrf_drv_gpiote.o(i.nrf_gpiote_event_is_set)
    nrf_gpiote_event_is_set                  0x00020a91   Thumb Code    14  nrf_drv_gpiote.o(i.nrf_gpiote_event_is_set)
    i.on_ble_evt                             0x00020aa4   Section        0  main.o(i.on_ble_evt)
    on_ble_evt                               0x00020aa5   Thumb Code   156  main.o(i.on_ble_evt)
    i.on_characteristic_discovery_rsp        0x00020b58   Section        0  ble_db_discovery.o(i.on_characteristic_discovery_rsp)
    on_characteristic_discovery_rsp          0x00020b59   Thumb Code   204  ble_db_discovery.o(i.on_characteristic_discovery_rsp)
    i.on_descriptor_discovery_rsp            0x00020c24   Section        0  ble_db_discovery.o(i.on_descriptor_discovery_rsp)
    on_descriptor_discovery_rsp              0x00020c25   Thumb Code   156  ble_db_discovery.o(i.on_descriptor_discovery_rsp)
    i.on_srv_disc_completion                 0x00020cc4   Section        0  ble_db_discovery.o(i.on_srv_disc_completion)
    on_srv_disc_completion                   0x00020cc5   Thumb Code    84  ble_db_discovery.o(i.on_srv_disc_completion)
    i.on_uart_event                          0x00020d20   Section        0  app_uart_fifo.o(i.on_uart_event)
    on_uart_event                            0x00020d21   Thumb Code   118  app_uart_fifo.o(i.on_uart_event)
    i.pan73_workaround                       0x00020da8   Section        0  app_pwm.o(i.pan73_workaround)
    pan73_workaround                         0x00020da9   Thumb Code    32  app_pwm.o(i.pan73_workaround)
    i.peer_instance_init                     0x00020de0   Section        0  device_manager_central.o(i.peer_instance_init)
    peer_instance_init                       0x00020de1   Thumb Code    46  device_manager_central.o(i.peer_instance_init)
    i.pending_user_evts_send                 0x00020e14   Section        0  ble_db_discovery.o(i.pending_user_evts_send)
    pending_user_evts_send                   0x00020e15   Thumb Code    34  ble_db_discovery.o(i.pending_user_evts_send)
    i.pin_in_use_by_te                       0x00020e40   Section        0  nrf_drv_gpiote.o(i.pin_in_use_by_te)
    pin_in_use_by_te                         0x00020e41   Thumb Code    20  nrf_drv_gpiote.o(i.pin_in_use_by_te)
    i.pstorage_access_status_get             0x00020e58   Section        0  pstorage.o(i.pstorage_access_status_get)
    i.pstorage_block_identifier_get          0x00020e80   Section        0  pstorage.o(i.pstorage_block_identifier_get)
    i.pstorage_clear                         0x00020ed4   Section        0  pstorage.o(i.pstorage_clear)
    i.pstorage_flash_page_end                0x00020f78   Section        0  pstorage.o(i.pstorage_flash_page_end)
    pstorage_flash_page_end                  0x00020f79   Thumb Code    32  pstorage.o(i.pstorage_flash_page_end)
    i.pstorage_flash_page_size               0x00020f9c   Section        0  pstorage.o(i.pstorage_flash_page_size)
    pstorage_flash_page_size                 0x00020f9d   Thumb Code    10  pstorage.o(i.pstorage_flash_page_size)
    i.pstorage_init                          0x00020fa8   Section        0  pstorage.o(i.pstorage_init)
    i.pstorage_load                          0x00020ff4   Section        0  pstorage.o(i.pstorage_load)
    i.pstorage_register                      0x0002109c   Section        0  pstorage.o(i.pstorage_register)
    i.pstorage_store                         0x00021150   Section        0  pstorage.o(i.pstorage_store)
    i.pstorage_sys_event_handler             0x000211e0   Section        0  pstorage.o(i.pstorage_sys_event_handler)
    i.pstorage_update                        0x0002122c   Section        0  pstorage.o(i.pstorage_update)
    i.pwm_channel_ppi_disable                0x000212bc   Section        0  app_pwm.o(i.pwm_channel_ppi_disable)
    pwm_channel_ppi_disable                  0x000212bd   Thumb Code    24  app_pwm.o(i.pwm_channel_ppi_disable)
    i.pwm_dealloc                            0x000212d4   Section        0  app_pwm.o(i.pwm_dealloc)
    pwm_dealloc                              0x000212d5   Thumb Code   128  app_pwm.o(i.pwm_dealloc)
    i.pwm_ppi_disable                        0x00021354   Section        0  app_pwm.o(i.pwm_ppi_disable)
    pwm_ppi_disable                          0x00021355   Thumb Code    20  app_pwm.o(i.pwm_ppi_disable)
    i.pwm_ready_callback                     0x00021368   Section        0  main.o(i.pwm_ready_callback)
    i.pwm_ready_tick                         0x00021374   Section        0  app_pwm.o(i.pwm_ready_tick)
    i.pwm_set_value                          0x000213ac   Section        0  main.o(i.pwm_set_value)
    i.pwm_transition_0or100_to_0or100        0x000213f0   Section        0  app_pwm.o(i.pwm_transition_0or100_to_0or100)
    pwm_transition_0or100_to_0or100          0x000213f1   Thumb Code   102  app_pwm.o(i.pwm_transition_0or100_to_0or100)
    i.pwm_transition_0or100_to_n             0x00021458   Section        0  app_pwm.o(i.pwm_transition_0or100_to_n)
    pwm_transition_0or100_to_n               0x00021459   Thumb Code   132  app_pwm.o(i.pwm_transition_0or100_to_n)
    i.pwm_transition_n_to_0or100             0x000214e4   Section        0  app_pwm.o(i.pwm_transition_n_to_0or100)
    pwm_transition_n_to_0or100               0x000214e5   Thumb Code   128  app_pwm.o(i.pwm_transition_n_to_0or100)
    i.pwm_transition_n_to_m                  0x0002156c   Section        0  app_pwm.o(i.pwm_transition_n_to_m)
    pwm_transition_n_to_m                    0x0002156d   Thumb Code   156  app_pwm.o(i.pwm_transition_n_to_m)
    i.read_acc_other_device                  0x0002160c   Section        0  client_handling.o(i.read_acc_other_device)
    i.registered_handler_get                 0x0002161c   Section        0  ble_db_discovery.o(i.registered_handler_get)
    registered_handler_get                   0x0002161d   Thumb Code    50  ble_db_discovery.o(i.registered_handler_get)
    i.scan_start                             0x00021658   Section        0  main.o(i.scan_start)
    scan_start                               0x00021659   Thumb Code    52  main.o(i.scan_start)
    i.simple_uart_config                     0x00021694   Section        0  simple_uart.o(i.simple_uart_config)
    i.simple_uart_put                        0x000216f4   Section        0  simple_uart.o(i.simple_uart_put)
    i.simple_uart_putstring                  0x00021710   Section        0  simple_uart.o(i.simple_uart_putstring)
    i.sm_state_change                        0x00021728   Section        0  pstorage.o(i.sm_state_change)
    sm_state_change                          0x00021729   Thumb Code    62  pstorage.o(i.sm_state_change)
    i.softdevice_assertion_handler           0x00021770   Section        0  softdevice_handler.o(i.softdevice_assertion_handler)
    i.softdevice_ble_evt_handler_set         0x0002177c   Section        0  softdevice_handler.o(i.softdevice_ble_evt_handler_set)
    i.softdevice_handler_init                0x00021790   Section        0  softdevice_handler.o(i.softdevice_handler_init)
    i.softdevice_sys_evt_handler_set         0x000217c0   Section        0  softdevice_handler.o(i.softdevice_sys_evt_handler_set)
    i.spi_master_buffer_release              0x000217d4   Section        0  spi_master.o(i.spi_master_buffer_release)
    spi_master_buffer_release                0x000217d5   Thumb Code    40  spi_master.o(i.spi_master_buffer_release)
    i.spi_master_get_instance                0x000217fc   Section        0  spi_master.o(i.spi_master_get_instance)
    spi_master_get_instance                  0x000217fd   Thumb Code    12  spi_master.o(i.spi_master_get_instance)
    i.spi_master_send_recv_irq               0x0002180c   Section        0  spi_master.o(i.spi_master_send_recv_irq)
    spi_master_send_recv_irq                 0x0002180d   Thumb Code   180  spi_master.o(i.spi_master_send_recv_irq)
    i.spi_master_signal_evt                  0x000218c0   Section        0  spi_master.o(i.spi_master_signal_evt)
    spi_master_signal_evt                    0x000218c1   Thumb Code    46  spi_master.o(i.spi_master_signal_evt)
    i.state_data_erase_swap_entry_run        0x000218f4   Section        0  pstorage.o(i.state_data_erase_swap_entry_run)
    state_data_erase_swap_entry_run          0x000218f5   Thumb Code    92  pstorage.o(i.state_data_erase_swap_entry_run)
    i.state_erase_data_page_entry_run        0x00021958   Section        0  pstorage.o(i.state_erase_data_page_entry_run)
    state_erase_data_page_entry_run          0x00021959   Thumb Code    12  pstorage.o(i.state_erase_data_page_entry_run)
    i.state_restore_head_entry_run           0x00021968   Section        0  pstorage.o(i.state_restore_head_entry_run)
    state_restore_head_entry_run             0x00021969   Thumb Code    36  pstorage.o(i.state_restore_head_entry_run)
    i.state_restore_tail_entry_run           0x00021990   Section        0  pstorage.o(i.state_restore_tail_entry_run)
    state_restore_tail_entry_run             0x00021991   Thumb Code    66  pstorage.o(i.state_restore_tail_entry_run)
    i.state_swap_erase_entry_run             0x000219dc   Section        0  pstorage.o(i.state_swap_erase_entry_run)
    state_swap_erase_entry_run               0x000219dd   Thumb Code    32  pstorage.o(i.state_swap_erase_entry_run)
    i.state_write_data_swap_entry_run        0x000219fc   Section        0  pstorage.o(i.state_write_data_swap_entry_run)
    state_write_data_swap_entry_run          0x000219fd   Thumb Code    42  pstorage.o(i.state_write_data_swap_entry_run)
    i.storage_operation_dummy_handler        0x00021a2c   Section        0  device_manager_central.o(i.storage_operation_dummy_handler)
    storage_operation_dummy_handler          0x00021a2d   Thumb Code     4  device_manager_central.o(i.storage_operation_dummy_handler)
    i.store_cmd_flash_write_execute          0x00021a30   Section        0  pstorage.o(i.store_cmd_flash_write_execute)
    store_cmd_flash_write_execute            0x00021a31   Thumb Code    82  pstorage.o(i.store_cmd_flash_write_execute)
    i.swap_erase_state_run                   0x00021a8c   Section        0  pstorage.o(i.swap_erase_state_run)
    swap_erase_state_run                     0x00021a8d   Thumb Code    24  pstorage.o(i.swap_erase_state_run)
    i.swap_sub_state_err_busy_process        0x00021aa8   Section        0  pstorage.o(i.swap_sub_state_err_busy_process)
    swap_sub_state_err_busy_process          0x00021aa9   Thumb Code    20  pstorage.o(i.swap_sub_state_err_busy_process)
    i.swap_sub_state_state_change            0x00021ac0   Section        0  pstorage.o(i.swap_sub_state_state_change)
    swap_sub_state_state_change              0x00021ac1   Thumb Code    12  pstorage.o(i.swap_sub_state_state_change)
    i.sys_evt_dispatch                       0x00021ad4   Section        0  main.o(i.sys_evt_dispatch)
    sys_evt_dispatch                         0x00021ad5   Thumb Code    34  main.o(i.sys_evt_dispatch)
    i.tail_restore_state_run                 0x00021afc   Section        0  pstorage.o(i.tail_restore_state_run)
    tail_restore_state_run                   0x00021afd   Thumb Code    22  pstorage.o(i.tail_restore_state_run)
    i.update_status_bit_reset                0x00021b18   Section        0  device_manager_central.o(i.update_status_bit_reset)
    update_status_bit_reset                  0x00021b19   Thumb Code    14  device_manager_central.o(i.update_status_bit_reset)
    .constdata                               0x00021b2c   Section       32  client_handling.o(.constdata)
    .constdata                               0x00021b4c   Section        8  main.o(.constdata)
    .constdata                               0x00021b54   Section       52  main.o(.constdata)
    m_connection_param                       0x00021b5c   Data           8  main.o(.constdata)
    m_scan_param                             0x00021b64   Data          16  main.o(.constdata)
    .constdata                               0x00021b88   Section        4  spi_master.o(.constdata)
    .constdata                               0x00021b8c   Section       48  device_manager_central.o(.constdata)
    .constdata                               0x00021bbc   Section       40  pstorage.o(.constdata)
    swap_sub_state_sm_lut                    0x00021bbc   Data          20  pstorage.o(.constdata)
    swap_sub_state_sm_lut                    0x00021bd0   Data          20  pstorage.o(.constdata)
    .constdata                               0x00021be4   Section        8  nrf_drv_timer.o(.constdata)
    m_default_config                         0x00021be4   Data           8  nrf_drv_timer.o(.constdata)
    .constdata                               0x00021bec   Section       12  app_pwm.o(.constdata)
    .data                                    0x20002800   Section        3  client_handling.o(.data)
    char_discovery_flag                      0x20002800   Data           1  client_handling.o(.data)
    m_client_count                           0x20002801   Data           1  client_handling.o(.data)
    m_base_uuid_type                         0x20002802   Data           1  client_handling.o(.data)
    .data                                    0x20002804   Section       12  main.o(.data)
    m_peer_count                             0x20002804   Data           1  main.o(.data)
    alarm_flag                               0x20002805   Data           1  main.o(.data)
    alarm_flag_orientation                   0x20002806   Data           1  main.o(.data)
    alarm_flag_sound                         0x20002807   Data           1  main.o(.data)
    m_memory_access_in_progress              0x20002808   Data           1  main.o(.data)
    rssi                                     0x20002809   Data           1  main.o(.data)
    m_dm_app_id                              0x2000280a   Data           1  main.o(.data)
    counter                                  0x2000280b   Data           1  main.o(.data)
    ready_flag                               0x2000280c   Data           1  main.o(.data)
    m_conn_handle                            0x2000280e   Data           2  main.o(.data)
    .data                                    0x20002810   Section        4  system_nrf51.o(.data)
    __tagsym$$used                           0x20002810   Number         0  system_nrf51.o(.data)
    .data                                    0x20002814   Section       16  ble_db_discovery.o(.data)
    m_initialized                            0x20002814   Data           1  ble_db_discovery.o(.data)
    m_pending_usr_evt_index                  0x20002818   Data           4  ble_db_discovery.o(.data)
    m_num_of_handlers_reg                    0x2000281c   Data           4  ble_db_discovery.o(.data)
    m_num_of_discoveries_made                0x20002820   Data           4  ble_db_discovery.o(.data)
    .data                                    0x20002824   Section       16  device_manager_central.o(.data)
    m_module_initialized                     0x20002824   Data           1  device_manager_central.o(.data)
    m_peer_addr_update                       0x20002828   Data           4  device_manager_central.o(.data)
    m_storage_handle                         0x2000282c   Data           8  device_manager_central.o(.data)
    .data                                    0x20002834   Section        8  app_uart_fifo.o(.data)
    m_instance_counter                       0x20002834   Data           1  app_uart_fifo.o(.data)
    m_current_state                          0x20002835   Data           1  app_uart_fifo.o(.data)
    m_event_handler                          0x20002838   Data           4  app_uart_fifo.o(.data)
    .data                                    0x2000283c   Section       36  pstorage.o(.data)
    m_state                                  0x2000283c   Data           1  pstorage.o(.data)
    m_swap_sub_state                         0x2000283d   Data           1  pstorage.o(.data)
    m_next_app_instance                      0x2000283e   Data           2  pstorage.o(.data)
    m_flags                                  0x20002840   Data           4  pstorage.o(.data)
    m_next_page_addr                         0x20002844   Data           4  pstorage.o(.data)
    m_head_word_size                         0x20002848   Data           4  pstorage.o(.data)
    m_tail_word_size                         0x2000284c   Data           4  pstorage.o(.data)
    m_current_page_id                        0x20002850   Data           4  pstorage.o(.data)
    m_num_of_command_retries                 0x20002854   Data           4  pstorage.o(.data)
    m_num_of_bytes_written                   0x20002858   Data           4  pstorage.o(.data)
    m_app_data_size                          0x2000285c   Data           4  pstorage.o(.data)
    .data                                    0x20002860   Section        8  nrf_drv_ppi.o(.data)
    m_drv_state                              0x20002860   Data           1  nrf_drv_ppi.o(.data)
    m_groups_allocated                       0x20002861   Data           1  nrf_drv_ppi.o(.data)
    m_channels_allocated                     0x20002864   Data           4  nrf_drv_ppi.o(.data)
    .data                                    0x20002868   Section       12  nrf_drv_timer.o(.data)
    m_cb                                     0x20002868   Data           1  nrf_drv_timer.o(.data)
    m_timer_event_handlers                   0x2000286c   Data           4  nrf_drv_timer.o(.data)
    mp_contexts                              0x20002870   Data           4  nrf_drv_timer.o(.data)
    .data                                    0x20002874   Section        8  app_pwm.o(.data)
    m_instances                              0x20002878   Data           4  app_pwm.o(.data)
    .data                                    0x2000287c   Section       20  softdevice_handler.o(.data)
    m_softdevice_enabled                     0x2000287c   Data           1  softdevice_handler.o(.data)
    m_ble_evt_buffer_size                    0x2000287e   Data           2  softdevice_handler.o(.data)
    m_evt_schedule_func                      0x20002880   Data           4  softdevice_handler.o(.data)
    mp_ble_evt_buffer                        0x20002884   Data           4  softdevice_handler.o(.data)
    m_ble_evt_handler                        0x20002888   Data           4  softdevice_handler.o(.data)
    m_sys_evt_handler                        0x2000288c   Data           4  softdevice_handler.o(.data)
    .bss                                     0x20002890   Section      896  client_handling.o(.bss)
    m_client                                 0x20002890   Data         896  client_handling.o(.bss)
    .bss                                     0x20002c10   Section       72  main.o(.bss)
    BLE_EVT_BUFFER                           0x20002c10   Data          72  main.o(.bss)
    .bss                                     0x20002c58   Section       36  main.o(.bss)
    .bss                                     0x20002c7c   Section       40  spi_master.o(.bss)
    m_spi_master_instances                   0x20002c7c   Data          40  spi_master.o(.bss)
    .bss                                     0x20002ca4   Section      128  ble_db_discovery.o(.bss)
    m_registered_handlers                    0x20002ca4   Data          16  ble_db_discovery.o(.bss)
    m_pending_user_evts                      0x20002cb4   Data         112  ble_db_discovery.o(.bss)
    .bss                                     0x20002d24   Section      643  device_manager_central.o(.bss)
    m_peer_table                             0x20002d24   Data         192  device_manager_central.o(.bss)
    m_bond_table                             0x20002de4   Data         224  device_manager_central.o(.bss)
    m_gatts_table                            0x20002ec4   Data          96  device_manager_central.o(.bss)
    m_connection_table                       0x20002f24   Data          96  device_manager_central.o(.bss)
    m_application_table                      0x20002f84   Data          12  device_manager_central.o(.bss)
    m_local_id_info                          0x20002f90   Data          23  device_manager_central.o(.bss)
    .bss                                     0x20002fa8   Section       32  app_uart_fifo.o(.bss)
    m_rx_fifo                                0x20002fa8   Data          16  app_uart_fifo.o(.bss)
    m_tx_fifo                                0x20002fb8   Data          16  app_uart_fifo.o(.bss)
    .bss                                     0x20002fc8   Section       96  pstorage.o(.bss)
    m_cmd_queue                              0x20002fc8   Data          84  pstorage.o(.bss)
    m_app_table                              0x2000301c   Data          12  pstorage.o(.bss)
    .bss                                     0x20003028   Section       56  nrf_drv_gpiote.o(.bss)
    m_cb                                     0x20003028   Data          56  nrf_drv_gpiote.o(.bss)
    STACK                                    0x20003060   Section     2048  arm_startup_nrf51.o(STACK)

    Global Symbols

    Symbol Name                              Value     Ov Type        Size  Object(Section)

    BuildAttributes$$THM_ISAv3M$S$PE$A:L22$X:L11$S22$IEEE1$IW$USESV6$~STKCKD$USESV7$~SHL$OSPACE$ROPI$EBA8$MICROLIB$REQ8$PRES8$EABIv2 0x00000000   Number         0  anon$$obj.o ABSOLUTE
    __ARM_use_no_argv                        0x00000000   Number         0  main.o ABSOLUTE
    _printf_a                                0x00000000   Number         0  stubs.o ABSOLUTE
    _printf_c                                0x00000000   Number         0  stubs.o ABSOLUTE
    _printf_charcount                        0x00000000   Number         0  stubs.o ABSOLUTE
    _printf_d                                0x00000000   Number         0  stubs.o ABSOLUTE
    _printf_e                                0x00000000   Number         0  stubs.o ABSOLUTE
    _printf_f                                0x00000000   Number         0  stubs.o ABSOLUTE
    _printf_flags                            0x00000000   Number         0  stubs.o ABSOLUTE
    _printf_fp_dec                           0x00000000   Number         0  stubs.o ABSOLUTE
    _printf_fp_hex                           0x00000000   Number         0  stubs.o ABSOLUTE
    _printf_g                                0x00000000   Number         0  stubs.o ABSOLUTE
    _printf_i                                0x00000000   Number         0  stubs.o ABSOLUTE
    _printf_int_dec                          0x00000000   Number         0  stubs.o ABSOLUTE
    _printf_l                                0x00000000   Number         0  stubs.o ABSOLUTE
    _printf_lc                               0x00000000   Number         0  stubs.o ABSOLUTE
    _printf_ll                               0x00000000   Number         0  stubs.o ABSOLUTE
    _printf_lld                              0x00000000   Number         0  stubs.o ABSOLUTE
    _printf_lli                              0x00000000   Number         0  stubs.o ABSOLUTE
    _printf_llo                              0x00000000   Number         0  stubs.o ABSOLUTE
    _printf_llu                              0x00000000   Number         0  stubs.o ABSOLUTE
    _printf_llx                              0x00000000   Number         0  stubs.o ABSOLUTE
    _printf_longlong_dec                     0x00000000   Number         0  stubs.o ABSOLUTE
    _printf_longlong_hex                     0x00000000   Number         0  stubs.o ABSOLUTE
    _printf_longlong_oct                     0x00000000   Number         0  stubs.o ABSOLUTE
    _printf_ls                               0x00000000   Number         0  stubs.o ABSOLUTE
    _printf_mbtowc                           0x00000000   Number         0  stubs.o ABSOLUTE
    _printf_n                                0x00000000   Number         0  stubs.o ABSOLUTE
    _printf_o                                0x00000000   Number         0  stubs.o ABSOLUTE
    _printf_p                                0x00000000   Number         0  stubs.o ABSOLUTE
    _printf_percent                          0x00000000   Number         0  stubs.o ABSOLUTE
    _printf_pre_padding                      0x00000000   Number         0  stubs.o ABSOLUTE
    _printf_return_value                     0x00000000   Number         0  stubs.o ABSOLUTE
    _printf_s                                0x00000000   Number         0  stubs.o ABSOLUTE
    _printf_sizespec                         0x00000000   Number         0  stubs.o ABSOLUTE
    _printf_str                              0x00000000   Number         0  stubs.o ABSOLUTE
    _printf_truncate_signed                  0x00000000   Number         0  stubs.o ABSOLUTE
    _printf_truncate_unsigned                0x00000000   Number         0  stubs.o ABSOLUTE
    _printf_u                                0x00000000   Number         0  stubs.o ABSOLUTE
    _printf_wc                               0x00000000   Number         0  stubs.o ABSOLUTE
    _printf_wctomb                           0x00000000   Number         0  stubs.o ABSOLUTE
    _printf_widthprec                        0x00000000   Number         0  stubs.o ABSOLUTE
    _printf_x                                0x00000000   Number         0  stubs.o ABSOLUTE
    __cpp_initialize__aeabi_                  - Undefined Weak Reference
    __cxa_finalize                            - Undefined Weak Reference
    __decompress                              - Undefined Weak Reference
    _clock_init                               - Undefined Weak Reference
    _microlib_exit                            - Undefined Weak Reference
    __Vectors_Size                           0x000000c0   Number         0  arm_startup_nrf51.o ABSOLUTE
    __Vectors                                0x0001d000   Data           4  arm_startup_nrf51.o(RESET)
    __Vectors_End                            0x0001d0c0   Data           0  arm_startup_nrf51.o(RESET)
    __main                                   0x0001d0c1   Thumb Code     0  entry.o(.ARM.Collect$$$$00000000)
    _main_stk                                0x0001d0c1   Thumb Code     0  entry2.o(.ARM.Collect$$$$00000001)
    _main_scatterload                        0x0001d0c5   Thumb Code     0  entry5.o(.ARM.Collect$$$$00000004)
    __main_after_scatterload                 0x0001d0c9   Thumb Code     0  entry5.o(.ARM.Collect$$$$00000004)
    _main_clock                              0x0001d0c9   Thumb Code     0  entry7b.o(.ARM.Collect$$$$00000008)
    _main_cpp_init                           0x0001d0c9   Thumb Code     0  entry8b.o(.ARM.Collect$$$$0000000A)
    _main_init                               0x0001d0c9   Thumb Code     0  entry9a.o(.ARM.Collect$$$$0000000B)
    __rt_final_cpp                           0x0001d0d1   Thumb Code     0  entry10a.o(.ARM.Collect$$$$0000000D)
    __rt_final_exit                          0x0001d0d1   Thumb Code     0  entry11a.o(.ARM.Collect$$$$0000000F)
    __asm___11_nrf_delay_c_532987f3__nrf_delay_us 0x0001d0d5   Thumb Code    30  nrf_delay.o(.emb_text)
    Reset_Handler                            0x0001d0f5   Thumb Code    26  arm_startup_nrf51.o(.text)
    NMI_Handler                              0x0001d10f   Thumb Code     2  arm_startup_nrf51.o(.text)
    HardFault_Handler                        0x0001d111   Thumb Code     2  arm_startup_nrf51.o(.text)
    SVC_Handler                              0x0001d113   Thumb Code     2  arm_startup_nrf51.o(.text)
    PendSV_Handler                           0x0001d115   Thumb Code     2  arm_startup_nrf51.o(.text)
    SysTick_Handler                          0x0001d117   Thumb Code     2  arm_startup_nrf51.o(.text)
    ADC_IRQHandler                           0x0001d119   Thumb Code     0  arm_startup_nrf51.o(.text)
    CCM_AAR_IRQHandler                       0x0001d119   Thumb Code     0  arm_startup_nrf51.o(.text)
    ECB_IRQHandler                           0x0001d119   Thumb Code     0  arm_startup_nrf51.o(.text)
    LPCOMP_IRQHandler                        0x0001d119   Thumb Code     0  arm_startup_nrf51.o(.text)
    POWER_CLOCK_IRQHandler                   0x0001d119   Thumb Code     0  arm_startup_nrf51.o(.text)
    QDEC_IRQHandler                          0x0001d119   Thumb Code     0  arm_startup_nrf51.o(.text)
    RADIO_IRQHandler                         0x0001d119   Thumb Code     0  arm_startup_nrf51.o(.text)
    RNG_IRQHandler                           0x0001d119   Thumb Code     0  arm_startup_nrf51.o(.text)
    RTC0_IRQHandler                          0x0001d119   Thumb Code     0  arm_startup_nrf51.o(.text)
    RTC1_IRQHandler                          0x0001d119   Thumb Code     0  arm_startup_nrf51.o(.text)
    SPI1_TWI1_IRQHandler                     0x0001d119   Thumb Code     0  arm_startup_nrf51.o(.text)
    SWI0_IRQHandler                          0x0001d119   Thumb Code     0  arm_startup_nrf51.o(.text)
    SWI1_IRQHandler                          0x0001d119   Thumb Code     0  arm_startup_nrf51.o(.text)
    SWI3_IRQHandler                          0x0001d119   Thumb Code     0  arm_startup_nrf51.o(.text)
    SWI4_IRQHandler                          0x0001d119   Thumb Code     0  arm_startup_nrf51.o(.text)
    SWI5_IRQHandler                          0x0001d119   Thumb Code     0  arm_startup_nrf51.o(.text)
    TEMP_IRQHandler                          0x0001d119   Thumb Code     0  arm_startup_nrf51.o(.text)
    TIMER0_IRQHandler                        0x0001d119   Thumb Code     0  arm_startup_nrf51.o(.text)
    TIMER2_IRQHandler                        0x0001d119   Thumb Code     0  arm_startup_nrf51.o(.text)
    WDT_IRQHandler                           0x0001d119   Thumb Code     0  arm_startup_nrf51.o(.text)
    __aeabi_uidiv                            0x0001d12d   Thumb Code     0  uidiv.o(.text)
    __aeabi_uidivmod                         0x0001d12d   Thumb Code    44  uidiv.o(.text)
    __aeabi_idiv                             0x0001d159   Thumb Code     0  idiv.o(.text)
    __aeabi_idivmod                          0x0001d159   Thumb Code    40  idiv.o(.text)
    __aeabi_memcpy                           0x0001d181   Thumb Code    36  memcpya.o(.text)
    __aeabi_memcpy4                          0x0001d181   Thumb Code     0  memcpya.o(.text)
    __aeabi_memcpy8                          0x0001d181   Thumb Code     0  memcpya.o(.text)
    __aeabi_memset                           0x0001d1a5   Thumb Code    14  memseta.o(.text)
    __aeabi_memset4                          0x0001d1a5   Thumb Code     0  memseta.o(.text)
    __aeabi_memset8                          0x0001d1a5   Thumb Code     0  memseta.o(.text)
    __aeabi_memclr                           0x0001d1b3   Thumb Code     4  memseta.o(.text)
    __aeabi_memclr4                          0x0001d1b3   Thumb Code     0  memseta.o(.text)
    __aeabi_memclr8                          0x0001d1b3   Thumb Code     0  memseta.o(.text)
    _memset$wrapper                          0x0001d1b7   Thumb Code    18  memseta.o(.text)
    memcmp                                   0x0001d1c9   Thumb Code    26  memcmp.o(.text)
    __aeabi_uldivmod                         0x0001d1e3   Thumb Code    96  uldiv.o(.text)
    __I$use$fp                               0x0001d243   Thumb Code     0  iusefp.o(.text)
    __aeabi_dadd                             0x0001d245   Thumb Code   328  dadd.o(.text)
    __aeabi_dsub                             0x0001d38d   Thumb Code    12  dadd.o(.text)
    __aeabi_drsub                            0x0001d399   Thumb Code    12  dadd.o(.text)
    __aeabi_dmul                             0x0001d3a9   Thumb Code   202  dmul.o(.text)
    __aeabi_ddiv                             0x0001d479   Thumb Code   234  ddiv.o(.text)
    __aeabi_d2ulz                            0x0001d569   Thumb Code    54  dfixul.o(.text)
    __aeabi_cdrcmple                         0x0001d5a9   Thumb Code    38  cdrcmple.o(.text)
    __scatterload                            0x0001d5d1   Thumb Code    28  init.o(.text)
    __scatterload_rt2                        0x0001d5d1   Thumb Code     0  init.o(.text)
    __aeabi_llsl                             0x0001d5f5   Thumb Code    32  llshl.o(.text)
    _ll_shift_l                              0x0001d5f5   Thumb Code     0  llshl.o(.text)
    __aeabi_llsr                             0x0001d615   Thumb Code    34  llushr.o(.text)
    _ll_ushift_r                             0x0001d615   Thumb Code     0  llushr.o(.text)
    __aeabi_lasr                             0x0001d637   Thumb Code    38  llsshr.o(.text)
    _ll_sshift_r                             0x0001d637   Thumb Code     0  llsshr.o(.text)
    _double_round                            0x0001d65d   Thumb Code    26  depilogue.o(.text)
    _double_epilogue                         0x0001d677   Thumb Code   164  depilogue.o(.text)
    GPIOTE_IRQHandler                        0x0001d71d   Thumb Code   224  nrf_drv_gpiote.o(i.GPIOTE_IRQHandler)
    SPI0_TWI0_IRQHandler                     0x0001d819   Thumb Code    34  spi_master.o(i.SPI0_TWI0_IRQHandler)
    SWI2_IRQHandler                          0x0001d845   Thumb Code    32  softdevice_handler.o(i.SWI2_IRQHandler)
    SystemInit                               0x0001d869   Thumb Code    64  system_nrf51.o(i.SystemInit)
    TIMER1_IRQHandler                        0x0001d8bd   Thumb Code    66  nrf_drv_timer.o(i.TIMER1_IRQHandler)
    UART0_IRQHandler                         0x0001d909   Thumb Code   110  app_uart_fifo.o(i.UART0_IRQHandler)
    __0sprintf                               0x0001d989   Thumb Code    36  printfa.o(i.__0sprintf)
    __1sprintf                               0x0001d989   Thumb Code     0  printfa.o(i.__0sprintf)
    __2sprintf                               0x0001d989   Thumb Code     0  printfa.o(i.__0sprintf)
    __c89sprintf                             0x0001d989   Thumb Code     0  printfa.o(i.__0sprintf)
    sprintf                                  0x0001d989   Thumb Code     0  printfa.o(i.__0sprintf)
    __0vsprintf                              0x0001d9b1   Thumb Code    30  printfa.o(i.__0vsprintf)
    __1vsprintf                              0x0001d9b1   Thumb Code     0  printfa.o(i.__0vsprintf)
    __2vsprintf                              0x0001d9b1   Thumb Code     0  printfa.o(i.__0vsprintf)
    __c89vsprintf                            0x0001d9b1   Thumb Code     0  printfa.o(i.__0vsprintf)
    vsprintf                                 0x0001d9b1   Thumb Code     0  printfa.o(i.__0vsprintf)
    __ARM_clz                                0x0001d9d5   Thumb Code    46  depilogue.o(i.__ARM_clz)
    __ARM_common_switch8                     0x0001da03   Thumb Code    26  client_handling.o(i.__ARM_common_switch8)
    __scatterload_copy                       0x0001da1d   Thumb Code    14  handlers.o(i.__scatterload_copy)
    __scatterload_null                       0x0001da2b   Thumb Code     2  handlers.o(i.__scatterload_null)
    __scatterload_zeroinit                   0x0001da2d   Thumb Code    14  handlers.o(i.__scatterload_zeroinit)
    action_tx_stop                           0x0001e325   Thumb Code    26  app_uart_fifo.o(i.action_tx_stop)
    app_error_handler                        0x0001e399   Thumb Code    18  app_error.o(i.app_error_handler)
    app_fifo_get                             0x0001e3c1   Thumb Code    34  app_fifo.o(i.app_fifo_get)
    app_fifo_put                             0x0001e3e3   Thumb Code    34  app_fifo.o(i.app_fifo_put)
    app_pwm_channel_duty_set                 0x0001e451   Thumb Code    32  app_pwm.o(i.app_pwm_channel_duty_set)
    app_pwm_channel_duty_ticks_set           0x0001e471   Thumb Code   134  app_pwm.o(i.app_pwm_channel_duty_ticks_set)
    app_pwm_enable                           0x0001e5c9   Thumb Code    18  app_pwm.o(i.app_pwm_enable)
    app_pwm_init                             0x0001e5dd   Thumb Code   364  app_pwm.o(i.app_pwm_init)
    ble_db_discovery_evt_register            0x0001e765   Thumb Code    66  ble_db_discovery.o(i.ble_db_discovery_evt_register)
    ble_db_discovery_init                    0x0001e7b1   Thumb Code    18  ble_db_discovery.o(i.ble_db_discovery_init)
    ble_db_discovery_on_ble_evt              0x0001e7c9   Thumb Code   156  ble_db_discovery.o(i.ble_db_discovery_on_ble_evt)
    ble_db_discovery_start                   0x0001e869   Thumb Code    86  ble_db_discovery.o(i.ble_db_discovery_start)
    client_handling_ble_evt_handler          0x0001eb3d   Thumb Code   286  client_handling.o(i.client_handling_ble_evt_handler)
    client_handling_create                   0x0001ec6d   Thumb Code    90  client_handling.o(i.client_handling_create)
    client_handling_destroy                  0x0001ecd1   Thumb Code    80  client_handling.o(i.client_handling_destroy)
    client_handling_dm_event_handler         0x0001ed35   Thumb Code    30  client_handling.o(i.client_handling_dm_event_handler)
    client_handling_init                     0x0001ed59   Thumb Code   134  client_handling.o(i.client_handling_init)
    debug_printf                             0x0001f111   Thumb Code    30  debug_util.o(i.debug_printf)
    dm_ble_evt_handler                       0x0001f4cd   Thumb Code   858  device_manager_central.o(i.dm_ble_evt_handler)
    dm_handle_initialize                     0x0001f83d   Thumb Code    22  device_manager_central.o(i.dm_handle_initialize)
    dm_init                                  0x0001f859   Thumb Code   170  device_manager_central.o(i.dm_init)
    dm_register                              0x0001fa91   Thumb Code    76  device_manager_central.o(i.dm_register)
    dm_security_setup_req                    0x0001fae9   Thumb Code   194  device_manager_central.o(i.dm_security_setup_req)
    initiate_security_request                0x0001fe1d   Thumb Code    86  device_manager_central.o(i.initiate_security_request)
    intern_softdevice_events_execute         0x0001fe79   Thumb Code   124  softdevice_handler.o(i.intern_softdevice_events_execute)
    main                                     0x00020029   Thumb Code   208  main.o(i.main)
    make_alarm                               0x00020175   Thumb Code    94  main.o(i.make_alarm)
    nrf_delay_ms                             0x00020235   Thumb Code    24  nrf_delay.o(i.nrf_delay_ms)
    nrf_drv_common_irq_enable                0x00020251   Thumb Code    78  nrf_drv_common.o(i.nrf_drv_common_irq_enable)
    nrf_drv_gpiote_init                      0x000202b1   Thumb Code    74  nrf_drv_gpiote.o(i.nrf_drv_gpiote_init)
    nrf_drv_gpiote_is_init                   0x00020305   Thumb Code    12  nrf_drv_gpiote.o(i.nrf_drv_gpiote_is_init)
    nrf_drv_gpiote_out_init                  0x00020315   Thumb Code   128  nrf_drv_gpiote.o(i.nrf_drv_gpiote_out_init)
    nrf_drv_gpiote_out_task_addr_get         0x000203a9   Thumb Code    16  nrf_drv_gpiote.o(i.nrf_drv_gpiote_out_task_addr_get)
    nrf_drv_gpiote_out_task_enable           0x000203bd   Thumb Code    38  nrf_drv_gpiote.o(i.nrf_drv_gpiote_out_task_enable)
    nrf_drv_gpiote_out_task_force            0x000203ed   Thumb Code    40  nrf_drv_gpiote.o(i.nrf_drv_gpiote_out_task_force)
    nrf_drv_gpiote_out_task_trigger          0x0002041d   Thumb Code    20  nrf_drv_gpiote.o(i.nrf_drv_gpiote_out_task_trigger)
    nrf_drv_gpiote_out_uninit                0x00020435   Thumb Code    40  nrf_drv_gpiote.o(i.nrf_drv_gpiote_out_uninit)
    nrf_drv_ppi_channel_alloc                0x00020465   Thumb Code   134  nrf_drv_ppi.o(i.nrf_drv_ppi_channel_alloc)
    nrf_drv_ppi_channel_assign               0x000204f5   Thumb Code    58  nrf_drv_ppi.o(i.nrf_drv_ppi_channel_assign)
    nrf_drv_ppi_channel_disable              0x00020535   Thumb Code    52  nrf_drv_ppi.o(i.nrf_drv_ppi_channel_disable)
    nrf_drv_ppi_channel_enable               0x0002056d   Thumb Code    52  nrf_drv_ppi.o(i.nrf_drv_ppi_channel_enable)
    nrf_drv_ppi_channel_free                 0x000205a5   Thumb Code   104  nrf_drv_ppi.o(i.nrf_drv_ppi_channel_free)
    nrf_drv_ppi_channels_include_in_group    0x00020615   Thumb Code   128  nrf_drv_ppi.o(i.nrf_drv_ppi_channels_include_in_group)
    nrf_drv_ppi_channels_remove_from_group   0x00020699   Thumb Code   128  nrf_drv_ppi.o(i.nrf_drv_ppi_channels_remove_from_group)
    nrf_drv_ppi_group_alloc                  0x0002071d   Thumb Code   136  nrf_drv_ppi.o(i.nrf_drv_ppi_group_alloc)
    nrf_drv_ppi_group_enable                 0x000207a9   Thumb Code    44  nrf_drv_ppi.o(i.nrf_drv_ppi_group_enable)
    nrf_drv_ppi_group_free                   0x000207d9   Thumb Code   122  nrf_drv_ppi.o(i.nrf_drv_ppi_group_free)
    nrf_drv_ppi_init                         0x0002085d   Thumb Code    20  nrf_drv_ppi.o(i.nrf_drv_ppi_init)
    nrf_drv_timer_clear                      0x00020875   Thumb Code     8  nrf_drv_timer.o(i.nrf_drv_timer_clear)
    nrf_drv_timer_compare                    0x0002087d   Thumb Code    42  nrf_drv_timer.o(i.nrf_drv_timer_compare)
    nrf_drv_timer_compare_event_address_get  0x000208a7   Thumb Code    14  nrf_drv_timer.o(i.nrf_drv_timer_compare_event_address_get)
    nrf_drv_timer_compare_int_disable        0x000208b5   Thumb Code    18  nrf_drv_timer.o(i.nrf_drv_timer_compare_int_disable)
    nrf_drv_timer_compare_int_enable         0x000208c7   Thumb Code    34  nrf_drv_timer.o(i.nrf_drv_timer_compare_int_enable)
    nrf_drv_timer_disable                    0x000208e9   Thumb Code    14  nrf_drv_timer.o(i.nrf_drv_timer_disable)
    nrf_drv_timer_enable                     0x000208fd   Thumb Code    16  nrf_drv_timer.o(i.nrf_drv_timer_enable)
    nrf_drv_timer_extended_compare           0x00020911   Thumb Code    46  nrf_drv_timer.o(i.nrf_drv_timer_extended_compare)
    nrf_drv_timer_init                       0x00020941   Thumb Code   152  nrf_drv_timer.o(i.nrf_drv_timer_init)
    nrf_drv_timer_uninit                     0x000209e5   Thumb Code    86  nrf_drv_timer.o(i.nrf_drv_timer_uninit)
    nrf_drv_timer_us_to_ticks                0x00020a49   Thumb Code    22  nrf_drv_timer.o(i.nrf_drv_timer_us_to_ticks)
    pstorage_access_status_get               0x00020e59   Thumb Code    30  pstorage.o(i.pstorage_access_status_get)
    pstorage_block_identifier_get            0x00020e81   Thumb Code    74  pstorage.o(i.pstorage_block_identifier_get)
    pstorage_clear                           0x00020ed5   Thumb Code   156  pstorage.o(i.pstorage_clear)
    pstorage_init                            0x00020fa9   Thumb Code    68  pstorage.o(i.pstorage_init)
    pstorage_load                            0x00020ff5   Thumb Code   158  pstorage.o(i.pstorage_load)
    pstorage_register                        0x0002109d   Thumb Code   170  pstorage.o(i.pstorage_register)
    pstorage_store                           0x00021151   Thumb Code   134  pstorage.o(i.pstorage_store)
    pstorage_sys_event_handler               0x000211e1   Thumb Code    72  pstorage.o(i.pstorage_sys_event_handler)
    pstorage_update                          0x0002122d   Thumb Code   134  pstorage.o(i.pstorage_update)
    pwm_ready_callback                       0x00021369   Thumb Code     8  main.o(i.pwm_ready_callback)
    pwm_ready_tick                           0x00021375   Thumb Code    52  app_pwm.o(i.pwm_ready_tick)
    pwm_set_value                            0x000213ad   Thumb Code    60  main.o(i.pwm_set_value)
    read_acc_other_device                    0x0002160d   Thumb Code    12  client_handling.o(i.read_acc_other_device)
    simple_uart_config                       0x00021695   Thumb Code    76  simple_uart.o(i.simple_uart_config)
    simple_uart_put                          0x000216f5   Thumb Code    18  simple_uart.o(i.simple_uart_put)
    simple_uart_putstring                    0x00021711   Thumb Code    24  simple_uart.o(i.simple_uart_putstring)
    softdevice_assertion_handler             0x00021771   Thumb Code    12  softdevice_handler.o(i.softdevice_assertion_handler)
    softdevice_ble_evt_handler_set           0x0002177d   Thumb Code    16  softdevice_handler.o(i.softdevice_ble_evt_handler_set)
    softdevice_handler_init                  0x00021791   Thumb Code    40  softdevice_handler.o(i.softdevice_handler_init)
    softdevice_sys_evt_handler_set           0x000217c1   Thumb Code    16  softdevice_handler.o(i.softdevice_sys_evt_handler_set)
    m_pwm_PWM1_timer                         0x00021b4c   Data           8  main.o(.constdata)
    PWM1                                     0x00021b54   Data           8  main.o(.constdata)
    m_service_context_store                  0x00021b8c   Data          16  device_manager_central.o(.constdata)
    m_service_context_load                   0x00021b9c   Data          16  device_manager_central.o(.constdata)
    m_service_context_apply                  0x00021bac   Data          16  device_manager_central.o(.constdata)
    Region$$Table$$Base                      0x00021bf8   Number         0  anon$$obj.o(Region$$Table)
    Region$$Table$$Limit                     0x00021c18   Number         0  anon$$obj.o(Region$$Table)
    SystemCoreClock                          0x20002810   Data           4  system_nrf51.o(.data)
    m_pwm_ready_counter                      0x20002874   Data           1  app_pwm.o(.data)
    m_pwm_PWM1_cb                            0x20002c58   Data          36  main.o(.bss)
    __initial_sp                             0x20003860   Data           0  arm_startup_nrf51.o(STACK)



==============================================================================

Memory Map of the image

  Image Entry point : 0x0001d0c1

  Load Region LR_IROM1 (Base: 0x0001d000, Size: 0x00004ca8, Max: 0x00023000, ABSOLUTE)

    Execution Region ER_IROM1 (Base: 0x0001d000, Size: 0x00004c18, Max: 0x00023000, ABSOLUTE)

    Base Addr    Size         Type   Attr      Idx    E Section Name        Object

    0x0001d000   0x000000c0   Data   RO          869    RESET               arm_startup_nrf51.o
    0x0001d0c0   0x00000000   Code   RO         2538  * .ARM.Collect$$$$00000000  mc_p.l(entry.o)
    0x0001d0c0   0x00000004   Code   RO         2816    .ARM.Collect$$$$00000001  mc_p.l(entry2.o)
    0x0001d0c4   0x00000004   Code   RO         2819    .ARM.Collect$$$$00000004  mc_p.l(entry5.o)
    0x0001d0c8   0x00000000   Code   RO         2821    .ARM.Collect$$$$00000008  mc_p.l(entry7b.o)
    0x0001d0c8   0x00000000   Code   RO         2823    .ARM.Collect$$$$0000000A  mc_p.l(entry8b.o)
    0x0001d0c8   0x00000008   Code   RO         2824    .ARM.Collect$$$$0000000B  mc_p.l(entry9a.o)
    0x0001d0d0   0x00000000   Code   RO         2826    .ARM.Collect$$$$0000000D  mc_p.l(entry10a.o)
    0x0001d0d0   0x00000000   Code   RO         2828    .ARM.Collect$$$$0000000F  mc_p.l(entry11a.o)
    0x0001d0d0   0x00000004   Code   RO         2817    .ARM.Collect$$$$00002712  mc_p.l(entry2.o)
    0x0001d0d4   0x0000001e   Code   RO         1912    .emb_text           nrf_delay.o
    0x0001d0f2   0x00000002   PAD
    0x0001d0f4   0x00000038   Code   RO          870    .text               arm_startup_nrf51.o
    0x0001d12c   0x0000002c   Code   RO         2541    .text               mc_p.l(uidiv.o)
    0x0001d158   0x00000028   Code   RO         2543    .text               mc_p.l(idiv.o)
    0x0001d180   0x00000024   Code   RO         2545    .text               mc_p.l(memcpya.o)
    0x0001d1a4   0x00000024   Code   RO         2547    .text               mc_p.l(memseta.o)
    0x0001d1c8   0x0000001a   Code   RO         2551    .text               mc_p.l(memcmp.o)
    0x0001d1e2   0x00000060   Code   RO         2830    .text               mc_p.l(uldiv.o)
    0x0001d242   0x00000000   Code   RO         2832    .text               mc_p.l(iusefp.o)
    0x0001d242   0x00000002   PAD
    0x0001d244   0x00000164   Code   RO         2833    .text               mf_p.l(dadd.o)
    0x0001d3a8   0x000000d0   Code   RO         2835    .text               mf_p.l(dmul.o)
    0x0001d478   0x000000f0   Code   RO         2837    .text               mf_p.l(ddiv.o)
    0x0001d568   0x00000040   Code   RO         2839    .text               mf_p.l(dfixul.o)
    0x0001d5a8   0x00000028   Code   RO         2841    .text               mf_p.l(cdrcmple.o)
    0x0001d5d0   0x00000024   Code   RO         2843    .text               mc_p.l(init.o)
    0x0001d5f4   0x00000020   Code   RO         2845    .text               mc_p.l(llshl.o)
    0x0001d614   0x00000022   Code   RO         2847    .text               mc_p.l(llushr.o)
    0x0001d636   0x00000026   Code   RO         2849    .text               mc_p.l(llsshr.o)
    0x0001d65c   0x000000be   Code   RO         2851    .text               mf_p.l(depilogue.o)
    0x0001d71a   0x00000002   PAD
    0x0001d71c   0x000000fc   Code   RO         1729    i.GPIOTE_IRQHandler  nrf_drv_gpiote.o
    0x0001d818   0x0000002c   Code   RO          708    i.SPI0_TWI0_IRQHandler  spi_master.o
    0x0001d844   0x00000024   Code   RO         2482    i.SWI2_IRQHandler   softdevice_handler.o
    0x0001d868   0x00000054   Code   RO          877    i.SystemInit        system_nrf51.o
    0x0001d8bc   0x0000004c   Code   RO         2077    i.TIMER1_IRQHandler  nrf_drv_timer.o
    0x0001d908   0x00000080   Code   RO         1361    i.UART0_IRQHandler  app_uart_fifo.o
    0x0001d988   0x00000028   Code   RO         2790    i.__0sprintf        mc_p.l(printfa.o)
    0x0001d9b0   0x00000024   Code   RO         2794    i.__0vsprintf       mc_p.l(printfa.o)
    0x0001d9d4   0x0000002e   Code   RO         2853    i.__ARM_clz         mf_p.l(depilogue.o)
    0x0001da02   0x0000001a   Code   RO           90    i.__ARM_common_switch8  client_handling.o
    0x0001da1c   0x0000000e   Code   RO         2857    i.__scatterload_copy  mc_p.l(handlers.o)
    0x0001da2a   0x00000002   Code   RO         2858    i.__scatterload_null  mc_p.l(handlers.o)
    0x0001da2c   0x0000000e   Code   RO         2859    i.__scatterload_zeroinit  mc_p.l(handlers.o)
    0x0001da3a   0x00000002   PAD
    0x0001da3c   0x00000158   Code   RO         2795    i._fp_digits        mc_p.l(printfa.o)
    0x0001db94   0x000006ec   Code   RO         2796    i._printf_core      mc_p.l(printfa.o)
    0x0001e280   0x00000020   Code   RO         2797    i._printf_post_padding  mc_p.l(printfa.o)
    0x0001e2a0   0x0000002c   Code   RO         2798    i._printf_pre_padding  mc_p.l(printfa.o)
    0x0001e2cc   0x0000000a   Code   RO         2800    i._sputc            mc_p.l(printfa.o)
    0x0001e2d6   0x00000002   PAD
    0x0001e2d8   0x0000004c   Code   RO         1362    i.action_tx_send    app_uart_fifo.o
    0x0001e324   0x00000024   Code   RO         1363    i.action_tx_stop    app_uart_fifo.o
    0x0001e348   0x00000020   Code   RO         1364    i.action_uart_deactivate  app_uart_fifo.o
    0x0001e368   0x0000002e   Code   RO          228    i.adv_report_parse  main.o
    0x0001e396   0x00000002   PAD
    0x0001e398   0x0000001c   Code   RO         2231    i.app_error_handler  app_error.o
    0x0001e3b4   0x0000000c   Code   RO         1099    i.app_evt_notify    device_manager_central.o
    0x0001e3c0   0x00000022   Code   RO         2253    i.app_fifo_get      app_fifo.o
    0x0001e3e2   0x00000022   Code   RO         2255    i.app_fifo_put      app_fifo.o
    0x0001e404   0x0000002c   Code   RO         1465    i.app_notify        pstorage.o
    0x0001e430   0x00000020   Code   RO         1466    i.app_notify_error_state_transit  pstorage.o
    0x0001e450   0x00000020   Code   RO         2288    i.app_pwm_channel_duty_set  app_pwm.o
    0x0001e470   0x0000008c   Code   RO         2290    i.app_pwm_channel_duty_ticks_set  app_pwm.o
    0x0001e4fc   0x000000cc   Code   RO         2291    i.app_pwm_channel_init  app_pwm.o
    0x0001e5c8   0x00000012   Code   RO         2294    i.app_pwm_enable    app_pwm.o
    0x0001e5da   0x00000002   PAD
    0x0001e5dc   0x0000017c   Code   RO         2295    i.app_pwm_init      app_pwm.o
    0x0001e758   0x0000000c   Code   RO         1936    i.are_app_channels  nrf_drv_ppi.o
    0x0001e764   0x0000004c   Code   RO          970    i.ble_db_discovery_evt_register  ble_db_discovery.o
    0x0001e7b0   0x00000018   Code   RO          971    i.ble_db_discovery_init  ble_db_discovery.o
    0x0001e7c8   0x000000a0   Code   RO          972    i.ble_db_discovery_on_ble_evt  ble_db_discovery.o
    0x0001e868   0x00000060   Code   RO          973    i.ble_db_discovery_start  ble_db_discovery.o
    0x0001e8c8   0x00000016   Code   RO          230    i.ble_evt_dispatch  main.o
    0x0001e8de   0x00000002   PAD
    0x0001e8e0   0x00000068   Code   RO          231    i.ble_stack_init    main.o
    0x0001e948   0x0000001c   Code   RO         1730    i.channel_free      nrf_drv_gpiote.o
    0x0001e964   0x00000044   Code   RO         1731    i.channel_port_alloc  nrf_drv_gpiote.o
    0x0001e9a8   0x00000010   Code   RO         1732    i.channel_port_get  nrf_drv_gpiote.o
    0x0001e9b8   0x00000038   Code   RO          974    i.characteristics_discover  ble_db_discovery.o
    0x0001e9f0   0x00000104   Code   RO         1467    i.clear_operation_execute  pstorage.o
    0x0001eaf4   0x00000024   Code   RO         1468    i.clear_post_processing_run  pstorage.o
    0x0001eb18   0x00000024   Code   RO            4    i.client_find       client_handling.o
    0x0001eb3c   0x00000130   Code   RO            5    i.client_handling_ble_evt_handler  client_handling.o
    0x0001ec6c   0x00000064   Code   RO            7    i.client_handling_create  client_handling.o
    0x0001ecd0   0x00000064   Code   RO            8    i.client_handling_destroy  client_handling.o
    0x0001ed34   0x00000024   Code   RO            9    i.client_handling_dm_event_handler  client_handling.o
    0x0001ed58   0x000000a0   Code   RO           10    i.client_handling_init  client_handling.o
    0x0001edf8   0x00000038   Code   RO         1469    i.cmd_process       pstorage.o
    0x0001ee30   0x00000020   Code   RO         1470    i.cmd_queue_element_init  pstorage.o
    0x0001ee50   0x0000004c   Code   RO         1471    i.cmd_queue_enqueue  pstorage.o
    0x0001ee9c   0x0000003c   Code   RO         1472    i.command_end_procedure_run  pstorage.o
    0x0001eed8   0x00000040   Code   RO         1100    i.connection_instance_find  device_manager_central.o
    0x0001ef18   0x00000024   Code   RO         1101    i.connection_instance_init  device_manager_central.o
    0x0001ef3c   0x00000044   Code   RO         1937    i.current_int_priority_get  nrf_drv_ppi.o
    0x0001ef80   0x00000054   Code   RO         1473    i.data_page_erase_state_run  pstorage.o
    0x0001efd4   0x00000028   Code   RO         1474    i.data_to_swap_write_state_run  pstorage.o
    0x0001effc   0x000000b0   Code   RO           11    i.db_discovery_acc_evt_handler  client_handling.o
    0x0001f0ac   0x00000064   Code   RO           12    i.db_discovery_evt_handler  client_handling.o
    0x0001f110   0x0000001e   Code   RO          684    i.debug_printf      debug_util.o
    0x0001f12e   0x00000084   Code   RO          975    i.descriptors_discover  ble_db_discovery.o
    0x0001f1b2   0x00000002   PAD
    0x0001f1b4   0x000000b4   Code   RO         1102    i.device_context_store  device_manager_central.o
    0x0001f268   0x00000054   Code   RO         1103    i.device_instance_allocate  device_manager_central.o
    0x0001f2bc   0x000000b8   Code   RO          232    i.device_manager_event_handler  main.o
    0x0001f374   0x0000009c   Code   RO          233    i.device_manager_init  main.o
    0x0001f410   0x0000006c   Code   RO          976    i.discovery_complete_evt_trigger  ble_db_discovery.o
    0x0001f47c   0x00000050   Code   RO          977    i.discovery_error_evt_trigger  ble_db_discovery.o
    0x0001f4cc   0x00000370   Code   RO         1109    i.dm_ble_evt_handler  device_manager_central.o
    0x0001f83c   0x0000001c   Code   RO         1114    i.dm_handle_initialize  device_manager_central.o
    0x0001f858   0x000000c0   Code   RO         1115    i.dm_init           device_manager_central.o
    0x0001f918   0x00000178   Code   RO         1118    i.dm_pstorage_cb_handler  device_manager_central.o
    0x0001fa90   0x00000058   Code   RO         1119    i.dm_register       device_manager_central.o
    0x0001fae8   0x000000d4   Code   RO         1120    i.dm_security_setup_req  device_manager_central.o
    0x0001fbbc   0x00000020   Code   RO         1475    i.flash_api_err_code_process  pstorage.o
    0x0001fbdc   0x00000080   Code   RO         1476    i.flash_operation_success_run  pstorage.o
    0x0001fc5c   0x0000000a   Code   RO         1477    i.flash_page_erase  pstorage.o
    0x0001fc66   0x0000000a   Code   RO         1478    i.flash_write       pstorage.o
    0x0001fc70   0x00000004   Code   RO         1126    i.gattc_context_apply  device_manager_central.o
    0x0001fc74   0x00000004   Code   RO         1127    i.gattc_context_load  device_manager_central.o
    0x0001fc78   0x00000004   Code   RO         1128    i.gattc_context_store  device_manager_central.o
    0x0001fc7c   0x00000040   Code   RO         1129    i.gatts_context_apply  device_manager_central.o
    0x0001fcbc   0x00000030   Code   RO         1130    i.gatts_context_load  device_manager_central.o
    0x0001fcec   0x000000a0   Code   RO         1131    i.gatts_context_store  device_manager_central.o
    0x0001fd8c   0x00000008   Code   RO         1132    i.gattsc_context_apply  device_manager_central.o
    0x0001fd94   0x00000008   Code   RO         1133    i.gattsc_context_load  device_manager_central.o
    0x0001fd9c   0x00000008   Code   RO         1134    i.gattsc_context_store  device_manager_central.o
    0x0001fda4   0x00000078   Code   RO         1479    i.head_restore_state_run  pstorage.o
    0x0001fe1c   0x0000005c   Code   RO         1135    i.initiate_security_request  device_manager_central.o
    0x0001fe78   0x00000080   Code   RO         2483    i.intern_softdevice_events_execute  softdevice_handler.o
    0x0001fef8   0x00000018   Code   RO         1938    i.is_allocated_channel  nrf_drv_ppi.o
    0x0001ff10   0x00000018   Code   RO         1939    i.is_allocated_group  nrf_drv_ppi.o
    0x0001ff28   0x0000000e   Code   RO         1940    i.is_app_channel    nrf_drv_ppi.o
    0x0001ff36   0x0000000c   Code   RO         1941    i.is_app_group      nrf_drv_ppi.o
    0x0001ff42   0x00000042   Code   RO          978    i.is_desc_discovery_reqd  ble_db_discovery.o
    0x0001ff84   0x00000048   Code   RO          878    i.is_manual_peripheral_setup_needed  system_nrf51.o
    0x0001ffcc   0x00000044   Code   RO         1480    i.is_page_erase_required  pstorage.o
    0x00020010   0x0000000c   Code   RO         1942    i.is_programmable_app_channel  nrf_drv_ppi.o
    0x0002001c   0x0000000c   Code   RO         1481    i.is_word_aligned   pstorage.o
    0x00020028   0x00000134   Code   RO          234    i.main              main.o
    0x0002015c   0x00000018   Code   RO         1482    i.main_state_err_busy_process  pstorage.o
    0x00020174   0x00000070   Code   RO          235    i.make_alarm        main.o
    0x000201e4   0x00000004   Code   RO         1136    i.no_service_context_apply  device_manager_central.o
    0x000201e8   0x00000004   Code   RO         1137    i.no_service_context_load  device_manager_central.o
    0x000201ec   0x00000004   Code   RO         1138    i.no_service_context_store  device_manager_central.o
    0x000201f0   0x00000042   Code   RO           13    i.notif_enable      client_handling.o
    0x00020232   0x00000002   PAD
    0x00020234   0x0000001c   Code   RO         1913    i.nrf_delay_ms      nrf_delay.o
    0x00020250   0x00000060   Code   RO         1709    i.nrf_drv_common_irq_enable  nrf_drv_common.o
    0x000202b0   0x00000054   Code   RO         1739    i.nrf_drv_gpiote_init  nrf_drv_gpiote.o
    0x00020304   0x00000010   Code   RO         1740    i.nrf_drv_gpiote_is_init  nrf_drv_gpiote.o
    0x00020314   0x00000094   Code   RO         1742    i.nrf_drv_gpiote_out_init  nrf_drv_gpiote.o
    0x000203a8   0x00000014   Code   RO         1744    i.nrf_drv_gpiote_out_task_addr_get  nrf_drv_gpiote.o
    0x000203bc   0x00000030   Code   RO         1746    i.nrf_drv_gpiote_out_task_enable  nrf_drv_gpiote.o
    0x000203ec   0x00000030   Code   RO         1747    i.nrf_drv_gpiote_out_task_force  nrf_drv_gpiote.o
    0x0002041c   0x00000018   Code   RO         1748    i.nrf_drv_gpiote_out_task_trigger  nrf_drv_gpiote.o
    0x00020434   0x00000030   Code   RO         1750    i.nrf_drv_gpiote_out_uninit  nrf_drv_gpiote.o
    0x00020464   0x00000090   Code   RO         1943    i.nrf_drv_ppi_channel_alloc  nrf_drv_ppi.o
    0x000204f4   0x00000040   Code   RO         1944    i.nrf_drv_ppi_channel_assign  nrf_drv_ppi.o
    0x00020534   0x00000038   Code   RO         1945    i.nrf_drv_ppi_channel_disable  nrf_drv_ppi.o
    0x0002056c   0x00000038   Code   RO         1946    i.nrf_drv_ppi_channel_enable  nrf_drv_ppi.o
    0x000205a4   0x00000070   Code   RO         1947    i.nrf_drv_ppi_channel_free  nrf_drv_ppi.o
    0x00020614   0x00000084   Code   RO         1948    i.nrf_drv_ppi_channels_include_in_group  nrf_drv_ppi.o
    0x00020698   0x00000084   Code   RO         1949    i.nrf_drv_ppi_channels_remove_from_group  nrf_drv_ppi.o
    0x0002071c   0x0000008c   Code   RO         1950    i.nrf_drv_ppi_group_alloc  nrf_drv_ppi.o
    0x000207a8   0x00000030   Code   RO         1952    i.nrf_drv_ppi_group_enable  nrf_drv_ppi.o
    0x000207d8   0x00000084   Code   RO         1953    i.nrf_drv_ppi_group_free  nrf_drv_ppi.o
    0x0002085c   0x00000018   Code   RO         1954    i.nrf_drv_ppi_init  nrf_drv_ppi.o
    0x00020874   0x00000008   Code   RO         2081    i.nrf_drv_timer_clear  nrf_drv_timer.o
    0x0002087c   0x0000002a   Code   RO         2082    i.nrf_drv_timer_compare  nrf_drv_timer.o
    0x000208a6   0x0000000e   Code   RO         2083    i.nrf_drv_timer_compare_event_address_get  nrf_drv_timer.o
    0x000208b4   0x00000012   Code   RO         2084    i.nrf_drv_timer_compare_int_disable  nrf_drv_timer.o
    0x000208c6   0x00000022   Code   RO         2085    i.nrf_drv_timer_compare_int_enable  nrf_drv_timer.o
    0x000208e8   0x00000014   Code   RO         2086    i.nrf_drv_timer_disable  nrf_drv_timer.o
    0x000208fc   0x00000014   Code   RO         2087    i.nrf_drv_timer_enable  nrf_drv_timer.o
    0x00020910   0x0000002e   Code   RO         2089    i.nrf_drv_timer_extended_compare  nrf_drv_timer.o
    0x0002093e   0x00000002   PAD
    0x00020940   0x000000a4   Code   RO         2091    i.nrf_drv_timer_init  nrf_drv_timer.o
    0x000209e4   0x00000064   Code   RO         2096    i.nrf_drv_timer_uninit  nrf_drv_timer.o
    0x00020a48   0x00000016   Code   RO         2097    i.nrf_drv_timer_us_to_ticks  nrf_drv_timer.o
    0x00020a5e   0x00000002   PAD
    0x00020a60   0x00000020   Code   RO         1752    i.nrf_gpio_cfg_sense_set  nrf_drv_gpiote.o
    0x00020a80   0x00000010   Code   RO          709    i.nrf_gpio_pin_set  spi_master.o
    0x00020a90   0x00000014   Code   RO         1753    i.nrf_gpiote_event_is_set  nrf_drv_gpiote.o
    0x00020aa4   0x000000b4   Code   RO          236    i.on_ble_evt        main.o
    0x00020b58   0x000000cc   Code   RO          979    i.on_characteristic_discovery_rsp  ble_db_discovery.o
    0x00020c24   0x000000a0   Code   RO          980    i.on_descriptor_discovery_rsp  ble_db_discovery.o
    0x00020cc4   0x0000005c   Code   RO          981    i.on_srv_disc_completion  ble_db_discovery.o
    0x00020d20   0x00000088   Code   RO         1372    i.on_uart_event     app_uart_fifo.o
    0x00020da8   0x00000038   Code   RO         2297    i.pan73_workaround  app_pwm.o
    0x00020de0   0x00000034   Code   RO         1139    i.peer_instance_init  device_manager_central.o
    0x00020e14   0x0000002c   Code   RO          982    i.pending_user_evts_send  ble_db_discovery.o
    0x00020e40   0x00000018   Code   RO         1755    i.pin_in_use_by_te  nrf_drv_gpiote.o
    0x00020e58   0x00000028   Code   RO         1483    i.pstorage_access_status_get  pstorage.o
    0x00020e80   0x00000054   Code   RO         1484    i.pstorage_block_identifier_get  pstorage.o
    0x00020ed4   0x000000a4   Code   RO         1485    i.pstorage_clear    pstorage.o
    0x00020f78   0x00000024   Code   RO         1486    i.pstorage_flash_page_end  pstorage.o
    0x00020f9c   0x0000000a   Code   RO         1487    i.pstorage_flash_page_size  pstorage.o
    0x00020fa6   0x00000002   PAD
    0x00020fa8   0x0000004c   Code   RO         1488    i.pstorage_init     pstorage.o
    0x00020ff4   0x000000a8   Code   RO         1489    i.pstorage_load     pstorage.o
    0x0002109c   0x000000b4   Code   RO         1490    i.pstorage_register  pstorage.o
    0x00021150   0x00000090   Code   RO         1491    i.pstorage_store    pstorage.o
    0x000211e0   0x0000004c   Code   RO         1492    i.pstorage_sys_event_handler  pstorage.o
    0x0002122c   0x00000090   Code   RO         1493    i.pstorage_update   pstorage.o
    0x000212bc   0x00000018   Code   RO         2298    i.pwm_channel_ppi_disable  app_pwm.o
    0x000212d4   0x00000080   Code   RO         2299    i.pwm_dealloc       app_pwm.o
    0x00021354   0x00000014   Code   RO         2300    i.pwm_ppi_disable   app_pwm.o
    0x00021368   0x0000000c   Code   RO          237    i.pwm_ready_callback  main.o
    0x00021374   0x00000038   Code   RO         2301    i.pwm_ready_tick    app_pwm.o
    0x000213ac   0x00000044   Code   RO          238    i.pwm_set_value     main.o
    0x000213f0   0x00000066   Code   RO         2302    i.pwm_transition_0or100_to_0or100  app_pwm.o
    0x00021456   0x00000002   PAD
    0x00021458   0x0000008c   Code   RO         2303    i.pwm_transition_0or100_to_n  app_pwm.o
    0x000214e4   0x00000088   Code   RO         2304    i.pwm_transition_n_to_0or100  app_pwm.o
    0x0002156c   0x000000a0   Code   RO         2305    i.pwm_transition_n_to_m  app_pwm.o
    0x0002160c   0x00000010   Code   RO           15    i.read_acc_other_device  client_handling.o
    0x0002161c   0x0000003c   Code   RO          983    i.registered_handler_get  ble_db_discovery.o
    0x00021658   0x0000003c   Code   RO          239    i.scan_start        main.o
    0x00021694   0x00000060   Code   RO          633    i.simple_uart_config  simple_uart.o
    0x000216f4   0x0000001c   Code   RO          636    i.simple_uart_put   simple_uart.o
    0x00021710   0x00000018   Code   RO          637    i.simple_uart_putstring  simple_uart.o
    0x00021728   0x00000048   Code   RO         1494    i.sm_state_change   pstorage.o
    0x00021770   0x0000000c   Code   RO         2484    i.softdevice_assertion_handler  softdevice_handler.o
    0x0002177c   0x00000014   Code   RO         2485    i.softdevice_ble_evt_handler_set  softdevice_handler.o
    0x00021790   0x00000030   Code   RO         2486    i.softdevice_handler_init  softdevice_handler.o
    0x000217c0   0x00000014   Code   RO         2488    i.softdevice_sys_evt_handler_set  softdevice_handler.o
    0x000217d4   0x00000028   Code   RO          711    i.spi_master_buffer_release  spi_master.o
    0x000217fc   0x00000010   Code   RO          713    i.spi_master_get_instance  spi_master.o
    0x0002180c   0x000000b4   Code   RO          717    i.spi_master_send_recv_irq  spi_master.o
    0x000218c0   0x00000034   Code   RO          718    i.spi_master_signal_evt  spi_master.o
    0x000218f4   0x00000064   Code   RO         1495    i.state_data_erase_swap_entry_run  pstorage.o
    0x00021958   0x00000010   Code   RO         1496    i.state_erase_data_page_entry_run  pstorage.o
    0x00021968   0x00000028   Code   RO         1497    i.state_restore_head_entry_run  pstorage.o
    0x00021990   0x0000004c   Code   RO         1498    i.state_restore_tail_entry_run  pstorage.o
    0x000219dc   0x00000020   Code   RO         1499    i.state_swap_erase_entry_run  pstorage.o
    0x000219fc   0x00000030   Code   RO         1500    i.state_write_data_swap_entry_run  pstorage.o
    0x00021a2c   0x00000004   Code   RO         1140    i.storage_operation_dummy_handler  device_manager_central.o
    0x00021a30   0x0000005c   Code   RO         1501    i.store_cmd_flash_write_execute  pstorage.o
    0x00021a8c   0x0000001c   Code   RO         1502    i.swap_erase_state_run  pstorage.o
    0x00021aa8   0x00000018   Code   RO         1503    i.swap_sub_state_err_busy_process  pstorage.o
    0x00021ac0   0x00000014   Code   RO         1504    i.swap_sub_state_state_change  pstorage.o
    0x00021ad4   0x00000028   Code   RO          240    i.sys_evt_dispatch  main.o
    0x00021afc   0x0000001c   Code   RO         1505    i.tail_restore_state_run  pstorage.o
    0x00021b18   0x00000014   Code   RO         1141    i.update_status_bit_reset  device_manager_central.o
    0x00021b2c   0x00000020   Data   RO           17    .constdata          client_handling.o
    0x00021b4c   0x00000008   Data   RO          243    .constdata          main.o
    0x00021b54   0x00000034   Data   RO          244    .constdata          main.o
    0x00021b88   0x00000004   Data   RO          720    .constdata          spi_master.o
    0x00021b8c   0x00000030   Data   RO         1143    .constdata          device_manager_central.o
    0x00021bbc   0x00000028   Data   RO         1507    .constdata          pstorage.o
    0x00021be4   0x00000008   Data   RO         2098    .constdata          nrf_drv_timer.o
    0x00021bec   0x0000000c   Data   RO         2306    .constdata          app_pwm.o
    0x00021bf8   0x00000020   Data   RO         2855    Region$$Table       anon$$obj.o


    Execution Region RW_IRAM1 (Base: 0x20002800, Size: 0x00001060, Max: 0x00005800, ABSOLUTE)

    Base Addr    Size         Type   Attr      Idx    E Section Name        Object

    0x20002800   0x00000003   Data   RW           19    .data               client_handling.o
    0x20002803   0x00000001   PAD
    0x20002804   0x0000000c   Data   RW          245    .data               main.o
    0x20002810   0x00000004   Data   RW          879    .data               system_nrf51.o
    0x20002814   0x00000010   Data   RW          985    .data               ble_db_discovery.o
    0x20002824   0x00000010   Data   RW         1145    .data               device_manager_central.o
    0x20002834   0x00000008   Data   RW         1375    .data               app_uart_fifo.o
    0x2000283c   0x00000024   Data   RW         1508    .data               pstorage.o
    0x20002860   0x00000008   Data   RW         1956    .data               nrf_drv_ppi.o
    0x20002868   0x0000000c   Data   RW         2099    .data               nrf_drv_timer.o
    0x20002874   0x00000008   Data   RW         2307    .data               app_pwm.o
    0x2000287c   0x00000014   Data   RW         2489    .data               softdevice_handler.o
    0x20002890   0x00000380   Zero   RW           16    .bss                client_handling.o
    0x20002c10   0x00000048   Zero   RW          241    .bss                main.o
    0x20002c58   0x00000024   Zero   RW          242    .bss                main.o
    0x20002c7c   0x00000028   Zero   RW          719    .bss                spi_master.o
    0x20002ca4   0x00000080   Zero   RW          984    .bss                ble_db_discovery.o
    0x20002d24   0x00000283   Zero   RW         1142    .bss                device_manager_central.o
    0x20002fa7   0x00000001   PAD
    0x20002fa8   0x00000020   Zero   RW         1373    .bss                app_uart_fifo.o
    0x20002fc8   0x00000060   Zero   RW         1506    .bss                pstorage.o
    0x20003028   0x00000038   Zero   RW         1756    .bss                nrf_drv_gpiote.o
    0x20003060   0x00000800   Zero   RW          867    STACK               arm_startup_nrf51.o


==============================================================================

Image component sizes


      Code (inc. data)   RO Data    RW Data    ZI Data      Debug   Object Name

         0          0          0          0          0       2540   acc_lis2.o
        28         10          0          0          0       7704   app_error.o
        68          0          0          0          0       2734   app_fifo.o
      1596         74         12          8          0      23888   app_pwm.o
       408         86          0          8         32      17012   app_uart_fifo.o
        56         18        192          0       2048        716   arm_startup_nrf51.o
      1358         78          0         16        128      15735   ble_db_discovery.o
      1120        128         32          3        896      70171   client_handling.o
        30          0          0          0          0       1263   debug_util.o
      2640        200         48         16        643      26300   device_manager_central.o
      1292        196         60         12        108      32807   main.o
        58          4          0          0          0       1643   nrf_delay.o
        96         18          0          0          0        824   nrf_drv_common.o
       876        128          0          0         56      20807   nrf_drv_gpiote.o
      1206         78          0          8          0      28269   nrf_drv_ppi.o
       564         46          8         12          0      23917   nrf_drv_timer.o
      2822        264         40         36         96      36034   pstorage.o
       148         30          0          0          0       5627   simple_uart.o
       264         24          0         20          0       6308   softdevice_handler.o
       348         26          4          0         40       7267   spi_master.o
       156         26          0          4          0       2183   system_nrf51.o

    ----------------------------------------------------------------------
     15154       1434        428        144       4048     333749   Object Totals
         0          0         32          0          0          0   (incl. Generated)
        20          0          0          1          1          0   (incl. Padding)

    ----------------------------------------------------------------------

      Code (inc. data)   RO Data    RW Data    ZI Data      Debug   Library Member Name

         0          0          0          0          0          0   entry.o
         0          0          0          0          0          0   entry10a.o
         0          0          0          0          0          0   entry11a.o
         8          4          0          0          0          0   entry2.o
         4          0          0          0          0          0   entry5.o
         0          0          0          0          0          0   entry7b.o
         0          0          0          0          0          0   entry8b.o
         8          4          0          0          0          0   entry9a.o
        30          0          0          0          0          0   handlers.o
        40          0          0          0          0         72   idiv.o
        36          8          0          0          0         68   init.o
         0          0          0          0          0          0   iusefp.o
        32          0          0          0          0         68   llshl.o
        38          0          0          0          0         68   llsshr.o
        34          0          0          0          0         68   llushr.o
        26          0          0          0          0         72   memcmp.o
        36          0          0          0          0         60   memcpya.o
        36          0          0          0          0        100   memseta.o
      2278        100          0          0          0        544   printfa.o
        44          0          0          0          0         72   uidiv.o
        96          0          0          0          0         84   uldiv.o
        40          2          0          0          0         68   cdrcmple.o
       356          4          0          0          0        140   dadd.o
       240          6          0          0          0         84   ddiv.o
       236          0          0          0          0        216   depilogue.o
        64         10          0          0          0         68   dfixul.o
       208          6          0          0          0         88   dmul.o

    ----------------------------------------------------------------------
      3898        144          0          0          0       1940   Library Totals
         8          0          0          0          0          0   (incl. Padding)

    ----------------------------------------------------------------------

      Code (inc. data)   RO Data    RW Data    ZI Data      Debug   Library Name

      2746        116          0          0          0       1276   mc_p.l
      1144         28          0          0          0        664   mf_p.l

    ----------------------------------------------------------------------
      3898        144          0          0          0       1940   Library Totals

    ----------------------------------------------------------------------

==============================================================================


      Code (inc. data)   RO Data    RW Data    ZI Data      Debug   

     19052       1578        428        144       4048     326497   Grand Totals
     19052       1578        428        144       4048     326497   ELF Image Totals
     19052       1578        428        144          0          0   ROM Totals

==============================================================================

    Total RO  Size (Code + RO Data)                19480 (  19.02kB)
    Total RW  Size (RW Data + ZI Data)              4192 (   4.09kB)
    Total ROM Size (Code + RO Data + RW Data)      19624 (  19.16kB)

==============================================================================

